:20000000004B002041420100FDC90110FDC90110FDC90110FDC90110FDC90110FDC90110E7
:1C002000FDC90110FDC90110FDC90110FDC90110FDC90110FDC901103BCA0110A4
:20003C00AD040021490400217D04002181040021110500219105002141060021F8B51047C2
:20005C00F8B50E4600210125AD0430470A48037800F00FF89B070BD0124C2078FF2807D0DF
:20007C00FF2121700E490F24240220436031C882F8BDF8B5014800476B020021E54C000014
:20009C00094801E00848000C064C05492278FF2A01D1CA7A22706031C8827046801C004737
:2000BC0000620840A4060021070F0808F0B4084770B503461546012906D0002906D0114A73
:2000DC002846FFF7BBFF70BD0F4800E00F480524834203D84008641E002CF9DCE340012053
:2000FC0040031818820B012907D00649002380312846FFF7A5FFE0B270BD0249044B6C31C2
:20011C00F6E70000835C0000A0BC862300830D2374060021F8B51A4E0546716B1948CC0942
:20013C00E401002D11D01849097802290FD0007B044372B60120154F4002B8471148203863
:20015C000088C109C90704D016E0C07AF0E7407BEEE70F497463CC61400AC0070CD001208C
:20017C008003316B002D01D0014300E08143084631630749403948630020B84762B6F8BD1C
:20019C0080020021880000219B0200217B3F00004040044010B5224A00215161214989685C
:2001BC00C90009D42149204BCA0598424B6B01D8134300E093434B631D49FFF777FF10BD17
:2001DC0038B51A4D287F002827D11A480088C009C00722D1124C606900281ED1684600F09F
:2001FC0045F868460078012817D168464078102813D208206061686A4009400120600E4ACF
:20021C000021D1620D4A02211160012108432060032108436862206038BD0948804738BDDB
:20023C0000400440180000210000930880020021CF680000680000210011044080E200E050
:20025C00C33B00000749002800D00420064A72B60978C90701D0105800E0802062B640B28C
:20027C00704700006B0200215860044003B40148019001BDA56F00000000000001000300BA
:20029C000A001F005900EB003902EA04F9099712EB1FA132784A0A66FA828C9E63B617C953
:2002BC0064D6EDDEC1E3E0E5FF000000A36100007F1407134D00F1242E1F133FB00A3F000A
:2002DC0007FF0000304000400140034007400F404F40CF40CF41CF43CF47CF4FCF3FCF2F32
:2002FC00CF1FCF0F000000000F00080000003F00000040003F000000040068000E00DC00EB
:20031C00060043001A00050000000000020000003F00000000000400C00000000400C00090
:20033C000000070050C00091007070C00091007082312100319110B10070018101B100A1BC
:20035C008231329110B101911110418141224F40F106007051C0019130181039833108D0BC
:20037C001831416F3100319110B1831414165B680070251050C00091F4C3C0C02014036F0D
:20039C003110410422C082312100319110B163393110410482C082312100319110B163392B
:2003BC003110A2C082312100319110B1501015310514059200703F6452C0311031066131A2
:2003DC00C102426412C13110213971065131E102426400708A65996588C02082503980391F
:2003FC00001E9F4041C001301814181A89C0308260398039001EA94041C001301914191A6E
:20041C003C64369110B1349110B154B0007154A064B0F0800022AF404012B09032B05382CB
:20043C005339533985643F6411C122C1426470C1C26811C1C2C0426470C1C76850C000914B
:20045C00277298921516141642105310F0C12182313131398139313151B070B272652772E4
:20047C00999270B262107310F0C331822131213981391B107265E2C08231608280318039AF
:20049C00020061B00071329110B151A061B0277230C2F36800008012B09032B0007050C01C
:2004BC0000912772999262107310F0C3318221312139813951B070B27E652772989270B21F
:2004DC0042105310F0C1218231313139813931311A107E6551A061B02772B0C018693F64D3
:2004FC0001C122C1426401C1C2C04264151A3C64359110B153828564C012B09032B0007033
:20051C003F6472C281C0426422C111C1426402C011C1426462C031C3426462C311C1426413
:20053C0002C311C14264538253398564E2C347641122404142C281C8426452C211C1426495
:20055C0072C2E1CE426402C281C8426402C201C84264B0C0546900703F6442C201C842645D
:20057C0052C211C0426472C2E1C0426402C001C1426462C001C3426422C101C1426462C333
:20059C0001C1426402C301C1426453828564007061B000711214231C7A4D339110B10070D9
:2005BC00329110B17269007061B000711318321C8649329110B10070339110B17E690070B6
:2005DC00C2C047641510C2C01216476441311514C0C0803105145410A07804040070E6C0D9
:2005FC00863101CC161467106182F0C3010417140070067305720B720E7250B00071818025
:20061C0060B050A092804122C3458080F1C11004301601110114016CD661D761D861D961BF
:20063C00DA61DB61DC61DE61E061E261E461366339639180F2C0210421318280422A1214DF
:20065C00321601112114016CEE610B62F4613963EE610B62F4613963E661E661E661E6610C
:20067C00E661E6619464E661F964E6612A65E6615665E6614667E6611012B0900E720673C6
:20069C00057210123090A761F0CF3C67D4C103C0C0C354644078509150781092607820925B
:2006BC007078309280784092907860923078909110824039F0060110103110140092426735
:2006DC00E661BCA0E2A054A0F08050221546408000222B470D6240A02D828D318D39108240
:2006FC00F1C0100409101A824A391A041082803910040E10AB10BC10C21063642972E0CFDC
:20071C003C6713B003B0C86653B050B054B064B013B0A5661082E0223846AE660071418035
:20073C0001222B47F08010224B46F022184764B03122384263B0CE661082E0223846706654
:20075C00386264B06F818F318F3DD0DFFF923C670071418001222B4764B0F080502265420C
:20077C0063B01182C1226046CE6605671182D122524670665262618172818131813D8231EE
:20079C00823DC0EFF19202933C670B62B081C091D381978290A2D3187F4EF30B1316E31CA8
:2007BC00A44AC391E3813B149062BA1C8B46231E8B4AE31C8B4E90B207228B4290A21B1A02
:2007DC009662E31CA44AC391E3813B18AB1CA04E9B1CA24ABC1CA442B2101082D0229D42D2
:2007FC00F0801022A4466364A566A462AB1094629B10946200703082F1C0100463B00071BC
:20081C00A86ABC10E0B00070B281C291D281018212185181121841828131813D121CBF4AF2
:20083C00E2B032B0B0DFF2923C67F1C72114C34E12C86291729131B0E1B0007008C006C034
:20085C0000C86091709100700182B081C091D0811018518110180614E18042828231823D29
:20087C00201CE44AE2B02122E84632B00510A0DFF5923C672122E842E2A032B03182413951
:20089C00F0C00104011EF642181610C01030081C04476010103C0610F1C76114FA4E16C85E
:2008BC00669171818131813D161C014B769131B006C008C0007061818131813D4082803992
:2008DC000118F11C174B0114B080C0221747BCB033B090EFF1920F933C67007003A063B033
:2008FC0064B0EFB056650071408000222B4764B02A65EFA00071408000222B4764B003B0EB
:20091C003862018262818231823D80EFF19202933C6703A05665E661A2806364E66150B04A
:20093C000071E661E092D08200223D47C0B20070A080F022594330B002C1623101C0A080B2
:20095C00001E5243F0225343A0F56031603953632010101A136F236E11161216546B0070C0
:20097C00A5C700000000000055A500000000000000000000B9950000577601004D1A010071
:20099C00B57001004569010029690100DD19010000000000000000004116010081310100D1
:2009BC00DD450100C5CF00001B7201000E3FA73FAB0C18B82BBC0BDA50E5900AD338D85846
:2009DC0009CD2CD24008CB24CE3207C920CB2A06C71CC92405C618C82004C518441803C466
:2009FC0014C61C024210C51801C310C416004100C312F6C008C0040083300100E15C01007C
:200A1C00CDC300003F76010021770100F90C0100095D01008F7601009B760100957601004A
:150A3C000000000061770100000000008D090100C80900000F55
:200A580000FF5D4501003C0A00005F7C0900001400704C00B0A30800000FF815B1A0B0D298
:200A780001B14901B700000300FA9803B325057F380000900D0020B421FD83015019AD0056
:200A9800008002AF0304401F01B35801B482B201BC03037005F70810B82084AEB8614E906A
:200AB80055B8D20701FA21FF030F008000230798FFE008003FA7781500BF20930300800575
:200AD800BB7004DE04788001886A03F5F401FF10580000FC0400C4FB2264BDE907180000A4
:200AF80038FF403A00A384060020FF40007F6440400003FF0507B12305330583FF05480A46
:200B18000306B87A02FF009F84020044C703FF0401026384100043FF02B00483880300A3A8
:200B3800FF88FB008460F13588FF601A418C60238202AF00DF7D43C47063C4B0FFC0000024
:200B5800C46FFA03332034730085E63F01916DFF0100293201005977FC024F09E9BF8104FB
:200B7800DD0E01006D74D701005F00304D23BF45A1D06F0000A98A2DDF0A7017FFE1604F76
:200B9800714FAF1251E1521752B70F0FFFE3FC04D3FFEFD40108020020596B6F0100B96FFC
:200BB80041CF084D55413F608B44874AC7AE00B8FFEF2A76F337B676FF4301077CB0C40D8B
:200BD800FFE081F68AF3C50D8AA04000011BF70000C800B002002A00DD028BB0180C0EFFEC
:200BF800E02600DB02020E300D0E8CE01200F5028C10E0017002000C00AD030170952B044A
:200C18007122FFE4FEBE7CBF3788840100059540F53D595E3F34C816002000316639D9042A
:200C3800FFE50DF0282898B307C2F1019531693F03FFEF020F20058075040030FEA3FF2ED9
:200C580008808000316C047F2A7329C5A7FFE3E17175161F00E41900200175027D02F5FD3E
:200C780030001E5000A00040019F8002F004E09B30FFEF0E40FD117CBD01004418002044D9
:200C9800003101BF026001B00031A04F260741404AFFEF123082AF1DF80B300031001330FB
:200CB800AA0031080034100034180034201A00342800349DFCFFE7B671BE0248FFE802F123
:200CD800FFE15818B00031600034556800347000347800348000341EFFEF129C0100200067
:200CF80031943193E97B7F26927F1485660100CA0197FF0014FFE2CCC5D0CCE1F04D1ACAB4
:200D180073B80600F3FFEF0CF00034C6FFEB1D1ED0B0FFEF010520007DA42A3000316C06DC
:200D38007000317400347CAA00348400348C00349400349CAA0034A40034AC0034B400349E
:200D5800BC04003476F27F49D03A4F054172DAB0FFF0007D000000EA1A0020DC003059E0E7
:200D7800007000F1004B00700500927F2001010000642C0174000044FFF000F301000007D4
:200D980000B958190020EC01A80252E41A0133340100052000313C0034FFF0009D0000014E
:200DB8006CDC02007200C04CEF1800200300C4AD58011F0011700100FFF000FD000004A826
:200DD800170020281947002001010000310029AC0170000031FFF0007B0100000F00F818E8
:200DF8000020016100FFF0002D2001005174010055750100003D000000A8170020FFF00080
:200E18000200000019170000000F08000000FFF00001000000FFF00001000004FFF000019D
:200E3800000004FFF0000000580A0000080200206A0D000044010020920D0000000100207F
:200E5800B30D0000A4010020D20D000078010020EF0D0000C80100200C0E0000E401002079
:200E7800180E0000F01A0020200E000000020020280E0000EC0100202F0E0000F001002029
:080E9800360E0000F8010020F5
:201000003C000000000000000000000034100000000000000000000001000000000000004F
:1C10200000000000000000000000000001000000000000000800000000000000AB
:20103C003400000000000000000000006810000000000000000000000100000000000000E7
:14105C00010000000000000000000000080000000000000077
:2010700030000000000000000000000098100000040000000000000001000000FFFFFFFF87
:10109000FF00000001000000080000000000000048
:2010A0002C0000000000000000000000C4100000040000000000000001000000FFFFFFFF2F
:0C10C000FFFFFFFF080000000000000020
:2010CC0038140000E410000095A1011091A70110A1C2011009B2011041B8011000000000EA
:0810EC00000000002D000000CF
:2010F400280000000000000000000000141100000000000000000000FFFFFFFF0000000093
:081114000800000000000000CB
:20111C00341400003011000065C2011069C101101BC2011091BA011000000000000000006D
:04113C002F00000080
:20114000341400005411000071C20110A5B6011099BF011045B601100000000000000000BD
:04116000300000005B
:201164002400000000000000000000008011000000000000000000000000000008000000AE
:041184000000000067
:20118800240000000000000000000000A41100000000000000000000000000000800000066
:0411A8000000000043
:2011AC00240000000000000000000000C8110000000000000100000000000000080000001D
:0411CC00000000001F
:2011D000000000006C1A002004000000000000000000000020000000701000003000000085
:2011F0001C110000741A00200400000000000000000000000C000000301300001800000099
:20121000401100007C1A00200400000000000000000000002400000048130000180000001C
:2012300000000000841A002004000000000000000000000010000000A01000002C000000F0
:20125000CC1000008C1A00200400000000000000000000002000000064110000240000001F
:20127000FFFFFFFF941A0020040000000000000000000000280000008811000024000000AB
:20129000FFFFFFFF9C1A0020040000000000000000000000580000003C1000003400000090
:2012B000FFFFFFFFA41A0020040000000000000000000000100000006013000018000000A5
:2012D000FFFFFFFFAC1A00200400000000000000000000001C000000AC110000240000001B
:2012F000FFFFFFFFB41A002004000000000000000000000038000000F4100000280000008C
:20131000FFFFFFFFBC1A002004000000000000000000000054000000001000003C00000027
:1813300018000000000000000000000040130000080000000000000032
:1813480018000000000000000000000058130000080000000000000002
:18136000180000000000000000000000701300000800000000000000D2
:0813780002000000108B0100CF
:041384000100000064
:0413880000000E0053
:04138C0000000F004E
:041390003200000027
:041394000100000054
:04139800E419002034
:04139C00000200004B
:0413A000BF76010013
:0413A400FDC901106E
:0413A8000000000041
:0413AC00000000003D
:0413B0000800000031
:0413B4000000220013
:0413B80030180020C9
:0413BC00010000002C
:0413C000FC190020F4
:0413C400080000001D
:0413C8000000000021
:0413CC00000000001D
:0413D0000000000019
:0413D400080000000D
:0413D8000000000011
:0413DC00000000000D
:0413E0000100000008
:0413E40028190020A4
:0413E80006000000FB
:0413EC0001000000FC
:0413F000C8160020FB
:0413F40000000000F5
:0413F80000000000F1
:0413FC0000020000EB
:0414000000000000E8
:021406002900BB
:021408000100E1
:02140A002500BB
:02140C002F00AF
:02140E003000AC
:021410002D00AD
:021412000100D7
:0114140001D6
:0814180003000000C48A01007A
:081420000000000000000000C4
:0414280000000100BF
:04142C0000000300B9
:0414300083C4011060
:041434003C14000064
:041438003C14000060
:04143C0000000000AC
:041440008000000028
:041444008000000024
:0414480000000000A0
:04144C00FC19002067
:0414500063720100C2
:041454002000000074
:04145800788A01008D
:04145C00DC89010026
:0414600009C30110AB
:04146400D73001007C
:041468001735010033
:04146C0095C801100E
:0414700097C8011008
:041474000000000074
:04147800778A01006E
:04147C00E088010003
:04148000F8880100E7
:04148400C888010013
:0214880008005A
:02148A00090057
:02148C0001005D
:02148E0000005C
:01149000015A
:041494000000000054
:041498000000000050
:04149C00000000004C
:0414A0000000000048
:0414A4006577010067
:0414A800D94F010017
:0414AC00F9620100E0
:0414B0008D53010057
:0414B4008B54010054
:0414B800DD580100FA
:0414BC00851801008E
:0414C0007B74010038
:0414C4005D2C01009A
:0414C8000DC801103A
:0414CC001DC8011026
:0414D0000800000010
:0414D40024000000F0
:0414D80018000000F8
:0414DC0028000000E4
:0414E00020000000E8
:0414E4003C000000C8
:0414E8000C000000F4
:0414EC0034000000C8
:2014F000C7482DE9F04F0C4620274FF0000C01211F40ADF14C0D6546DFF81893DFF818837D
:20151000DFF818A3DFF818B30170002F0F93C0490E9205EA020081F800C008BF00287CD136
:201530000E984FF0E047194662460F401040002F08BF002845D10F9E0E9B4FF48601B9F8E4
:20155000B200DFF800C3CDF8289002EA0607002F01EA030108BF00291AD1B94902EA0607C5
:20157000002F01EA030108BF002970D0374643460E9EDC8003F128011881002F81E8C000F1
:2015900004BF311CB1F1806F61D102285FD111E0374643460E9EDC8003F128011881002F2A
:2015B00081E8C00004BF311CB1F5803F4FD1B0F5505F4CD1186A674643693868214698472B
:2015D00043E04646C249B6F9067091F90000BC42A0F10100087017D1328906F1280003C8FD
:2015F000002904BFB0F5803FB2F5505F08D0002904BFB0F1806F022A02D010F071FF03E090
:2016100012F070FA15F028FC524692F90000401E10706FF00101F18015E0B64E3778434621
:201630006FF00100991D08806FB1B3480078832802D08120594608704646316919B160469E
:2016500088472146E7E7CDF82890B9F8B2000F9E0E9A2F46022137401140002F08BF0029C2
:2016700000F07A83A5490B91A64A119243F20141814200F04B83C91C814200F04783944919
:201690000A4691F900104746491E1170B7F906108C4205D043F60401814240F0468342E353
:2016B0004046283090E800032F464FF4820607EA090706EA0800002F08BF002811D15648EA
:2016D000283003C82F464FF400320F400240002F08BF002A02D110F003FF26E312F002FA60
:2016F00023E328460B9F109097F8380081245D4618B92F780FB115F0DDFD2C70804C00206E
:2017100067786081119EE770054635702069DFF8F891017A457A05F0070201EB022135F0AE
:201730007F05A1F104011FFA81F840F0D782B8F5006F80F2D3820A3041460EF095FFE169E3
:2017500004F114000522083115F0CEFBA8F1030305200D961FFA83F8E27DA57D217E0B9B81
:201770006081C2F3011B93F83860617105EB02255EB161480078862807D1BBF1020F04D153
:2017900005F00700022840F0A982281300F0020ABAF1020F58DAA37805F00700022841D140
:2017B0004E467068002B0C903CD1E16909A801220D3115F099FB062060810C9880478046AC
:2017D0000C96C74F4C48B6683A680078862819D122B915F06FFD48463A6886689DF92400B9
:2017F00015F0B0FF9DF924705077002090774046D777B04705F0100010F090F904E0C046CA
:20181000E81A00204046B04715F082F96AE2C046D01A0020280D002028160020D11A00207F
:2018300004320020344800780026862808BF0126CDF830905EB1002012F0C6F9E77805E0D3
:2018500000000C8C94190020CDF83090A37887B17BB9012F00F03D82022F03D115F0070F08
:2018700040F03782032F04D105F00700032840F03082280908D315F4405F00F02A82C74800
:201890000778002F00F02582BAF1020F02DAA80A80F01F82C3480078C0F381098611B9F197
:2018B000010F00F01682012E00F01382BBF1030F00F00F82BA48BBF1020F0BD010F80910D2
:2018D000805D4018C7B22EB3E80923D3BF1E0EE0D21A002000EB09018019097900794018CA
:2018F000C7B2E80912D259EA060313D0BF1CFFB210E0C0462414002008320020EC13002008
:2019100090310020063200208C14002059EA060308BF0227C5F3002BA7EB0B008045C0F28B
:20193000D881A8EB07002909584480B2208124BF2521109110994018743080B215F0C6FB9C
:2019500094F80280E060002800F0C381002174220FF00BFA0020B8F1000F207103D10D992F
:2019700005F0200008700D9803784FF00008002B52D0BBF1000F4FD1D748008805F0070197
:2019900003291ED18108424609D3554991F82E30A3B90B681BB15B7E33F07F030ED16AB98F
:2019B0008008C24607D3D7498B68887813B1984794F8048010B9BAF1000F02D004202071DD
:2019D00080460B9894F805A090F8383033BBCE49002352460220B8F1000FCB7201F10A0A90
:2019F0008AF80000AAF1020007D000F1020A9AF8001041F010018AF800100A990271052231
:201A1000A1F87820C1F8840014F0F0FB504603210EF02AFE94F8048094F805A0E16801F1FD
:201A300074004860886523890B812089A1F85C0028090ED3CBF1030082B2A1F85C20886DA8
:201A5000D44915F051FAE1688A6DB1F85C00801888655448CF4B0078C0F3011218788D81AD
:201A7000BBF1000F00F0780040EA020048EA00050D744FF0FF038B7318BF4FF0000A81F877
:201A9000306081F83A9081F849A06089002FA0EB0B0085B2658100F01481E069E7802918C0
:201AB0003A460831684615F01FFA3E48EE19B5B26581E16800780A7C6E46C0F38103C0F3D2
:201AD000011BC0F38108002B02F0400A4AD0C0F301100023022805D1D0090FD202E0C04694
:201AF000640E00209DF801209DF8000000EB0220A1F844000DF10206A1F84200AD4AB1F88E
:201B10004400B2F84A20824203D04FF6FF72824222D1B8F1030F12D072783078A54B00EB4F
:201B3000022082B24A86B3F84810B61C0120914211D04FF6FF71914218BF00200BE0E06813
:201B50003146323015F0DAFDE0689A4932303F3114F0ECFF08360346002B00F0B580204697
:201B7000E168C07D831125D0BBF1020F03D0087CC00903D309E05AEA080206D172783078F3
:201B9000B61C00EB0220A1F84200032B0CD07078327802EB00220A850CE0C04644120020D9
:201BB000D08A0100A7310020E0683146283015F0A5FDE16888890009C0F08380886D3A4679
:201BD000694615F091F9E068816D79188165E669B0F85C1001227F18A919A0F85C7008318E
:201BF0000DF1250015F080F96F1CBDB26581E1689DF82500896D0870E2689DF825609DF8EA
:201C10002530906D401C9065B2F85C00401CA2F85C0006F0070082F82400C3F3C10182F82C
:201C30002510208992F824708046002F4CD05F4F7F183E78361D8642E68045DCE069291860
:201C50003246083105A815F04FF93A789DF817C0111D481980B29DF81450608105EB0C60B4
:201C7000E3689DF8165000EB05409DF81550042900EB052098610BDDE06806A9521E1C3013
:201C900015F032F93878E3686844C07D83F82600986D05A9324615F027F9E068816D711870
:201CB0008165B0F85C10A8EB06077118A0F85C10791E89B22181B0F85C2001818918A0F89A
:201CD0005C1000F07FF80DE015F054FC10F008FC08E015F05FFA05E02015002015F05AFA02
:201CF000CDF83090DDF83080D8F804008047E1690A68002313710968E161D8F80810884762
:201D100013E0C0463C1A00209818002040462A4F00784146401C087097F900003946401E35
:201D3000087010F0DDFB14F055FC0A980B9D214F00216FF00106A0F8B21095F83800FE8010
:201D500010B11198007808B915F086F81B481B4990F90000401E0870174890F9000010B976
:201D7000134800210170154890F90000A0B10F9F0E9A4FF0E040022138401140002808BF9F
:201D900000290DD00D4890F90000002808DC15F091FA05E0A63100200020014605F0A2FEDB
:201DB0000749002013B00870BDE8F08FAC8A0100CE1A002028160020D21A0020D11A002090
:201DD000E81A00202DE9F04FB84CE0686189E2692589806DADF13C0D0E46891808312A46DB
:201DF00015F082F8A81986B2E068816D6D188565E0690122311808310CA815F075F8761C10
:201E1000B5B20422E06965812918083104A815F06BF89DF813109DF8100000EB0160E36874
:201E30009DF812102D1D00EB01409DF81110658100EB0120049015F067F9D863049814F0E9
:201E5000F7FDA3F84000EA2014F0BFFE0220B849E26808702079117C084310749DF9300038
:201E700015F070FC82F8460011899DF93000DFF8C4B282F8480002F174009065B2F85C0050
:201E9000401A51684FF0000909185160908982F84790830A18D2030957D310F0070F07D001
:201EB00000F00700032812BF081C5068401C48E05068C17801F00703491001F0380101EB64
:201ED00043014018001D3CE0171C02D115F0F2F9E268B889800A2ED379684878C6112AD19E
:201EF0003E89796648464D780B7805F07F056D0005EBE3157E2D0DD07F2D09D003F07F0306
:201F10001818801C5B1880B2991C8642EBDC08E0494600E00121801C87F8601080B28642FE
:201F300001DA484605E07968411879603989091A3981A7F86800506E10B1B2F86800B0B198
:201F5000506850619089000916D292F86000002800F0FE80104611F007FAE268D06C002878
:201F700000F0F680B2F85000002840F0F18015F0EFFA4846E060E0E14846154605904E4699
:201F9000069005A907AB06AA95F824700796284604F0F7FC002840F0D080059A6E6968688A
:201FB0002B89311A581A1FFA80F80AB915F082F9B5F85C0000900196CDF808800698001D94
:201FD00003900598A969AB6D3A4615300AF05AFC002840F0B280B54895F860302E89C15D09
:201FF000701A288113B1284611F0BEF9AE8906F00706032E02D168680078E87395F80F80B7
:20201000732009A913F0B4FE83200DF1320108F095F8484649460D900AE0C278012A03D180
:20203000002F08BFDC2027D0001D491C0990C9B29DF8320088427FDD09988278032E07D081
:202050000378B3420DD09BF800300BB1022E08D0032EE9D10378032BE6D103465B784345AD
:20207000E2D1BB10B3EBA20F05DA02F0030207F003039A42D1DD48468246059895F80FC0D7
:2020900090F814E04946D84601E0491CC9B28E454CDD07694B00032E03EB070208D1FB5C37
:2020B000032BF2D152786245EFD10AE0903100201278B24205D098F80020002AE5D0022E11
:2020D000E3D10698077D002F08BFBAF1DC0F33D0A869B0F1FF3F27D0712008A913F048FE19
:2020F000AA69089B484605998B4207D10699064601EB8601C9680D96914213D8401C2C339E
:202110000228F0DB06980D99521CB2F1FF3F00EB8100C26002D107980121817085F8019006
:2021300048460BE0DB2009E0DB2006E0DC2004E00432002024140020DD206870E2685070E4
:202150009069577850651FB1F22014F03EFDE2687C4DDFF8F88195F83800002874D0918923
:20217000794E01F00701022938D1A778002F35D15778002F32D106F11C010888EB6D401CAE
:202190000880506E8DF831900DF131020421984730B94046006818B19DF8311080F8681008
:2021B000E1680DF12E0000906D6E486E4A460BAB2831A84766480078862808D1F08BE76874
:2021D000401CF083B88900F010000FF0A7FC15F0BFF94846E06014F09BFCB0E05D490F785A
:2021F0004FB35778002F40F0A8809DF83000378C20702379781C002B308402F1280602F13C
:202210001C020CBF4B46082353484946016014F0DBFD0146009351480192038832460D206C
:2022300005F086FA10B913F0E1FF01E014F00EFC5846E268007838B1D5F8801021B11046B0
:2022500088475846E26800780A9210B1907BFF286FD0938913F007003DD0401E53D0801E1F
:2022700067D1C3F30130022803D15068007807282FD0108900285CD0104641684A1C4260DF
:202290000F788446C7739CF824608EB9002F50D00A2F4EDA0189324EF01910F8010C8842A2
:2022B0000BD0082F45D1082907D042E0B08A0100C07B00283DD00A283BDA60460189491E33
:2022D0000181C17B0B3101700A99C87B401CC8731BE0322018E0234E96F871000F280CD03E
:2022F00014F030FF48B9181300F00200022804DA4046001D01680A98884796F8A7000A9A1F
:202310001074152000E0162010700A99454605F1280013F019F8144E7068804795F8301030
:20233000491C85F83010B1688847202015F012F84FE70AA812F00AFA4BE710F0D1F80FB08C
:20235000BDE8F08FEC130020C8180020640E002008320020063200209C18002032120020AE
:20237000D8860100A81100208C1400202DE9FE4FE54980460122A1F130000260DF48076821
:20239000002FFCD0DE4ADF4EC027E048E04B17603268920808D2324652F8042C03F14104F3
:2023B000120C42F0F00222704FF0000A8346C1F800A0DFF864C3DBF80810D64D0191880E9A
:2023D00043D2480E41D3802018744FF6D802A3F8512018702868C0F30464162CA8BF203CDF
:2023F0001F460F3F387800F01F001628A8BF2038844223D0624602F1980EDA4ACEF800A0DA
:20241000261A022E05DC16F1020FB8BF6FF0010600E002263018166800F01F06844246F483
:20243000F856A7F866604FF001061660E8D11068374617601068CEF800601068284600680C
:20245000C0F30420162808DB06E0A5F1D0000068C0F30460162800DB203800EB2170401C60
:20247000162805DA10F10A0FB8BF6FF0090000E01520DE4F00F01F0040F4F850A3F8590075
:20249000386880083ABFEA48C0F800A041F04061019E6246A5F13804C80E8F0E80F00100B2
:2024B00000F00100106087F0010000F0010090602068C0F38367C0F38F21B00C23D23046A3
:2024D00040F3072000280BD542425046490805D17F0806BF0127391C4FF6FF71521EF5D195
:2024F000002810DD4FF6FF72490041F001018A4207D27F0047F001070F2F92BF01210F273B
:20251000111C401EF0D141EA0741182012F032FE2068D24E2768C94CA6F10409C0F3870157
:2025300007F0030041EA0021D9F8040040F2FF3253468FB22C21466800972746A7F140005C
:20255000B0470C3D2868C0F30D011C2012F012FEB84955F8080C014000F07C4001431420C5
:2025700012F008FE55F80C1C01F47C000904090C0143102012F0FEFD624955F8042C096831
:20259000C2F30350C2F30343490813D2DBF800100D0510EB257003D41028A8BF0F2000E0E8
:2025B0005046090413EB217303D4102BA8BF0F2300E0534643EA001302F47F4002F0FF01CB
:2025D000B8F1220F40EA034041EA000124BF02F0804211430C2012F0CDFD974DB8F1220FD7
:2025F00032BF01202868C0F30070B8F1220F4FEA400040F0200084F8090126BF2868C0F3B5
:20261000407001208E4EB8F1200F40F0100084F8090138BF514606D33168C80C00F44070E7
:20263000C1F384510143282012F0A4FDB8F1200F26BF3068C0F301505046B8F1220F4FEAD0
:20265000400040F0600084F80C0126BF2868C0F3C0605046B8F1220F4FEAC00040F08000B0
:2026700084F8010126BF2868C0F345505046B8F1200F4FEA800040F47C40A4F89C0138BFC8
:2026900070490AD3306801038A15920501F47C1100F00F00114341EA0031082012F06AFD00
:2026B0004FF48000A5F1D0012060674A886D40F21E236FF31F40834216D90868030E13F04E
:2026D0000F0F03F00F01C0F3034018BF491E072805D006280EBF0720801C00F00F0041EAA9
:2026F0000011A2F108000170DDF804C0CCF381477F1E13D07F1E3BD036E0C046940222434E
:2027100000600C40B03F005040100940AC3F00501562084088130050000020432846006807
:20273000810C21D24FF480412160D2F80210430AC0F3033703F0800321F08F010B4347EAD8
:202750000301C2F80210D2F80130060A66F30303C2F80130116800F0E70721F0E70147EAC3
:20277000010004E02C2009404FF00040224610603B480068C0F3C0070FB94020A0624FF4A6
:202790000070206428684027C0F3C14040F0300084F8C800CCF3815050B3401E03D0401EC4
:2027B0001FD002211EE0012013F08AF90646042031460FF08DFF042013F082F98642FAD1AB
:2027D0002248066826F07F4012F048FFD9F81400036807214FF06022300E98474FF480607A
:2027F0002060032104200FF073FF08E000000940042001210FF06CFF154812F02FFF203DC5
:202810002868144947F6180600F03F0084F8CB0F144B0E80D9F800201868D1680220884753
:2028300011480D4D076001212960BDE8FE8FC04694042A43FCFCFC008C13005040A00C4077
:202850009813005000803F400A600840A83F0050BD37860070B00C4094046042A4010010B0
:20287000B03F00502C20094000600C402DE9F04F0320ADF15C0D12F021FFD14D00240220C3
:2028900005F11C0141F80C4F401E8C60FAD105F14000062701467F1E21F80C4BFBD14FF0AA
:2028B0000808C849A0F80080C74E8160C749361D26F003000B1A2B62A861E861AA6905F150
:2028D0001C09B44607460E46914200F2E581991000EB810121F8044CE8233B804FF6FC7700
:2028F00007EA0C0200F1E803B61A2B6107EA0601EC39A0F8E81020460DF0F0FD6861C949B9
:20291000D9F80000DFF8C89228610A6809F10C00026049684160C4498246424613F0AEFCE6
:2029300028B9C24801685246116040685060C048C14FC24EC24BC764BE490665C14A43654D
:20295000C14F816400F1480B8265C04EC765C04B0666816C436609B1204688470FF04EF9CB
:202970002146D24E15910C220E9106F120000EF0FCF9CF4F0222ADF8208041F270737762CD
:20299000708CADF82220696AB3621027099740F01900708408A8884700280CBF0A9F271CEA
:2029B0000120ADF82C80696AADF82E000BA888479DF830004D4628700D9969605FB1D0210D
:2029D00039707C70B870FC703C713946BC600220FC6011F095FFB749182001220DF0EEF924
:2029F000E220514614F056FC182012F075FB68706868B246CAF808000BF028FC0AF170003A
:202A1000AD4EA860DAF80870C6F824B0AB4DB76005F10C0105F118000DF008F8A8600F2073
:202A300014F036FB00B1A046042014F031FB08B948F01008A249A86814F060FDA149C82225
:202A500005F1240011F02EFA9F48B8F1100F68604BD113F077F8706A002846D0C268002AB2
:202A700043D006278DF810700220ADF8120004ADADF8144095E80300904725468DF81070B7
:202A90000320ADF81200706AC268ADF8145004AB93E8030090476D1CB5F5FA7FF3DB756AE2
:202AB0008DF81070042004ABADF81200EA68ADF8144093E8030090478DF81070052004ABFE
:202AD000756AADF81200EA68ADF8144093E80300904704AD8DF81070706AADF81270C268CF
:202AF000ADF8144095E803009047DFF8E09109F1180009F10C010CF099FFC9F8000020465A
:202B100014F01AFD25464FF006084FF0040B149009F1020707F8024F0220787014F00CFE75
:202B30000146149AD9F80000C9B212F06DF96D1C042DEFDB664909F124004FF4FA7211F0DB
:202B5000B1F9706A002850D00769DFF888916FB10096494612A80A688988026012AD818095
:202B700095E8030001232246B847706A00283CD0C26852B1494612A80B688988036012AF0E
:202B9000818097E803009047706A70B3076967B38DF80880ADF80A8010A8ADF80C4002ADB0
:202BB000009095E8030022460223ADF84020B847756ABDF840006F69B080B7B10AE0C04630
:202BD0008C140020C564010009320020004B0020141A0020BDF8400002AD401CADF8400002
:202BF00095E80300022210ABB8472DA014F0FAFA706A00283ED00769002F3BD08DF81880CB
:202C1000ADF81AB00EA8ADF81C4006AD009095E8030022465B46B847E0B90E981930159086
:202C300028E0C046C8FF0100F08A0100F012005008020020919E00009D450100912A0100E9
:202C5000E5140100010C010045020100ED0D0100A93601008DF818802046776AADF81AB066
:202C700006ADADF81C407C690F9095E803005A460FABA04715980E900DF000FFE0200E21D5
:202C900013F0D6FF13F072FE0AF10200012113F097FE01F093F9FCE722F8024B14E6C0465B
:202CB00054492053656E736F7200C0469012002020BF0200F9880000A41000201417002084
:202CD00089520100796D0100116F01005C170020F5050100248B01002DE9F04FADF18C0DD6
:202CF0001C911E93CC491D920A6806460DF156000260496841603046694612F09DF90028F7
:202D10001F9004BF0020229000F0F78102200027B61CDFF84CB32090D34D2297304602A95C
:202D300010F09FFB5FEA000900F0E48122990EA816220EF01AF89DF809707F1E00F08280EC
:202D50007F1E40F0CF81B9F10A0F40F3D681B61C316804A80160361D318805AF42F20B0082
:202D700039800DF1160110F025FEBDF81600BDF81410884200F3C181B61C16F8010B16F8B5
:202D9000017B16F8014B8DF8380016F8011B8DF839700EAA8DF83A40304605F017FBBF49FC
:202DB00009780028064400F0A8811F9C012904F1020400F091814FF400500DF14E0110F035
:202DD000F9FD0DF14E000DF15601082213F056FA40B11C990DF14E00082213F04FFA00283F
:202DF00040F07A8142F2010004A907F0F9F842F20B0005A907F0F4F842F205000EA907F017
:202E1000EFF80DF1390142F2060007F0E9F80DF13A0142F2070007F0E3F80DF13B0142F2BD
:202E3000090007F0DDF89DF83B0028B1022840F0538142F2030001E042F20D000FA907F0CE
:202E5000CFF849E1B9F1040F40F35781B61C16F8010B16F8017B16F8014B8DF8380016F80E
:202E7000011B8DF839700EAA8DF83A40304605F0ADFA0028064400F040811C9806A909F0B0
:202E9000A1F99DF83600002840F00A819DF83B0000287AD195F82D70002F00F0FD8095F844
:202EB0002F00874207D095F888000A2801D10AF05DF9686B1EE06F6B4FF400500DF15E012F
:202ED00010F078FD13F0D6FA4FF0FF08229C2190A24695F82D00A04240DC686BB8F1FF0FBB
:202EF00008D008EB88040019007912F0F7FA686B071923D195F82D300746002B08BF229C18
:202F100019D05846229C40681946D8467F1F7F1DFA782AB1491E04F10104F8D17F1D0AE000
:202F3000804795F82F10491C85F82F10D8F80810884795F82D30A34200F094801C980BF094
:202F500085FF38710120F870FC788DF8364038798DF83700229B8DF82330A1E0387910F008
:202F7000EDFE014608220DF15E0013F087F940B138880104219814F0CFFB82453CBF82463F
:202F9000A046641C7F1DA4B2A3E795F82C70002F00F0828095F82E00874207D095F8880085
:202FB0000A2801D10AF0E2F8286B1EE02F6B4FF400500DF1660110F0FDFC13F05BFA4FF076
:202FD000FF08229C2190A24695F82C00A0424DDC286BB8F1FF0F08D04FEA48140019C07FB0
:202FF00012F07CFA286B071925D195F82C300746002B08BF229C1CD0DBF80400229C1946DA
:20301000D846203F2037BA7F42B1491E04F10104F8D120370DE0C046E08A0100804795F86D
:203030002E10491C85F82E10D8F80810884795F82C30A34216D02299384620220DF095FEAC
:203050001C980BF003FFF8770123FF2039462022BB770446787206A8FC720CF01BFB1FE0A9
:203070008C140020612055E0AC2E0020F87F10F065FE014608220DF1660013F0FFF838B13E
:203090007968219814F048FB82453CBF8246A046641C2037A4B297E764203BE0ED13002065
:2030B0009DF836000EA9162240F004008DF8360008A80CF0EFFA1F9C9DF83B00A41C40B186
:2030D0009DF84D700FA839460FF01CFE3F1A8DF8357006A80FF0A6F820984844801C80B25F
:2030F000209003E01F9C4E44B61CA41C209884423FF714AE2098022803DC229A672011467D
:2031100004E01F9A911C121A2298921C1D9B19801E990A8023B0BDE8F08F70472DE9F04F2C
:203130000F46C64E42680168ADF14C0D726080687162C54CB06077B1C1487A68C761BD69FD
:203150004262BA68026225B1BE4D14302860BA690260F86820604FF008084FF0010AADF8E5
:20317000188006A8ADF81AA08847B84D9DF81C10089B69706B6108B113F050FB386880474F
:20319000706880474FF400578346ADF800801E200197716AADF802006846884711F070FDB5
:2031B0002068406880472068C16810A888472068836810AA002001469847606008B913F0D9
:2031D0002DFB13F04DFDA248A34FA24A2861A34C1760A4495460A24BD160A34FA448936023
:2031F000A24C1761A34F546100F118013964BA64A14B3B651439796403F140029F4B7B613B
:2032100003F16A01B9619E4BFA649F497B629D4B19609E4959603B669D4999600024AC6068
:2032300080F838409B49D9609B4999619B4999629B499C4A99639D4B13619D4B53619D4B0E
:20325000D3619D4B13629D4B1C635C634FF0FF0983F8389083F83B4083F83C4083F83D4038
:20327000AF49C0F89C10904B53601123BB81944AC263944B0364944A4264944B8364944A73
:20329000C264944B0365944A4265944B8365944AC265944B0366944A4266944B8366944AEC
:2032B000C266944B0367944A4267944B8367944AC267944BC0F88030934AC0F88420934BD8
:2032D000C0F88830924AC0F88C20924BC0F89030914AC0F89420914BC0F89830914A1460E7
:2032F000914B83F800A05C80022012F045FE0222E862494614F02AFAE81C0222494614F0A4
:2033100025FA022012F038FE8849086008680222214614F01BFA11A80FA911F0CDFCE86A4A
:203330009DF84410421C01709DF8440010703C709DF84400A87013F05DF8A861716AADF8EE
:2033500008801420ADF80A0002A888471527ADF810800398ADF81270716AE86104A88847A7
:20337000744F05983C70801E2862734B1C70704D6C70AC7040F60D00EC6013F0A7FE40F2A1
:20339000FF7907468DF8284009A94246ADF82A909DF829002F6100F0F0008DF82900286965
:2033B000099713F0A1FD2C62EF616448A0F8009011F0ACF9624D2878012803D0204601466C
:2033D00004F090FB5F4804705F4F3C702878012803D02046014604F085FBB16858468847A6
:2033F00002F046FC13F02CFD5848007811F078FB5046214604F076FB11F048F9544804701D
:203410002878012803D02046014604F06BFB0FF099F81820ADF830804E4FADF832004E4DCD
:203430000D97716A0E950CA8884708B113F042FF01F074FD13B0BDE8F08FC0468C140020CB
:2034500028160020A4170020EC31002068180020BB3C0100B830002045870000A1270100B1
:203470009B670100D1C0000049DF000045100100EC1300201415002040300020B2830100FC
:203490001DE30000243100203DAF0000A5A20000E9370100F94E010001280100B1EB000045
:2034B000F5760100640E00209D6D000041CC0000C15E0100550F0100794A0100F017002077
:2034D000DDF700006575000015130100815001006580000055EA0000614C0000E92C00004D
:2034F00089FF0000997E00005DCB000051700100F19F0000C5390100B960010005D40000B1
:2035100005B5000011AE0000D7670100F5E80000B935010095600100A940010021290100EC
:2035300089740100E83100206C0A00202C2D0020903100200432002006320020F00D002089
:20355000E81A002008320020003200204F12002005320020DBF70000E01900202DE9FF476E
:20357000D64C0F460546F80B80F08B81B80880F07881F80A80F05181DFF84483DFF844A331
:20359000B80F80F0D080207A002854D1380954D3002525700126A671284612F0BBFFD1480A
:2035B00013F070FFD0492A4604F1580014F0A9F804F1400090E8000313F060FD2379B0EBC7
:2035D00008004FEA103071EB09010905012B40EA0100E0640DD194F85010B0EBC12F08D816
:2035F000E07830B904F1D4004FF0005113F0C4FC17E040F609002671BC49208504F12803C7
:2036100094F83500E57000F0F00040F0010084F8350094F834000B6000F0F00084F8340007
:20363000E5622846294604F1400282E80300E06427F008074DE1380972D2B80B5ED2780B1F
:20365000C0F04781AE69CEB14046B04216D0A86843681BB105F1200199424DD1407B10F09C
:203670000F0F0BD1688C40F60901814206D128466FF4807100224FF00073B04704F1580098
:203690005146002214F03DF8A96800264FF0010840F602026672088884F80080824207D070
:2036B0000A8B4FF61F60104040F43470088306E00A8A4FF61F60104040F4347008826E741C
:2036D00013F0DCFCD4F83C21E36804F59E719A4208BFB046A56C45B1854226BF281A401E97
:2036F000401B01EB8801000B8860A664192013F039FE27F48057ECE01846A9E704F11800C1
:2037100014F014F8061C08D0706830B17568F068B6F9241000222023A84727F40057D8E040
:203730000020207284E7A968088840F60209814507D00A8B4FF61F60104040F434700883D1
:2037500006E00A8A4FF61F60104040F43470088204F1400090E80C00002B08BF002A1AD0AA
:20377000042012F0ADF9B0B1266C13F087FC864226BF801B401E801B000BE860E968688A1D
:20379000401840F6C411E860814203D340F2EE22824200D9E960AE699EB14046B04210D0EF
:2037B00094F8350010F00F0F0BD1698C09F10700884206D128466FF4807100224FF0007311
:2037D000B04704F158005146002213F09AFFB4F8AC004FF6FF71814209D10220ADF80000CF
:2037F000684612F0EDFABDF80800A4F8AC000120207013F0ADF84FF00008192084F8058043
:2038100013F0B0FD6E692EB1414628464FF080630A46B04727F000575BE014F079F805466B
:2038300004F1140013F082FF061C15D0E06810B1703012F02FFFF068E060284614F064F8A5
:2038500013F01CFCA0642A4813F01CFE4FF4006104F1D40013F090FB002027F480672072FB
:2038700037E004F12005284613F060FF07F0B0FD284613F05BFF27F0020708B147F00207AF
:2038900027E014F045F8014604F11C0013F04EFF0646B569A80817D2B6B125EA0500B06199
:2038B000084614F031F8706888B185B12A46F068B6F9241075680023A84708E0700A00201A
:2038D0006380000091BA0000084614F01DF827F4804727B104F1D400394613F04DFB009066
:2038F000BDE8FF8785E700006D6101000010044039A90000B0B50446BC480768ADF1480D07
:20391000002F00F0AC812078401E112800F2A781DFE810F06E0156013C0127011F010801E7
:20393000F100E300C300B2008D005D0053004200A5012A001C001200F86B002800F08F8126
:20395000684621460CF0A6FBF96B86E1386C002800F085816846002101220DF006FA607851
:203970008DF80000396C78E1F86A002800F07781684600210E220DF0F8F9A11C684613F0E7
:203990000BFAA57BA1890022ADF80A1005B101228DF80C20F96A61E1B86B002800F05F819D
:2039B0006846002102220DF0E0F9A5788DF8015060788DF80000B96B4FE1786B002800F08F
:2039D0004E81684621460CF065FB796B45E1386B08B36846002114220DF0C7F9A5788DF8CB
:2039F0000150A3680193A289ADF80820A17B8DF80A1060788DF80000E57B8DF80B50237CD8
:203A10008DF80C3094F911208DF80D2061690491396B684688476068002800F0208101461D
:203A3000F22008700020487010F06AFF17E1B86A002800F014816846002124220DF095F944
:203A50006078A11C8DF800000DF1020013F0A4F904F10C0103A813F09FF9257EE08A04F152
:203A700019018DF818500B22ADF816000DF119000BF010FEB96AF0E0786A002800F0EF80CB
:203A90006846002102220DF070F9A5788DF8015060788DF80000796ADFE0386A002800F011
:203AB000DE806846002112220DF05FF9658862796078ADF8025023798DF80520E11D8DF8E0
:203AD0000000A5798DF804300B220DF107008DF806500BF0DFFD396ABFE0F869002800F060
:203AF000BE806846002101220DF03FF960788DF80000F969B1E0B86910B120460FF05EFC60
:203B1000A07D002800F0AB80A07820B9A069002800F0A58003E0A069002800F0A08012F0D8
:203B300049FC9CE07869002800F099806846002113220DF01AF96D46A01C01684068296085
:203B50000B22686004F10A0102A80BF0A3FD796983E03869002800F0828020460BF076F84C
:203B70007DE0F86800287AD0684600210E220DF0FCF86078A11C8DF800000DF1020013F0F9
:203B90000BF9A089ADF80C00F96866E0B868002865D06846002114220DF0E7F8A01C01680D
:203BB0006D46296040686860A07A0B2204F10B018DF808000DF109000BF06CFDB9684CE0BC
:203BD000786800284BD06846002110220DF0CDF860786588211D8DF800000B22ADF8025043
:203BF00001A80BF057FD796837E0C0461C1A00203868A0B36846002119220DF0B6F8A01C05
:203C100001686D46296040686860A07A410824BF01218DF80810810824BF01218DF809104E
:203C3000C10824BF01218DF80A10010924BF01218DF80B10C10924BF01218DF80C1030F0C8
:203C50007F001CBF01208DF80D000B220DF10E0004F10B010BF01EFD39686846884712B017
:203C7000B0BD70472DE9F04FDFF8B4C292F808B009AF88460646ADF1240D049338F07F0548
:203C9000039206BF604600884FF6FF700590F08A800934BF002008203076F08AC00834BF2A
:203CB000102080207076F08A400903D260460E30007800E00020B076F08A41082CBF202432
:203CD0000024000928BF44F010047568002108F07F08307D06916D1E02280EDB0C2808DC01
:203CF0000C2803D1022044F40854069044F0030404E00D280CBF02200120044396F88800A1
:203D100008B144F00804210900D328B1DFF89C9299F89C3013B908B1DF203BE121096DD358
:203D300096F88950DFF888A206F1240133891AF8052007910AEB0001097908908918491D4D
:203D5000C9B2C918B1F5006F80F2268100284CD0049A039906F1800009F0F4FE0799002821
:203D700008603FD0806AB0F1FF3F39D070680023401E8DB196F88A10524600F80119515DD3
:203D9000491EC9B241B1721892F87F20491EC9B2002900F80129F6D1079970660968896ABE
:203DB000B162090E00F8011996F82A1000F8011996F82910089A00F8011996F8281005F0A7
:203DD000030500F8011902F0070141EAC501017071683289091AC9B270608918318105E023
:203DF000DB2700E0F3277770D7E00023F08A7370C00828BF44F0100475686D1E336DA3B93E
:203E1000B36D93B999F8B510012903D13089B0F5EE7F06DA200904D202290AD144F4005496
:203E300001E044F48054012002E044F408540220069044EA8834B8F1020FA4B20AD0B8F1B9
:203E5000030F10D1ED1F09F1A801284613F056FC6D1E08E0B9F88E00001205F8010999F891
:203E70008E0005F80109069802280CD0B8F1000F15D0BBF1000F0CD004990598814208D1EF
:203E900044F040040BE0BBF1000F08D1B8F1000F05D00599081205F8010905F8011944EA8A
:203EB0008B24BBF1020FA4B209D0BBF1030F0ED10399ED1F284613F021FC6D1E07E0039976
:203ED0000888001205F80109087805F80109BBF1000F05D00498011205F8011905F8010945
:203EF0003878F8B933480178307D0D2814D068B9306D28B999F87800411C89F878100AE09F
:203F100099F89D00411C89F89D1004E099F88600411C89F88610014605F8011904E0C04621
:203F30003212002044F48074201205F801092C7070683189401B7560C0B2401830812009A6
:203F500027D3B06D00B130621B48007810B1307D0D281ED1726A12F1150002D113F0AAF91D
:203F7000726A916A481C9062306A3289B162471B0092D21B019090B20290706A96F8882046
:203F90002B46153007F0D4FB00281CBF7070071C07D10020707005E0E5277770F32012F0CA
:203FB00014FEF8B209B0BDE8F08FC046A8110020AC8A010095310020241400202DE9F041BD
:203FD000CB4CCC4DDFF834836088ADF1600D4108C0F08C800CA808A90DF0B8FF012879D18F
:203FF000404624300068D8B10769CFB1062002268DF808000022ADF80A600FABADF80C205F
:2040100002AE009396E803000C23B84740B9BDF83C006084109F67621198A06213F01AF898
:204030009DF82D00012805D002202077BDF82210A1820AE0032009AF20773A6804F11401E5
:204050000A6078684860BDF82210BDF8200009AA00230EF0B9FC011C02D0A1A013F030FBBB
:20407000022011F0A5F9BDF830009DF82C7028870DA985F83A7005F1480013F0C9FABDF814
:20409000320005F13E0609A9A5F84600304613F0BFFABDF82200298FA887502012F0BCFDF4
:2040B000B5F84610532012F0B7FD4A20314613F0F1F895F83A10E12012F0BAFDA98F4B20C3
:2040D00012F0AAFD05F10800102112F079FC0120207005E0012011F06BF9002013F06EF8DC
:2040F000A01C012112F05EFC2046408880080DD3606A11F013FB11F04FFE00B2A081E08185
:2041100002F00AF9A01C022112F04CFC2889410805D305F10800012112F044FC2889810803
:2041300005D305F10800022112F03CFC288901094BD395F8540005F1080600283DD0401EEB
:2041500039D0401E02D0401E33D039E095F85010472012F06DFD95F85110542012F068FD13
:20417000A98F4B2012F058FD298F502012F054FD0927032395F83A008DF8597016AA8DF80A
:204190005A305D498DF8580001278DF85B7018200BF014FEB4F84E00B4F84C1088420FD199
:2041B00095F8520001280BD13046202112F008FC06E0032002E0022000E001200DF0FEFF46
:2041D0003046082112F0EEFB2889410911D395F8520005F10806032818BF042802D1A86D6D
:2041F00011F084FA10F0F4FC3046102112F0DAFB2889810907D30CF0D1FF05F108002021A2
:2042100012F0D0FB2889C10907D30CF0F3FA05F10800402112F0C6FB2889400A0DD395F8F9
:20423000550012F0CBFF41F2883011F08FFA05F108004FF4807112F0B5FB4546E8884008B1
:204250000DD368780026000904D3A878012801D110F092FB6E70A81D012112F0A3FB608893
:20427000002839D10A200825254CADF812004FF0FF37ADF81050616A059704A888470028F9
:204290002AD10720ADF84850616AADF84A0012A88847149E1596F8B91A499DF84E20087878
:2042B00090420ED19DF84C004A78824206D089684B6C33B100213246984702E03046FFF7AE
:2042D00019FB159840B1ADF818500320ADF81A00616A079606A8884718B0BDE8F081C04664
:2042F00041757468204572726F723A20307800C090120020481300204F760100A410002059
:204310008C140020141A00202DE9F04F09AFADF13C0D08900A92388809911E46ADF81800DC
:20433000101C08BF002000F08481002700F101094FF0FF3A4FF0010BB8466CE1252940F0B7
:2043500063811078521C0A922D2818BFADF8068005D15846551CADF8060010780A95302871
:204370001CBF4246434605D10A9908785A465B46491C0A912A28CDF80080554616D1306856
:2043900004930A99CDF808A0C01C4B1C20F00300001D306050F8044C0A93002C08780094EE
:2043B00018D5ADF806B06442009413E044460AE0610001EBC40140180A99A0F130040878B2
:2043D0000094491C0A91302801DB3A28F0DBCDF808A004932E282BD10A9908782A2801F11B
:2043F00001010A9111D13068CDF80880C01C20F00300001D306050F8045C002D48BF454646
:2044100008782B46491C0A9111E0454643460AE0690001EBC50140180A99A0F13005087850
:204430002B46491C0A91302801DB3A28F0DB02930AB1224604926C2804D04C2818BFADF8F4
:20445000048005D10A990878ADF804B0491C0A910BA9CDF80C800FAB07916428059300F00B
:204470008B80692800F08880BDF818C0752872D078286ED06F286AD0702850D063283DD02D
:2044900073281ED009980A990128A1F101010A9115D96B490C68B5F1FF3F03D0A84288BFE9
:2044B0006D1C00D8099D029508A80AA932466B46A047C7190A99039801F1010974E04046E7
:2044D0002AE030680A99C01C20F00300001D306050F8040CBCF1000F01F10109014608B9D3
:2044F00055A00146079112F04BFE0390B5F1FF3F5BD0A842C4BF281C039056E03068C01CFD
:2045100020F00300001D306010F8040C5D468DF82C000A990395584601F1010945E008203D
:2045300035680490E81C20F00300001D306050F8041C082210230FA80DF028FB401E0790E5
:20455000402101700A99079801F1010929E0082302E0102300E00A230A99306801F10109AE
:20457000C01C20F00300001D306050F8041CAA42BCBF2A1C049210E00A99306801F10109BD
:20459000C01C20F00300001D306050F8041CAA42BCBF2A1C04926FF009030FA80DF0F6FAB5
:2045B0000790059D281A0390009C241ABDF8065000945DB906E008A8202109AA11F072FB56
:2045D000009C7F1C641E0094F5D503980546401E039075B9BDF80600E8B10098401E0090D5
:2045F00019D408A8202109AA11F05CFB00987F1CF4E70798411C0791017809AA08A811F043
:2046100051FB03987F1CE1E708A809AA11F04AFB7F1C09F101094A460A9812F8011C401C43
:2046300000290A907FF48AAE089808B14146017038460FB0BDE8F08F286E756C6C2900C07E
:20465000488B0100BA492DE9F84F00254820C1F8F35FB84CC1F8FF0F94F8E200002800F02D
:204670006381012800F02F81B34E02283CD0032840F05A8151F8310CD4F8B8100029A0F538
:20469000C060C4F8D400B8BF49420028B8BF4042814226DA4FF08057D7F8A4014568B4F891
:2046B000BC0030214FF47F42082300903046A847D7F8A4014568B4F8C00004214FF4F802CA
:2046D000122300903046A847D7F8A401B4F8D070456820214FF440620A2330460097A84744
:2046F000012584F8D8501AE151F8318C12F0F4FE2F4600B901273946904F38680028FCD0A3
:20471000B146012609F10409D9F82CA03E6009B112F0E8FECAF30720C4F8BC0012F0DCFE4F
:20473000AA4600B9B2463B68002BFCD0D9F800B0BAF1000F3E6001D012F0D4FECBF384402E
:20475000C4F8C00012F0C8FEAA4600B9B2463B68002BFCD0D9F81C90BAF1000F3E6001D024
:2047700012F0C0FEC9F38120C4F8D000B8F5C061C4F8B81000F09C8094F8D80068B9C4F8E1
:20479000D410D4F8C000C4F8C800D4F8BC70C4F8C470D4F8D030C4F8CC30D4F8D410D4F82D
:2047B000BC30002954BF02206FF0010004F1C802176801EB41014018411000EB917107EB4B
:2047D000A1001060D4F8C810C4F8C43000291CDD1E293CDDD4F8CC0030B93429B4BF153943
:2047F0001E21C4F8C81025E02A29BABFD4F8C8000B381E20C4F8C800D4F8C4003F28B4BF02
:20481000401C3F20C4F8C4001FE0D4F8CC00032812D011F10B0FC6BFD4F8C8000B30301CED
:20483000C4F8C800D4F8C4000028C4BF401E051CC4F8C450032508E011F1150FC6BFD4F8D3
:20485000C8001530301CC4F8C800C4F8CC504FF08057D7F8A401B4F8C43030214FF47F4214
:204870004568354800930823A847D7F8A40104214FF40032112345682F480096A847B4F8BA
:20489000C860D7F8A40104214FF4F8021223456829480096A847D7F8A40120214FF4406298
:2048B0000A23B4F8CC60456823480096A84701E084F8D85040F2FF50404502D8801C4045C0
:2048D0002DD208202EE051F8311C1D4F4BF2F5204843060A3868C0F3814001280AD111F08B
:2048F0005BFA10F067F812F003FE3111C010484306EBE03694F8E50030B91248006820F021
:204910007F408019460801E084F8E5500E48310C0660012741600D4D8760287808B90B20C0
:2049300000E0052084F8E40004F08AF9BDE8F88F39400C40940F002000A00C4000800C401F
:20495000B43F0050102009403C600C409A8A01002DE9F04FAF4E82463068ADF1140D08B94C
:2049700012F0A8FCAC490120AC4F08703978012902D0002103F0B6F830680489456812F0B5
:20499000B7FEDFF89C922888000937D399F83800002833D031684A6A4F6E906AC846B0F1E3
:2049B000FF3F25D027B3431C93628862030E07F80139306890F82A0007F80109306890F8DF
:2049D000290007F80109306890F8280038703268106A00940190401B201A80B20290916A18
:2049F000506A92F888202B46153006F0A1FE00E0DB20D8F87C10002840F00081214628468B
:204A10000BF032FE642003A90FF0E0F9854999F838700878884637B98348007809F0BAFF19
:204A3000012805D0E6E009F0B5FF012840F0E280DFF8F8C1A01C241D6D1EA1B2ACF87800B3
:204A5000C1F3022040F0080005F8010929709DF80C70CCF88450002F4FF00005ACF86A501E
:204A70000CBF49F24E0047F60E206446C4F8C0006F4EC4F8800070688047B3466D4E049061
:204A9000BAF1010F6BD0BAF1040F68D0BAF1000F65D094F84000BAF1050F04F13007C0F3C1
:204AB000C0003ED0E8200DF10D010FF08FF999F8380030B39DF80D00032822D1787B3B7C67
:204AD00000F0F00007F1110140F00300787343F018003874F4200FF079F9D9F89C0080470E
:204AF000A064306A544BD0F808C06586294602208DE80300D8F80C002A463946E047374676
:204B100067E0306A87684C4BA4F86A50294602208DE80300D8F80C002A4604F16801B84716
:204B3000EDE728B9787B00F0F00040F0010004E0787B00F0F00040F003007873B146294671
:204B5000D9F820003E4B8668658602208DE80300D8F80C002A463946B0474E46CFE794F8C0
:204B70003D0000F0F00040F0030084F83D0094F8400004F130018A46113140F0180084F854
:204B90004000F4200FF022F999F83800002808BF4FF4FA5002D0D9F89C0080472949A064D6
:204BB0003746D8F80C000B783E6A43B9A4F84E5002212A468DE8060004F14C0105E065860B
:204BD00002212A468DE8060051462A461A4BB568A8471A490880DBF80810002808D41A4A01
:204BF00092F900006834401C10700498FC600DE0049888471A200BF02DFC08E0002908BF1C
:204C1000E420F8D0114A00201070E420884705B0BDE8F08F640E0020CF1A0020E81A002054
:204C3000EC130020881900204F120020280D00208C140020281600202D9D000098180020F6
:204C500085C90000CA180020D11A0020083200202DE9F04F002898461546ADF12C0D00F012
:204C7000F58011F47C1F40F0EE8011F00F0F00F0ED8007460591002006900A904FF0000A79
:204C90000990544608944FF0010BCDF810B0044650460790059805990BEA000021EA0B01A7
:204CB0004FEA4B0B401E059100F0AD80401E69D0801E56D0001F40F0C08005B12F660720E8
:204CD000152642F2D002022307F8010B01A907F8016BA2F1CF0007F8013B0EF06BFE68468C
:204CF00003A90AF049FB8B48019A018842F2D0064FF47A63701890FBF3F0009B3E46C018AC
:204D10000090824206D8801ABDF80C300090581CADF80C00009B5008514681460904180497
:204D3000030C19430004534610EB090041EB0A0102F024FA0090BDF80C309DF80C009DF859
:204D500000209DF8011006F8010B181206F8010B9DF8023006F8012B9DF803200934BF1D7D
:204D70004BE00220152607F8010B042307F8016BB8F1000F07F8013B0CBF099898F800000F
:204D9000241D57E01DB1EF6595F86B0006900520152642F2D002049B07F8010B0DF10E01BE
:204DB00007F8016BA2F1CC0007F8013B0EF002FE02A80FF069FD5848029AB0F8B61042F2F3
:204DD000D00670189DF80E604FF47A6390FBF3F150189DF80E30069AE41D000200EB6600A4
:204DF000B0FBF3F03E4602903F1D06F8012B9DF808109DF809309DF80A2006F8011B06F827
:204E1000013B327018E00320152607F8010BB8F1000F07F8016B034607F8013B04BF0A9837
:204E300007F8010B05D098F8000007F8010B98F80100641D07F8010BA4B2059800287FF43C
:204E500029AF264661E011F00F0F01D000205DE080468A4602264FF4803908F1020509EAC3
:204E70000A002AEA090A4FEA4909B0F580301AD0B0F5803014D0B0F500300ED0B0F58020F6
:204E900009D0B0F5002004D0B0F580102AD1072404E0062402E0052400E00424002704E009
:204EB0000224012701E001242746A81C214600F047FC47B104F00F04C0F30A0141EAC421F6
:204ED00041F4004105E004F07F0400F0FF0141EA042105F8011B36180912B61C2970B6B25B
:204EF00045196D1CBAF1000FB9D1022ED8BF00260BDDB01E4FF6FE7708F8010BB819C0F38A
:204F1000022040F0A00088F8000030460BB0BDE8F08FC046A62E0020F02D00202DE9F04F2E
:204F3000AC4C04F128000068ADF1240D0FF0CEFA08B111F065FCA248DFF89CA2DFF888B223
:204F50000068A24E089011F02BF811F053FAE569A769B5F57A7F13D0C01B4FF47A720023CE
:204F7000A5FB000102F00AF980464FF47A72002311F0DEFF2A46002302F000F9C01901E05D
:204F9000A0EB0708A0618D488C49006820F00200086070688047DBF80010DBF804304546C6
:204FB0006918B1F57A7F0DD34FF47A72B1FBF2F2D2184FF47A73CBF804201F46B1FBF7F227
:204FD0005A43891ACBF80010B168884770688047DAF8041002466818B168CAF80400104644
:204FF0008847DAF8000000285FD007464FF00009706880474FF000081FFAA5F3079083B9AA
:205010005FFA95F36BB93979E8B2884204DD79682846884209D20AE03879E9B2401A387157
:2050300008E079682846884201D3414601E07968091A7960B88878B9FB8853B9FB6843B1EF
:205050003B8933B1B87A19460AF0F4F8F8687860B88808B9FB880BB13B896BB9B9F1000F08
:2050700004BF3868CAF8000003D03868C9F800003868B846074601E0B9463F68B16807989D
:205090008847B8F1000F0ED0B8F8043043B9B8F806302BB998F80A00B8F808100AF0CAF8D3
:2050B000404611F077F9002FA2D144484349006840F002000860E06828B3804723E015F833
:2050D000060C2169A5F10C07032819D0E16A9DF816000978884210D115F8080C10F096FB93
:2050F000B979012903D0022908BFA87000E02870002029460DF0ACFB05E011F081FB02E078
:2051100009B12846884708200727ADF81000716AADF8127004A88847069D0028CFD0294825
:2051300000680088C8B1706880472649096800220D880A80B1688847089A0020294620708D
:2051500090470546FF202070706880471D4909680A8815430D80B168884710F021FF07462C
:20517000B7F1FF3F1CD0706807B9194F216AB94238BF0F1C80471C230546626AADF80230B1
:205190000820ADF80000716A019268468847A16A3846491CA1620FF0D1FBB1682846884735
:2051B00008200A27ADF808004FF0FF35ADF80A70716A039502A88847C5E6C04610E000E0DA
:2051D000348B01002C2D0020541A00208C1400208EC2F52868180020E43100202DE9F04FA1
:2051F0008146002000212022ADF1540D009003A80BF0BBFDD9F82400B9F8221001236A46BC
:2052100007F088FD0024A046002876D10098002873D006467079042869D100200190F188C1
:20523000B06801AA002307F075FD00285FD1019800285CD007467879BD68001F3AD0401EE0
:2052500004D0401E2FD0401E10D04AE0F888202847DC03A8002120220BF087FDFA8803A800
:2052700029460AF017FA44F002043AE00BA86B682968436005F1080201600DAB116850684C
:20529000196002F10805586029686B680FAA083553602846116011AB026841681A6044F064
:2052B000080459601DE029880DF10A0044F00404018016E0298802A80180BDF8081042F2D3
:2052D0000E0012F077F815F8028F44F0010408F00100C8F3800BC8F3401A1390C8F3400373
:2052F00014933F68002FA6D1019811F094FE3668002E8FD1009811F08EFE99F82870634D54
:20531000022F18D0A008C0F0BC805F4903A8202210F0B4FF002840F0B480012F04D1E87897
:20533000401CE87099F82870032F04D12879401C287199F82870002F4DD1A86A401CA862F5
:20535000600820D3B8F1000F04D105F13E00494612F05EF942F20F00414612F032F8139997
:2053700042F20A0012F02DF8149942F2100012F028F842F21100594612F023F842F212005E
:20539000514612F01EF84FF40050494612F0BCF9B9F81A10502011F03FFCB9F81A00B9F872
:2053B0000010D9F82C304A460DF00EFBB9F81A004946288705F13E0012F02AF9687801289F
:2053D0005AD0002001210CF06DF941F2707003210CF068F950E0022F4ED1E00805D3BDF866
:2053F0000A1042F2140011F0E5FF200913D342F215000BA912F088F942F216000DA912F0C5
:2054100083F942F217000FA912F07EF942F2180011A912F079F9286B4946401C28634FF4BE
:20543000005012F071F9002003210CF03BF96878012821D0012000276870154C6F7104F1DC
:20545000E000064611F066FF012802D1304612F071F911F0EBFD074611F0E8FD42F21071FB
:2054700000EB07200DF024FA206A01F57A6112F0EEF8304612F05CF9D5F8981009B1484622
:20549000884715B0BDE8F08F8986010048130020A41000202DE9F04706460020ADF1380D49
:2054B000DFF89092ADF80C00A0480F460168A34D097D252900F00E81006805A96C3006F0A1
:2054D00081FE002818BFC0B240F02D8197480068C18AC9080DD3007D03280AD09DF81F0075
:2054F00038B99DF820004C463870B5342070002019E101A804A909F03FFFA5F12F018A4606
:2055100091F82F30019A3468DAF808104FF47A78404641F208155843891A08FB120008FB11
:2055300001F1001B091B8D42C8BF002965DC854205DD002803DD346804F5915434609DF816
:205550001F00002857D042F204000DF135010EF031FA10F09FFF044606980DA9241A42F28A
:2055700006000EF027FA9DF834109DF81D00FF2904BF0A218DF83410FF2808BF0A209DF8DF
:2055900034206B499DF81C30B4FBF1F1801880B24843991008FB01F1814298BF081C2D180B
:2055B00005A810F024FD9DF81C203468C446B0FBF2F15143411A8BB20CFB02F2614659439E
:2055D000531A521A1B1B121B954201D9002A08D56942994216D2002B14D5B5FBFCF109B2ED
:2055F00003E06900B1FBFCF189B232684FF4916303FB012405E0002004E0306841F630346B
:205610002418346005460DF1120102A809F0B4FE0298DAF80810B4FBF8F21018029081425F
:2056300003D99AF82F30834204D94B4603F15804267836BB9DF81C0055190004A84298BF17
:205650002D1A9DF81F00002808BF9DF8200016D09DF81C00B5FBF0F084B29DF833000EF078
:205670006DFB9DF83120014620460EF0ABFC044610F0AAFC024608A920460EF0F1FA4C46B0
:205690000DE0814204D8BDF81200401CADF812004C46BDF8120094F85B100CF05EF9387049
:2056B000224E84F8B5003068007D05287FF41FAF2148007800287FF41AAF387803A9ADF870
:2056D0000C0042F20C0004F08BFCBDF80C00A4F8B0000CE768460DF10E0109F04DFE30685C
:2056F000009A2B7841F208144FF47A7101FB0202009259438A1A944210DCA1F5FA61914288
:20571000BCBF00F5FA6030604C4694F85B10208F0CF023F901460020397002E039784C469A
:20573000652084F8B5100EB0BDE8F087640E0020A0860100F02D002035120020672F0020A6
:20575000F0B504460846ADF16C0D401E6BD0401E0DD0801E00F00381401E00F0E980401EEA
:2057700000F0DB80401E00F0A88000203CE142F2010007A90EF01EF942F20B0008A90EF033
:2057900019F942F206000DF165010EF013F942F207000DF166010EF00DF942F2050019A9A0
:2057B0000EF008F904A809F0A1FC05460DF1670142F209000EF0FEF89DF86700002808BFCB
:2057D000002303D0022010F0F7F8034607A8006808A920600988271D3C46B81C218005F060
:2057F00007079DF865609DF864109DF8662000F8011B9DF8674000F8016B03F0030600F865
:20581000012B620747EA926104AC41EA8611012700F8011B9DF8672000942946019706F064
:2058300049FE0A3099E042F206000DF165010EF0C1F842F207000DF166010EF0BBF842F284
:20585000040019A90EF0B6F804A809F04FFC05460DF1670142F208000EF0ACF89DF867004B
:20587000002808BF002303D0012010F0A5F803469DF864009DF8657004F8010B9DF8666066
:2058900004F8017B9DF867209DF86770790704F8016B03F0030705F0070646EA916004AE3E
:2058B00040EA8710294604F8010B002700962046019706F0FFFD001D4FE042F2150011A9A4
:2058D0000EF078F813AD42F2160029460EF072F815AE42F2170031460EF06CF817AF42F288
:2058F000180039460EF066F811A801682160406860606A6804F108035A602868186030686E
:2059100003F10801086074684C60386801F1080528607A686A60202066E042F214000DF1EB
:2059300022010EF047F8BDF8221002200A1258E009A8002120220BF018FA42F2130009A980
:205950000EF038F809A811F01BFC024609A9204609F0A0FE09A811F013FC80B244E042F2FE
:205970000E0002A90EF026F80DF10A0142F20F000EF020F80DF10B0142F20A000EF01AF888
:2059900003A942F210000EF015F80DF10D0142F211000EF00FF80DF10E0142F212000EF055
:2059B00009F8BDF808009DF80B209DF80C709DF80D609DF80E509DF80A1004F8010B02F0AA
:2059D0000102001204F8010B07F0010042EA400206F0010042EA800205F0070042EA401215
:2059F000042004F8011B22701BB0F0BD2DE9F04F06469E48001D0068ADF1340D80470B9004
:205A10000AA9822004F09AFB9DF8280018BB00248DF828404FF6FF75ADF804509DF8280088
:205A3000ADF80650FF2108228DF8000002A811F08DFE8DF81840D420694601F067FF9DF8EA
:205A50002800401CC0B28DF828003228E4DB82200AA901F05BFF0020DFF808A2DFF80882D8
:205A70008DF8280081469DF828008DF8019069468DF80000D02004F061FB01274D46E8B9FF
:205A90009DF80B30012B07D19DF80A0020B90DF1020011F011FA88B9747B002C0CBF052250
:205AB00009224F469C4209D10DF1020006F10E0110F0A0FD002818BF012507D1002F40F05F
:205AD000BF801DB9707F002800F0BA804C469DF828008DF8214008A98DF82000D12004F0F0
:205AF0002DFB002832D19DF82200FF282ED08DF800006946D42004F021FB002833D102A859
:205B1000311D082210F076FD00B330887788ADF80400ADF8067045B1307B9DF82810B769CE
:205B30008DF818000DEB81010F61D420694601F0EDFE75B1307F9DF82310884209D08DF88A
:205B5000230008A9D12001F0E1FE02E0641C322CBDDB322C74D14F468DF80070D420694678
:205B700004F0ECFA28B1DAF808100B988847192074E002AB184611F09FF94C4600B101246D
:205B90002046341D30B918462146082210F032FD00284AD030887388327BADF804009DF857
:205BB0002810ADF80630002D8DF818200DEB810000F110000CBF4946B1690822016002A8B5
:205BD000214611F091F998F8380030B1D8F888201AB19DF80010204690474C469DF82800A6
:205BF0008DF8214008A98DF82000D12004F0A6FAE82807D09DF82200FF2803D0641C322C5E
:205C1000ECDB10E09DF800008DF82490337F8DF8220069468DF82330D42001F077FE08A904
:205C3000D12001F073FE322C02DB7F1C322F93DB322F05D1DAF808100B9888471A200DE0A2
:205C50009DF82800401CC0B202288DF82800FFF60AAFDAF808100B98884748460DB0BDE8D8
:205C7000F08FC0468C140020EC1300208C1400202DE9FF47854FDFF830828C4CF8680028D7
:205C90003ED18F4D8249843D2868814210D0814981420DD0804981420AD08049814207D017
:205CB0007F49814204D07F49814201D011F002FB10F0D0FD29684FF0FF32012805D1C1F39A
:205CD0000330083805D0C01F01D0012A01D1012000E00020F8700EF039FC142804D140466C
:205CF00000F1E001C0F8A4100FF084FF216A19B911F0E0FA2046016A096A07F11000884781
:205D1000632002A90EF062F8DFF8A49109F1B70000780FF059FF06464046D0F8981090F897
:205D30009D20B0F896C041F00F0102F03F02C0F898102CF0070C80F89D204CF0010CA0F87F
:205D500096C0B37A4FF0000A00F188057BB99DF8083002F0C0023F3303F03F0313436B7557
:205D7000EB8A4FF6C0721A4042F018020DE09DF8083002F0C00203F03F0313436B75EB8A33
:205D90004FF6E0721A4042F02002EA82307B052814BF2420292088F89C00F27A307B401D7A
:205DB0005043E2690A230CF0010C90FBF3F0C0044CEA1040E881F07A1923800390FBF3F007
:205DD00060F31C212961288B117D4FF6F77361F3020003EA00012883107D00F008000843EA
:205DF000288399F9A6000DF057FEA8F8A200716833683089401EA8F88AA0414303EB510004
:205E10004FF47A71B0FBF1F0A8F8A800C8F88CA0687B00F0F00040F00100687311F09EFB1B
:205E3000A0B9F07A234A99F8B730B1FBF0F01070F07A022BB1FBF0F0C0B2B1FBF0F0787095
:205E500004D11D4802214170A8260670F86850B9206A0668616A194807F110032A46B047E1
:205E70003C4605460DE050460BF020F9206A86684FF002098DE80006F868524629461346B1
:205E9000B047E5600090BDE8FF87C0468819002000F0022000F0012000F00020008002205F
:205EB0000080012000800020280D002028160020A8110020CC190020C8180020302D002083
:205ED000181300502DE9F04F0128ADF1140D40F0F180DFF81882D8F8DC00012840F0E7807C
:205EF0000220C8F8DC0011F00BFD029001200EF027FA061C06D00120C8F8DC00029811F0A9
:205F1000FBFCD9E011F0F4FC03906D484FF00009C0F8009001200FF0D3FD012818BFCDF843
:205F3000009004D148460DF077F9012000906548654FC0F800903868112011F0EBFA0028B8
:205F50000CBF4F460127102011F0E4FA08B147F002070F2011F0DEFA08B147F004070B2073
:205F700011F0D8FA28B159480068594D016B288888470A2011F0CEFA4D4600B101254FF02F
:205F9000805B28460BF5DC7520B12868514C016B208888475048012404602868816947F0A4
:205FB000200088474D48046011F0AEFA00F001010191400814D24A4811F03BFA8246BAF153
:205FD000040FF8D0BAF1010F05D1DBF8D80142684348032190474349086820F003000860F2
:205FF000484600F085F838482B680068986B8047019801280DD0BAF1010F05D1DBF8D80175
:2060100042683748214690473649086840F0030008602C48046028684169384688470B20F5
:2060300011F078FA20B12868294BC16A188888470A2011F06FFA20B12868264BC16A18883D
:206050008847254804600322C8F8DC20234BC3F800902868416B384688470128F9D1042056
:206070000EF06EF90546184F15481F490460386808688009FCD30098012802D120460DF071
:20609000CBF811F02FFA08200EF05AF907460398C8F8DC4011F028FC0CF0C4FC029811F04A
:2060B0002BFC57EA050018BF4FF0FF3604E06FF0040601E06FF00106304605B0BDE8F08F35
:2060D0000C400940000222432C200940B8010010AA880100A688010028200860800104437C
:2060F000004003402422084014100940940F00202DE9F047DFF80CA20746AAF13500DFF889
:20611000F8810068800880F0E7800FF045FE814908310B6800261C17641C990D0AD2C0F16B
:206130003E0110F10A0F4FEAE101D8BF08218C42B8BF0C1CDFF8C4C1990E0FD2590E0DD383
:206150006246143A1168C1F304211629A8BF20391268C2F30462162A0EDB0CE0634AD2F8C7
:206170007C11C1F304611629A8BF20391268C2F30442162A00DB203A61189146162905DA12
:2061900011F10A0FB8BF6FF0090100E01521584C584D01F01F0242F4F85222802A6812F0CD
:2061B000030F18BF0126D20828BF46F002060FB146F00406424692F90740041B052C04DA38
:2061D0009479B44208BF918866D00F28A0F10F0827DB08EB0014A4F1F0084FEA282EBEF1E3
:2061F000070F88BF4FF0070E7546062D88BF06255CF82570042404EB850465462C59E41BC6
:2062100004F0FF05F70824BFC4F307273D44B70824BFC4F307473D44770828BF05EB146537
:2062300001E00025AE465CF82EC0F7080CF0FF0424BFCCF307273C44B70824BFCCF3074715
:206250003C44770828BF04EB1C64ADB2A8EB0E27B9EB010105FB07F505F1800504EB15246D
:20627000D8BF012103F0FF0334254D43A9B259434FF6FF73B1FBF4F18B4238BF191C802897
:2062900089B2918005DA10F1800FB8BF6FF07F0000E07F20D0719671194800681F29106096
:2062B0004FF0000008D340F2FF128A4206D24908401C8A42FBD301E01F219180124F0F39AB
:2062D000090940EAC10047EA0001CAF8FB1F0026CAF8FF6FBDE8F0870C490D4F42460820D0
:2062F0000F60921D1070BDE8F087C0463C1100506E62084024220840F43100209C13005047
:20631000082009403500094000E7A48030100940FDFDA400AC3F0050F0B500214422ADF147
:20633000540D02A80AF021FDF22013A910F0AAFF804DBDF84C0013A9A5F86800F32010F011
:20635000A1FFBDF84C000DF10901A5F86A00E22010F088FF688CADF81200410806D305F131
:206370000C01096805A80160BDF81200810805D3291D098806A80180BDF81200C10807D3E9
:2063900005F1100109680DF11A000160BDF81200010908D30DF11E0005F14C01242209F0B2
:2063B00079F9BDF81200400903D3A86A12906F6A1197012010F048FCBDF8120041082CBFE0
:2063D0000F240B24810824BFA41CA4B2C10824BF241DA4B2010924BF2434A4B2400924BFBF
:2063F0000834A4B220460FF0AFFC071C00F09F8005260DF1090100F8016B0A68026049689D
:206410004160BDF81210083011F090F8BDF81210844648080BD3BDF81410604611F086F866
:20643000BDF8161011F082F8BDF812108446880807D3BDF81810604611F078F8BDF8121020
:206450008446C8080BD3BDF81A10604611F06EF8BDF81C1011F06AF88446BDF81210364A63
:206470009388080949D3BDF81E10604611F05EF8BDF8201011F05AF8BDF8221011F056F876
:20649000BDF8241011F052F8BDF8261011F04EF8BDF8281011F04AF8BDF82A1011F046F828
:2064B000BDF82C1011F042F8BDF82E1011F03EF8BDF8301011F03AF8BDF8321011F036F828
:2064D000BDF8341011F032F8BDF8361011F02EF8BDF8381011F02AF8BDF83A1011F026F828
:2064F000BDF83C1011F022F8194611F01FF8117811F01CF8BDF812108446480906D31199E6
:2065100060460EF0A0FB12990EF09DFB05F11401224630463B4604F0C7FE0820ADF8026099
:20653000064D01972968ADF800006846884715B0F0BDC04690120020A4100020B0140020BB
:206550002DE9FE4F0646824AF07B20B91146491C0978022908DB012803D11046007802282C
:2065700002DBF120BDE8FE8F346AB6F8289096F8347096F835B0B58B4FF000085FEA040A64
:2065900017D0744890F83830002B2ED0016D00292BD004F0FF0088476E49096D04B20AF4FA
:2065B0007F008847001900B2001D00B2C43084B200E0C4240DB12D1DADB26748007801283A
:2065D00009D147B16548C11991F8048010F80B002418641DA4B205EB090020184044801CCE
:2065F00080B20FF039FE071C02D11A20BDE8FE8F08EB09002B193881002D07EB03007860CE
:206610000EBF0020E019801C00217422C7F8A00007F10C0011F09AF84C442D1907F13C0031
:20663000FF211022A7F84C5011F090F807F12C000F21102211F08AF800243C707C7078688F
:20665000716A328D09F026F807F1800006F12C010B2209F01FF807F18C00314610F0A8FA03
:206670007089A7F89600307B87F89800707B06F10E0587F899002A6869460A60AB888B8024
:20669000AA798A719DF800102046012908BF01209DF80110012908BF40F004009DF802103D
:2066B000012908BF40F008009DF80310012908BF40F010009DF80410012908BF40F02000DE
:2066D0009DF80510012908BF40F040009DF80610012908BF40F08000A7F89A00707D87F8AE
:2066F0009C00B07D87F89D00B28BA7F8A42022B1D7F8A000B16908F0CDFFB07F87F8A60091
:20671000306AC7F8A800B7F8A400C0B1D7F8A000A8B17868401E7860F82101707868401EFE
:2067300078600470B7F8A410B7F8A4607868401A786039897018801C38817868B8650848E9
:20675000007839460CF084F82046BDE8FE8FC046920E0020EC13002044120020AC8A010090
:20677000141500202DE9F043002B08BF002A10D10029BCBF00204FF0004106DB50EA010713
:206790001CBF6FF000006FF000410AF0BAFDBDE8F0835FEA530898EA610803D50026404237
:2067B00066EB01015FF0000913F0004E03D00026524266EB03031C461546002C08BF8D426A
:2067D0009CBF2C1C0025070C47EA01470E0CB44208BFBD429EBF240444EA15442D04070A31
:2067F00047EA01670E0AB44208BFBD429EBF240244EA15642D02470847EAC1774E08B442BF
:2068100008BFBD4200F29280870847EA81778E08B44208BFBD427BD8C70847EA4177CE08B3
:20683000B44208BFBD4265D8070947EA01770E09B44208BFBD424FD8470947EAC1674E099C
:20685000B44208BFBD4239D8870947EA81678E09B44208BFBD4223D8C70947EA4167CE09E4
:20687000B44208BFBD420DD8E60146EA5566EF01B14208BFB84201D3C01BB14159EB0909FA
:206890004EEB0E0EA60146EA9566AF01B14208BFB84201D3C01BB14159EB09094EEB0E0E11
:2068B000660146EAD5666F01B14208BFB84201D3C01BB14159EB09094EEB0E0E260146EA2F
:2068D00015762F01B14208BFB84201D3C01BB14159EB09094EEB0E0EE60046EA5576EF001D
:2068F000B14208BFB84201D3C01BB14159EB09094EEB0E0EA60046EA9576AF00B14208BF3E
:20691000B84201D3C01BB14159EB09094EEB0E0E660046EAD5766F00B14208BFB84201D349
:20693000C01BB14159EB09094EEB0E0EA14208BFA84201D3401BA14159EB09094EEB0E0E7F
:20695000A34208BFAA423EBF2D0A45EA0465240A8AD373464A465FEA080803D50026404216
:2069700066EB01015FEA480803D50026524266EB03031E4617460B46024631463846BDE83E
:20699000F0832DE9F043044694F830900F46984615468B20ADF1340D0DF10A0103F0CEFBB8
:2069B0008A20694603F0CAFB94F8250000283ED1B9F1000F19D1BDF80A104FF6FE708842DF
:2069D00005DCBDF80A1088422FD1694615E0B4F844009DF80A608DF80C0000128DF80D0065
:2069F000BDF80A008DF80E601BE0B9F1020F09D0B9F1030F19D104F1280103A810F07EFE5B
:206A1000092612E0207CC00934BFB4F84200B4F844008DF80C0000128DF80D00208D8DF8A8
:206A30000E00001205268DF80F00002013E002280CBF05260926012818BF04F11C0104D11E
:206A5000892006A903F07AFB06A9324603A810F04BFA94F8260006EB0D01C8723A4603A839
:206A700031460AF013FC002840F08E80B9F1000F19D1BDF80A104FF6FE70884205DCBDF89B
:206A90000A1088422FD1694615E0B4F844009DF80A608DF8200000128DF82100BDF80A0053
:206AB0008DF822601BE0B9F1020F09D0B9F1030F19D104F1280108A810F020FE082012E084
:206AD000207CC00934BFB4F84200B4F844008DF8200000128DF82100208D8DF822000012AD
:206AF0008DF8230004203E6881460BA9822003F025FB9DF82C10307B8142D8BF9DF82C004D
:206B1000002841D007460024722029460FF030F9B0689DF82C102018C8F800000078814276
:206B30002EDD2B68C10001EB0011D8F80000C91829604278012A1FD0807828BBB9F1040F43
:206B500006D0091D08A80FF0F1FF012816D017E008884B888DF82800042208A98DF82A30BE
:206B700000128DF8290018128DF82B000AA80FF041FD012802D003E0807828B9002004E0C1
:206B90007F1E04F10304BFD1F3200DB0BDE8F0832DE9F047064637680C465FEA0208ADF159
:206BB000180D14BF00214FF0FF3107F14800814610F096FE002808BF0B2000F0DF80002514
:206BD00065707148FC60B8F1010F057004D065700220FC600EF072FD2078012840F29080F6
:206BF000801E012857D9801E01282CD9801E012800F2B88010F08CFE8246A078009021783E
:206C10002846062908BF0120019001200290A068228A6368E16806F063FE0746504610F099
:206C300073FE002F40F0A080B8F1000F02D010F0BFF802E030460FF0EDF9002800F08780B7
:206C500010F072FD21E010F063FE012782460097A168A278606824782B46042C08BF3B1C86
:206C700008F096FA0746504610F04EFE002F7BD1B8F1000F02D010F09BF802E030460FF05E
:206C9000C9F9002863D00EF0A1FC3E49C1F8B0510D60074668E010F03BFE8246E08A0090EE
:206CB000E0680190208B0290A0780390207D04900121059122782846022A08BF081CA368F0
:206CD000E178626802F0F4FD0746504610F01CFE002F49D1B8F1000F02D010F069F802E08B
:206CF00030460FF097F9002831D00EF09FFC071C3AD1E078A168E28A236909F0FDFEC8E793
:206D100010F006FE8246E08A0090E0680190208B0290A0780390207D049001200590277856
:206D300007B90546E1786268A368284602F07EFE0746504610F0E8FDB7B9B8F1000F02D06C
:206D500010F036F802E030460FF064F908B9142014E00EF053FC071C06D1E07821690CF033
:206D70004BFC96E74FF0FF37B8F1010F02D002200EF08CFC484610F0AFFD384606B0BDE884
:206D9000F087C04650450240023200202DE9FE4F794C074694F83D00002800F0DA80DFF8B4
:206DB000DC81B7F84210B8F88A00884240F0D18007F128000FF090F8002800F0CA800025B2
:206DD00098F88D0084F83D5010B102200FF0F2FB6148007810B101200FF0ECFB387C4009C8
:206DF00005D310200FF0E6FB802010F0B3FA20200DF058FE594E06F120000CF065FD7A68BD
:206E100051781078334600EB0120C0F30321C0F3003684F8391000F00F0184F83A60C0F33E
:206E3000031684F83E1098F8B30088F890600F2804D0884202DDD67806B9014688F87110A3
:206E500098F871A083F84050BAF10F0F09D194F83B0002287DD10EF043FA07F073FBBDE84F
:206E7000FE8F3F480078012803D00120294600F039FE43484068804700900FF0DBF93948E5
:206E9000DFF80091DFF8E0B0066898F8712099F80030D9F80400311A980091FBF0F05BF84C
:206EB00022100DF093FCC9F804605BF82A0001912E4EB060F0600CF061FE019831680EF069
:206ED00029FA09F03FFA2E4900988968884794F83B0002280DD127480CF0F6FC98F8712031
:206EF00034F812004FF470719140091A21480FF02FF898F89030388929460FF02AFA206377
:206F10000F2B14D098F8711094F83900994208D0401C6FF00F0598408101A1EB80016D18FF
:206F300005E0401C98408501A5EB8005A03D6563022004F1200584F8380028460CF0C4FCCE
:206F50000B48A062616B28460FF002F8102010F001FABDE8FE8FC0467F30002024310020F2
:206F7000E81A00206016002050890100281A00208107010034310020F0170020A8110020FF
:206F90008C140020CC1900202DE9F04F7A4C804608460026ADF1440D0028089004F105011D
:206FB0000E701ABF006800684FF0FF30B8F11D0F0C900CBF1E201D20099009F0DBFD2422C5
:206FD0004046314610F09EF915250D9605210E9620460F96C0880A9104460B94A1427EDA54
:206FF00065484779002F6AD1641F404602AAA4B221460AF079FCBDF814709DF81130781D25
:207010001FFA80FAD80951D233F07F035AD0029A0C98904256D0099829460AF095FA002801
:2070300050DC8EB9611E40463A4689B20FF082FA50B90299E01B80B2B1F5805F0B9041D18F
:207050000F904FF0040906E0A9460AEB0500B9F1000F85B236D007EB09001FFA80FB21467A
:20707000052206AB40460FF096FD099806AA59460CF0EEFF26B90E98401C80B20E9006E0A0
:20709000E01B81B209984A4653460CF0DDFA0D989DF818205946401C22F0400280B20D9085
:2070B00009988DF8182010F02DF90BE098080CD2544507DA3049052048710F4638714FF0C5
:2070D000FF3056E0E41BA4B204E0404621460DF027F804460A98A04282DB2748C0880B9973
:2070F000761C0446022E0A91FFF678AF0C98B0F1FF3F14D020480899C58008890090C868B7
:2071100001908A88CB880868099904F057FF1A480D9E0746C588FC80701C80B20D900F98E8
:20713000C0B101460C2202AB40460FF034FD0D9F02980E9EC5F5805404210C22ADF80E4030
:2071500002ABADF81070401C02900998ADF812600AF034FA09980CF079FC0748407900283D
:20717000ADD10548C580404609F004FDC5F5805738B211B0BDE8F08F481A00202DE9F04146
:207190001C4615468C4208BF854282BF00230022E5E0002C08BF002D0AD100290EBF002862
:2071B0006FF000006FF0000100F0E1F8BDE8F0815FF000085FF0000E002C08BF8D429CBF50
:2071D0002C1C0025070C47EA01470E0CB44208BFBD429EBF5FEA044444EA15445FEA0545C8
:2071F000070A47EA01670E0AB44208BFBD429EBF5FEA042444EA15645FEA0525470847EA99
:20721000C1774E08B44208BFBD4200F29380870847EA81778E08B44208BFBD427CD8C708E2
:2072300047EA4177CE08B44208BFBD4266D8070947EA01770E09B44208BFBD4250D8470981
:2072500047EAC1674E09B44208BFBD423AD8870947EA81678E09B44208BFBD4224D8C709D8
:2072700047EA4167CE09B44208BFBD420DD8E60146EA5566EF01B14208BFB84201D3C01B88
:20729000B14158EB08085EEB0E0EA60146EA95664FEA8517B14208BFB84201D3C01BB14138
:2072B00058EB08084EEB0E0E660146EAD5666F01B14208BFB84201D3C01BB14158EB08082C
:2072D0004EEB0E0E260146EA15762F01B14208BFB84201D3C01BB14158EB08085EEB0E0E2A
:2072F000E60046EA5576EF00B14208BFB84201D3C01BB14158EB08084EEB0E0EA60046EADB
:207310009576AF00B14208BFB84201D3C01BB14158EB08084EEB0E0E660046EAD5766F0056
:20733000B14208BFB84201D3C01BB14158EB08085EEB0E0EA14208BFA84201D3401BA1418B
:2073500058EB08085EEB0E0EA34208BFAA423EBF2D0A45EA0465240A89D3734642461E46D2
:2073700017460B46024631463846BDE8F08170472DE9F04306467078ADF1140D002840F0B1
:20739000D78096F8961002291CBF0329E82096F88B108029C8BFE82096F88C10092901DB7F
:2073B0000A2900DDE82096F88D10002900F0BF80042980F2BC80002840F0BA80614C04F113
:2073D000B7000078884204D006F18D01E82001F061FF06F18C01E72001F05CFF06F18B0198
:2073F000E12001F057FF06F19801502001F052FF96F8960002280CD04FF6FE70A4F88400F6
:2074100006F18E0104F17A0010F078F906F18E0504E006F18E052888A4F884004A4806F1A5
:2074300080010B220FF060FD4FF001080220A6F816802946307501A80FF0BAFB96F89A708B
:20745000B6F89890706806F19A01002FA0F1010070600CBF002040464F780FB140F0020021
:207470008F780FB140F00400CF780FB140F008000F790FB140F040004F790FB140F08000D2
:2074900071684A1E7260314B0870377D71680025481C3062781E087030893565801C30817F
:2074B0001878B565A0B30427F08A86F8695006F18E0186F86B70C00934BF94F8890094F8A7
:2074D000B20086F86A0006F16C0010F017F9204C206810F47F0F0CD086F82C70206806F194
:2074F0002C01424600F47F003063304602F01EF9206810F0FF0F0BD02A2086F83C00206845
:2075100006F13C0100F0FF003064304606F0B0FC00953046832101AA4B46FCF7A3FB071CED
:2075300002D1304606F030FE381C01D106E0E82070701820307030460BF068FC05B0BDE8D3
:20755000F083C046A8110020743000202414002014870100F0B542F20400ADF11C0D0DF16F
:2075700015010CF027FA42F2050005A90CF022FA664C67489DF81510A06664204143216619
:207590006449C4F884109DF814104843E0676248C4F8A0006148007880B942F2020069460E
:2075B0000CF008FA68460EF0E5FE04F15C000BF08BFD04F134000BF0CFFF27E042F203002A
:2075D00069460CF0F7F90EF0FFFC0546684629460BF098FB2D1A04F1780084F85B500BF03B
:2075F00073FD04F134000BF019FD012742F20200694684F854700CF0DDF968460EF0BAFE4E
:2076100004F15C000BF060FD84F85870E8200DF116010CF0DBFB9DF81600032804BF0120C4
:2076300084F8B40094F8B80000286DD13C4D0021302205F1080009F098FB204600213322FE
:2076500009F093FB3748E861374F6F6105F110000BF03AFD42F21B000DF117010CF0AAF939
:207670009DF817000DF1170185F82C0042F21C000CF0A0F99DF817109DF8170085F82D1088
:2076900095F82C10012641B148010EF075FC286308B910F03FF895F82D0040B100EB8000A7
:2076B00080B20EF069FC686308B910F033F81F4905F138000A270A684B6802607F1E4360E0
:2076D00000F10800F7D1002195F82C7085F8881047B1286BFF220346C2777F1E997703F1AB
:2076F0002000F8D195F82D7047B1686BFF22034602717F1ED97003F10500F8D12846062281
:2077100009F033FB84F8B86007B0F0BDF02D002079390100E9F20000A1760100ED13002037
:20773000AC2E002069B00000002A7515E88A01002DE9FE4F0CAF8A4699460446D7F804B065
:207750000292594603F0C4FA06466A480578002E00F0CB803888F082DFF8AC8134751DB1A4
:20777000012C04BF1520307506F1800059460B220FF0BAFB012C04D00D2C1CBF7068401CEF
:2077900000D170683062002598F8380035650028B56543D0DFF864B1052C18BF012C38D198
:2077B0004FF0040AF18A86F86BA0534886F86950C90938BF29380078029986F86A0006F17A
:2077D0006C000FF09BFF0BEB8407386810F47F0F0CD086F82CA0386806F12C01012200F4E0
:2077F0007F003063304601F0A1FF386810F0FF0F4FF0030A0BD02A2086F83C00386806F1F0
:207810003C0100F0FF003064304606F031FB98F8380018B1D8F898100D2C13D00095029AAA
:207830004B4630465146FCF71DFA071C5ED1E41F012C03D8707E40F020007076304606F0A3
:20785000A3FC53E005205C4686F86B00343409B1FF208847206810F0F70F12D02A2086F84E
:207870003C0098F80120206806F13C01012A00F0FF0030641CBF20F008003064304606F0AE
:20789000F7FA0095029A4B4630460321FCF7EAF9071C2BD11A4806603489756801A9642006
:2078B0000CF094FA174E6D1E231DA01C99B2A6F87800C1F3022040F0080005F801090A1FA3
:2078D000297091B2AA1CC6F88450104608F0CCFE9DF8040000280CBF49F24E0047F60E20CC
:2078F000C6F8C000C6F8800000E01A27F8B2BDE8FE8FC046241400205A1200200C87010041
:207910009C180020280D0020EC1300202DE9F041724B734ADFF8C0810C46D128014610DCB8
:20793000D12879D0713800F0B280401E00F0AA80401E00F0A380113810D04C3800F087809D
:2079500007E0D23853D0401E40D0401E33D0401E28D008460FF06BFC0B2802D1F420BDE86B
:20797000F0815B4D05EB8005A97809B9E87850B1E878884208BFFB2000F0A8802278914294
:207990006ADC904268DB534E7068804729786A7807464046401821460FF0A6FAB1683846F1
:2079B000884792E02178022956DA1846641C042200EB810086E0207832284DDA1746C10075
:2079D000241D182201EB001178187BE026783046022841DA2C2505FB0680611C10223930EC
:2079F0000FF082FA616905FB0680C1646DE022786178022A30DA02292EDA40462C2301EB9D
:207A100042064F1C03FB0205022285F8387000EB460000F5DE7018E022786178022A1BDA55
:207A3000322919DA2C23404603FB020595F830309942A4BF4B1C85F83030322303FB021139
:207A500001EB4101032240189030A41C3AE020786778022800DA17B1E820BDE8F0814146E9
:207A70002C22C5197E1C02FB00136A0083F8286002EBC50288180A227C30E6E72CB318467D
:207A900008221FE00CB310464FF496621AE0B4B9404600F17C04A0F1080200F1900300F5EB
:207AB000DE71022042F82C4F9360401E116104F10A0403F1960301F10401F3D105E0404617
:207AD0005822243021460FF00FFA0020BDE8F081287901008C140020A82100201C28002074
:207AF0006C2300202DE9FF47604C804660680F468047A246674E684D654C8146B8F1010F92
:207B10005AD00FF0B5F9002851D05948007800284DD158480078002849D15748007800283D
:207B300045D156480078002841D15548007800283DD154480078002839D153480078002803
:207B500035D152480078002831D1002009F0EAFA68BB207858BB012FA0461FD04F4F326AC9
:207B7000E86897F90010344611F1020F05D0926B97F900109047E868226A494E96F900101D
:207B900011F1020F05D0926B96F900109047E868226A6FF001013170397003E00C35203679
:207BB00028683268012188F80010D1698847DAF808104846884755E0012009F0B3FADAF8BB
:207BD000081048468847207801283DD1DFF8D49099F8BA000028FBD1306A436CE86802211B
:207BF00002AA98479DF80800A84660B199F8BA0048B92078012827D10020012F207023D076
:207C10000FF042F920E0DAF804008047264F0221814600222170306A7A81244B85688DE805
:207C30000600D8F80C0008373946A847002801D50FF040FB1E4991F90000401C0870DAF8D6
:207C50000810F7604846884720781A4D022803D1287808B10FF02EFB2878012802D0207897
:207C70000228FCD00090BDE8FF87C0468C140020043200200632002008320020053200201E
:207C900007320020CE1A0020CF1A0020D01A0020E91A00202816002088190020CC1A002018
:207CB000CD1A0020302D0020280D0020CD2E0100D11A0020E81A00202DE9F843644C074664
:207CD000207808B10FF0F6FAA0460120614988F800000978012902D00021FFF703FF5F4DE1
:207CF00060495F485C4C012F2A68D1F800900078A77035D9BF1E52D07F1E13D07F1E02D0D6
:207D1000781E47D043E092F86900207192F86A00E0700020607102F0A5FE2A68002A64D144
:207D3000BDE8F883002860D0564ED6F8981021B1032088472A6896F83800002855D0776D54
:207D5000002F52D0D06D20B102210023B8472A68776D106E002848D008210023B84743E0CD
:207D700000202071D18A4048C90934BF90F8891090F8B210E170A77837B990F867701FB1A0
:207D90000229C4BF0220E07002F06CFE2CE00FF091FA29E0002020710FF0E0FC24E0334FA6
:207DB00038788600D9F83C00804779683C22401AB0FBF6F0B0FBF2F151436278401A910197
:207DD000A1EB8201091AD9F83C003C318FB28047274906FB0700086791F8740000F0F0001B
:207DF00040F0020081F874002A682248007878B912B90FF05FFA2A685168087800F02000B1
:207E1000E0718878A0710878800901D20FF0ACFBA078042819D0184D68688047A178022901
:207E30000CD016490F7817B915490F7837B1022188F80010A9688847BDE8F883832188F8FC
:207E50000010A96888470EF035FCBDE8F883C04608320020E81A0020C8180020640E0020BF
:207E70002414002048160020A8110020CC190020280D0020003200208C1400200432002081
:207E900006320020EC1300202DE9F043894614460546ADF12C0D69460DF0CEF85FEA000804
:207EB00000F0C480AD1C0226284602A90BF0D9FA071C00F0BB809DF80900814509D0F6190C
:207ED0007D1908F10200B61CAD1CB6B2B042EBDCACE0401E05F1020500F08B80401E52D0E3
:207EF000801E38D0401E2BD0401E24D0401E18BF622040F0AB80202F40F0988028686F6811
:207F100005F10801206004F10806676001F108050A684B68326004F1100773602A68686811
:207F30003A6005F108067860306804F11801086073684B6089E0022F78D12888208084E090
:207F5000202F73DC20460021202208F00EFF3A462046294677E0042F68D12888AD1C208074
:207F700015F8010BA070287800F00100E0702878C0F3400020712878C0F38000607128787F
:207F90004011A07161E00A2F50DD0DF112000021162208F0EAFE28682D1D20602988271D30
:207FB00042F20B00398004A90BF004FDBDF81000A18888423ADCA81C10F8011BA17110F840
:207FD000011BE17110F8011B217210F8011B0123C1F3C202A2720DF1120200F0F7F928B3CB
:207FF0009DF82700A0819DF81670E78104F1100026E0042F1ADD0DF112000021162208F07B
:20801000B4FE15F8010B207015F8010B607015F8010BA07015F8011B0DF112020023C1F3D1
:20803000C2002071284600F0D1F908B967200DE09DF82700E0809DF81670278104F10A00A2
:208050000DF11601112207F025FB00200BB0BDE8F083FEE72DE9F04F674C2068ADF12C0D72
:20807000002840F0C58004F124063068002800F0BF8062480078022800F0BA80614D281DDC
:20809000006880470A90606AB046074678B35C4E4FF0000A4FF01D093B7D0820711E11F8FF
:2080B000012F9A421ED0401EF9D14046394652460CF052FD787E30F07F0005D194F82F0080
:2080D000401E84F82F0004E094F82E00401E84F82E0087F8019057F80CBC384609F0FAFD4C
:2080F0005F4602E0BA4657F80C7C002FD4D1352007F0B8FB444EA968002849D1452007F0FE
:20811000B1FBA96800283DD1D8F8000038B1017D252904D050F80C0C0028F8D110E078B199
:2081300096F8580050B3684601A907F025F9374800990078001F884213D8012086F8550081
:20815000152007F08FFBA96848B10A98884720680DF106016C3004F035F858B10FE00A98FA
:2081700045E0252007F07EFBA9680A988847002086F855000420FFF79FFD39E0192001F0A7
:208190004FF935E00A98884708200BF0FBFD2FE00A98884796F8B400A8B10EF04BF93178E0
:2081B00000290EBF0921491EC9B201EB81017118D1F802100FF0B0FA42F21071814284BF77
:2081D0006431081A00D800206968002808BF0620DBD0C6F8980088470446D6F8A010D6F894
:2081F000980006F1A8020CF0ABFFA968204688470BB0BDE8F08FC046640E00207F1600201E
:20821000F88A01008C140020F02D0020672F0020BCB50546694800880021820804D2B5F8F5
:208230009A20D20828BFE82110F0600F04D1B5F89A00800828BFE8212889B0F5006FA8BF7B
:20825000E82195F8980030B995F89400002808BFF52100F0AF80002940F0AC80DFF860E115
:20827000D5F8A870DFF860C19EF8381017B9012903D028E0002900F09C80D5F8A8106046FE
:208290008D3041F002010778C5F8A8101FB141F00801C5F8A810D5F8A81011F0FF0F05D001
:2082B0002A2085F83C0001F0FF072F6411F47F0F07D00420D5F8A87085F82C0007F47F008B
:2082D00028639EF83810002059B33E4995F894700B6804226FB925232B750968C98AC909A2
:2082F00034BF9CF889109CF8B21085F86A10891C08E015212975D98AC90934BF9CF889104B
:208310009CF8B21085F86A1085F86B2005F18C0785F869003B6805F16C010B607A684A608C
:2083300001E00121297595F89C70EF760446AC65B5F89A102C6595F89D30E9826A682B7712
:2083500095F82C702A620F2F09D00246B5F8A40005F12C0100B90122284601F0E7F928BB87
:2083700095F83C10FF2901D1AF6D27B105F13C01284605F07DFDC8B9009495F89810B5F81F
:20839000963005F18C022846FBF76CFC071C0CD12889B0F5006F03DA284605F0F5FE04E0DF
:2083B000E5206870284609F095FC3846011C01D1BCBD1821284607F04BFDBCBD201500203E
:2083D000EC130020640E0020A81100202DE9F04F154601F00708C1F3C2074FEAA119044699
:2083F00083460C22ADF1240D0021684608F0BDFC6248B8F1000F36D0B8F1010F7ED122880D
:2084100001A9A6780A80E41C8E7014F8011B01F00F018DF8081022880DF10A031A80BDF832
:208430000A30A41C4FF0000C6B75019ECDF818C04168B14207D1017A9DF80820914202D179
:208450004189994208D006990C30491C06290691EED96046614601E0017840788DF80010CE
:208470008DF8010022E014F8013B14F8016B8DF8003000228DF801600C38079210F80C1FD7
:20849000994202D14178B14207D00799491C06290791F3D91046014603E04168027A408995
:2084B000687501918DF80820ADF80A0003A806F01DFE9DF800109DF80100B8F1000F11D051
:2084D000B8F1010F1AD1019904989DF808209DF81460484086EA02010918BDF80A20BDF83C
:2084F000160004E09DF80C2051409DF80D205040401803D1EF701FB1022F05D0002039E034
:208510002188281DA41C0180B9F1010F27D0B9F1020F2CD1BDF80A10281DC91DCA10214678
:2085300007F0B8F8BDF80A00C11D04EBE104F0B1401E811000EB5171C910C9B26D182B7959
:208550008710012600EB577121F00701401AC0B2401C06FA00F0FF301840287107E0291D1C
:2085700020460AF055FF207804EB8004641CA4EB0B04A0B209B0BDE8F08FC046D4150020D0
:208590002DE9F04FADF1840D209002F007FB0EF061F90026012804D10EF09EFB022808BF9F
:2085B00001265B490868C0F38150012806D151F80C0C0127010E07FA01F006435548007804
:2085D0000DF0A8FD544D2C46286038B1FF2204F1400107467F1E01F8012BFBD12099096809
:2085F0004FF0000901F0FF02FE2A1DD0DDF880C001F0FF074A460123FF2F0ED0B84203D97A
:2086100003FA07F73E4201D002207EE001F0FF0147EA0909611881F840205CF8041F521C13
:2086300001F0FF07FE2FE7D1092005F04BFD2098002124220823606017A80FF049F94FF09F
:20865000010804F1240017AA8DF8748041460FF03BF9236843B3002794354FF0040BBA4635
:2086700008FA07F0064219D119EA000F04BF07F0FF0141F4C04105D0E019209B90F840105C
:2086900053F82110254804F027FCF8B24FF0FF310EF018F92368C5F800A001E0C5F800B06C
:2086B0007F1C2D1D9F42DBD301A80021302208230FF006F91A4E30780025102101AB099046
:2086D000184A009504F108000FF0F6F80DA82822082329460FF0ECF80DAA7068124914959A
:2086F0002B46139004F160000FF0DEF80F4951F80D0C474620F4F85040F4005041F80D0CB3
:208710000B4EC1F8FF7F2846376021B0BDE8F08FB43F005001320020542B0020007FC767DD
:20873000088B0100F1680100754101000D300940080009402DE9F843644C0026054666765F
:20875000687D0628A4BFE8216176A97D0E2903DD03281CBFE8216176032805D15C48008863
:2087700040083CBFE820607695F8280008B1E8206076E87D092801DB0A2801DDE82060761C
:20879000287E08B1042801DBE820607604F11807294638460CF058FE291D112207F12C0094
:2087B00006F078FF95F8280004F11809002804BF84F86060A87D04D095F8290084F86000BF
:2087D000688DA4F85600687E84F85800A87EDFF8048184F85900E87E822784F85A00287F05
:2087F00098F8A76084F85B0098F8B63084F85C70394F84F85D6005F11D01E763042684F878
:20881000406098F8B72084F85E3009F1490084F85F200B220EF068FB607E00284ED1687866
:2088300000284BD1287EA77E8DF800000FB1EA20607605F11701E72000F02CFD94F86000DA
:2088500028B1287E022808BF01208DF8000098F8B7009DF80010884203D0E820694600F0C2
:2088700019FDA77E1E4C601C007808B10EF022FDB8F88A0019490880C7B1032F12D0052F95
:2088900005D0012F03D0022F01D00EF013FD022060700BF03BFF4FF6FF70A8F88A00114981
:2088B000088005E00BF032FF032000E0012060702720287030460DF07DFE01E02A2028708B
:2088D00028460AF0A3FABDE8F883C046B830002020150020A8110020657301009019002085
:2088F00090310020721600202DE9FE4F544E0746301D00688047534C00258346A01C057053
:208910001FB10DF077F90AF045F994F83800B04610B1E06B00B1804709F014FEDFF87491AD
:2089300009F11C0090F900000EF002FC0DF0FCFA0EF0F4FB0EF078FA0EF06AFADFF808A15A
:2089500007270AF1240656F8040B00B180477F1EF9D13E480560456005614FF470018160ED
:20897000C1600AF1040007680FB10BF0EFFE38484E4600688AF80E508A3EC0B112E048469B
:208990000CF0EAFA029002A80BF0E0FE21E048460CF0E2FA019001A80BF0D8FE14E06846BE
:2089B0000BF0D4FE07F012FD00280090F7D129480078012803D028460146FFF793F82648CB
:2089D000264F057007F12409786A0028DFD109F10409B86A0028D2D17D62BD622048A06163
:2089F00087F82E501F4BE36187F82F501E4A22621E4961621E4B87F830501E4AA362204B68
:208A1000E2621D4963601F4A21631C4FA260204B65701D4967631D4FE16058462761D8F86C
:208A300008106361884706F18D01522000F032FC96F8A7000AF020FF2846BDE8FE8FC04672
:208A50008C140020EC13002014150020281A00202C2D0020E81A002003320020640E0020FA
:208A700003EB0000EF76010091610100218200002DD30000856501004573010025B600007D
:208A9000CBBF000091B100002533010069F500008D240100321200202DE9F041071CADF125
:208AB000200D00F0C480F86B002800F0C080B7F84020002A00F0BB80007817F130014FF036
:208AD000000603D097F83810052902D0002E00F0AE80594C401E2ED0801E18D0C01E40F0F5
:208AF000A680012A40F0A380524C0725E0788DF81C5000280CBF0121311C3046E17009F08D
:208B100055F9E07802228DF81D0028460EE0012A40F08D80B4F85400401CA4F854000220A7
:208B30000EF092F8042001228DF81C00394607AB02F0BAFB7BE0684631460C2208F015F929
:208B5000B7F840000B284CD1FD6B15F8010B84F820002B786878AD1C03EB002328460EF0E0
:208B700044FA8046281D0EF040FA0546387A2077022806D0396804F1140001607A68426041
:208B900001E03888A08203F00100190928BF40F00800590928BF40F010006084834218BFC4
:208BB0000226B8F57A7FADF8020008D32348404505D3C4F8248040460CF0B0FD00E00226F6
:208BD000606AB5F57A7F019007D342F21070A84203D3A5620EF03EFA00E00226A06A029058
:208BF00000E0012602258DF8016068468DF800500AF07AFD0DF10D009DF801108DF80C50CB
:208C10000EF094FCBDF802100EF090FC01990CF01AF802990CF017F839460D2203AB28464D
:208C300002F042FBB4F85A00401CA4F85A0008B0BDE8F081A410002090120020407E050076
:208C50002DE9F843634C5C4D5C4EDFF87881604F94F8E4100846401E0B2864D8DFE800F0E0
:208C70007E2C43062343062343067967042907D001220A2945F8212C14BF0220032004E059
:208C9000202045F8210C0120024684F8E200002045F8390C0827C5F8FF7FC5F8F37F45F8DB
:208CB000392CBDE8F883052914BF09200620002784F8E400376078E094F8E170383D0120E6
:208CD000002FC5F81B0004BF0620002102D00021F160032084F8E400032045F8010C3160AE
:208CF0003068800861D294F8E4103548012703290ED00068456800216022052300914046EB
:208D1000A84794F8E400062814BF0A200720CFE700684568002160220523022000904046C4
:208D3000A8470420C4E70EF0BBFDBDE8F8832648264F0026012506600E203D6004F036FE07
:208D500002200CF0A3FC84F8E45084F8E360BDE8F883002038600C25786024E04FF08059DA
:208D7000D9F8A0010168202088472C3D0F2045F8010C41F61D56C5F80360D9F8A401466829
:208D900000214FF4C0720723022540460095B047D9F8A401C66800214FF4C07207234046E0
:208DB000B0470120386084F8E45004F178000EF073FDBDE8F883C04639400C4038600C4099
:208DD000A401001000A00C402C500C4004800C4034600C40940F00202DE9F0430446666846
:208DF000A7680D46ADF1340D0EF092FD3178012903D10EF089FD0020A9E04FF0010886F8FB
:208E100000800EF081FD287870706878B07068687060A868B060E868F06028693061287D9F
:208E30003075687D7075A87DB075A869B061287F3077687F7077A87FB0774FF00009C6F8D7
:208E50002090C6F830904D4675627563B562B56386F82C50102386F83C3086F82D5086F8D3
:208E70003D50786805F02EF9204605F0AFFA204606F028FE70B937480068C168386888472B
:208E9000786804F093FD0EF043FD35700EF03CFD2C465BE001A82946302208230EF010FDF7
:208EB0000694387BCDF800902B4A0990B96801AB06F180000EF000FD01A829462822082326
:208ED0000EF0F6FC05942549386901AA2B46079006F19C000EF0E8FC01A829462422082339
:208EF0000EF0F6FC8DF81C80B07838B906F1D000294601AA0EF0E8FC19483061707838B9AA
:208F100006F1EC00294601AA0EF0DEFC1548F06001A82946242208230EF0BAFC0695ADF842
:208F300014501149079406F584700A2201AB0EF0ABFCB969FA6906F140000EF06FF90B4AE5
:208F500006F16C00042123460CF062FF20460DB0BDE8F083D0010010A9BB0000514E010093
:208F70007F76010077760100F5FE0000857301002DE9FE43604C614D0E46B00959D35D4882
:208F900000F1280980464DE00178D0290EDBD02909D181783970C17879700179B97085682A
:208FB0007D60C168B9600EF04BF947E004F10805286009F02BFF28460BF0C8FB3EE0884753
:208FD00098F83010491E88F83010A9688847009801788DF80410A0604778CFB1DC2F0DD0D9
:208FF000DD2F0BD0E42F09D0F32F07D0DE2F05D0DF2F03D0E82F18BFDB2F0BD104F08EF983
:209010009DF80400162805D168460BF09FFB01E009F0FCFE9DF80400162803D004F10800D5
:209030000BF094FB48460BF097FF002869680090C5D1F00BA846C00305D0314F07F0C6F9A1
:2090500000280090A0D1700905D32E208DF8040001A809F0DBFE700805D325208DF8040016
:2090700001A809F0D3FEB00805D326208DF8040001A809F0CBFEF00805D327208DF8040003
:2090900001A809F0C3FE300905D329208DF8040001A809F0BBFEF00908D300208DF80500A1
:2090B0002D278DF8047001A809F0B0FE300A08D300208DF8050030278DF8047001A809F052
:2090D000A5FE6068D8F8041080B18847616800270091D8F8081067608847009804F1080697
:2090F000306009F093FE30460BF030FB0020BDE8FE83C046640E0020141500208C140020C3
:209110003C1A00202DE9F04F0746880FADF1140DC0F0B280002009F04DFE5B4D4FF000089C
:209130001C35C5F80080564845F81C0C01200DF0F1F956480EF0A6F955482838BC6890F8A2
:20915000342040F60A06C34600F1280189468246A0F82A8090F835300E8002F0F002C0F852
:209170002CB003F0F00180F8342041F00101A4F802809AF8042080F83510012A01D17B7C9B
:20919000ABB1B8680088A6F10801814205D0218B4FF60F400840208304E0218A4FF60F4035
:2091B00008402082B86887F8118004F04BF8B868694604F089F968460EF09CF83346D91F58
:2091D0004A1C00E03446666836B13088834203D0814218BF8242F5D1C4F80490607B00F07B
:2091F000F00060730AF114000EF0A0FA80680088814220D082421ED03E8C0EB397F82C00DA
:2092100097F82D60C7F824B000F0F00087F82C0006F0F00040F0010087F82D0007F1200326
:20923000CAF82C3099F80D00A7F8228000F0F00089F80D0004E0D9460AF1400080E800030A
:2092500028680028FCD0C5F8008001200CF038FC012808D0607B00F0F00040F0010060732C
:2092700008480EF00FF9B9680A8A4FF6FF3010400882B86845F81C0C05B0BDE8F08FC04621
:2092900001010E04492B0100001004406D350000980A00202DE9F0475E4E80460F46B8F1C0
:2092B000450F07D106F13004342220460DF01CFEF466ACE00DF05AFA3A2808BFF42000F010
:2092D000A780554C04EB8004A07810B9E178002938D0E178814208BFFB2000F09980B8F128
:2092F000580F25D0B8F1600F1BD0B8F1E00F0FD0B8F1E80F05D03A78904220DC91421EDBC7
:2093100020E006F1B7003978007881421AD17EE097F900000AF0C0FB4FF6FF7181420ED0BF
:2093300010E038880A280ADBB0F5804F07DA09E038888F2803DB46F2B041814202DAE820F3
:20935000BDE8F087354D6868804721786278824606F164008146401839460DF0C5FDA968C4
:2093700050468847404650384FD0801E37D0401E48D08D3841D0401E28D0401E3AD0801FFD
:2093900045D16868804704460DF05AFDFCF770FC96F9A6000DF0CCFE0CF0C6FD0DF0BEFE9F
:2093B0000DF042FD0DF034FDA9682046884796F8A7000AF061FA09F129015220FFF76AFF6E
:2093D0000EF0CCF818BB09F0BDF820E096F8A7000AF052FA01281AD01A20BDE8F08796F8C8
:2093F0008D0018B902200BF05DFB10E002200DF0A9FF0CE00DF00CFD09E096F9A6000DF0C6
:2094100097FE04E00DF010FD01E00DF087FE0020BDE8F087A8110020308201008C140020CE
:209430002DE9F8435B4D804695F83800002798B12A6F8AB1D5F8900070B142F21A006946D9
:209450009047D5F89000804730B19DF8000018B1B8F1E10F08BF01274F4A02F1B70000787F
:209470000CF0B2FB407B02280CBF052601264D4C2068002800F08B80B8F1000F91466ED020
:20949000B8F11B0F02D1017D052968D1B8F1E90F25D027BBB8F1E10F16D10DF0E5FD90B119
:2094B0002068C18AC9080FD299F89810817699F886104A1C89F88620406881703046FEF72F
:2094D000FBFBBDE8F8832068B8F11C0F16D1216A002949D0884700202060BDE8F883F120B6
:2094F0000DF073FB2768B87E50B90DF0BDFD20B12068C18AC90801D2D6E7206847462FE043
:209510007868398907F0B0F878680088000905D395F8380010B10BF001FB2768F88AC0085B
:2095300011D3387E00F07F003876387D032803D1787E40F004007876F0200DF046FBE16801
:20955000206888470FE015490126B87E0E70401EB876F0200DF039FB11480078AFE7002721
:20957000477008F0B7FB2068C08A000A0AD395F8380018B999F8A7000AF07EF999F9A6004A
:209590000DF0D6FD0020206010200DF0E3FEBDE8F883C046EC130020A811002000320020CD
:2095B000CA180020640E00202DE9FE4F5E4C814604F1140A50460EF0B9F890468B460746E7
:2095D00008F0010000900EF0A3F98425BBF1FF3F019017D1A6692EB1A069C068814508BFA0
:2095F000A0690DD00EF094F9DAF800608AE0F168894540F086800EF087F9301C00F0878030
:20961000B0F924B058460CF0C9FA00287FD0A16981425CD0B84217D104F1B0000DF03AF83A
:2096300060690068606197F82700394640F0040087F827000AF10C000BF004FE5FEA980034
:2096500021D3676901221AE00FB905B31CE0396888423AD104F1B0000DF01CF83968086860
:20967000386091F8270040F0040081F827000AF10C000BF0E7FD5FEA980004D30022484670
:20969000394608F0FFFC002501980EF03DF9A179627A607941EA0203184310D1012939D0E8
:2096B000012A37D026691D480DF0ECFE022104F1D4000DF061FC30460DF0E4FE2AE004F1F3
:2096D000D40002210DF058FC24E03F68BCE7009F90F82720012505FA07F13E1C41EA0201D1
:2096F00080F8271014BF0E480E480CF069FB5FEA980004D3616948462A4608F0C3FC002570
:2097100005E03668002E7FF472AF0EF0FDF801980EF0FAF82846BDE8FE8FC0466D35000030
:209730000100020401000104700A00202DE9FE4F07461046002F00910CBF4FF0E80B4FF070
:20975000000B002900F0AB80BBF1000F40F0A98060B17868401E7860F82101707868401EA7
:209770007860002606703889801C3881009C4FF000094FF0020ADFF83081CDF80490083CFB
:2097900014F8080F00F00F010F2900F08580012820D004287AD1454D95F83800002875D015
:2097B000296D60688847061C26D03889B7F84C103018801C81421FDB78686D6D6168019BC8
:2097D0003A46801BA847B8B178683D89801B786076195AE00098019E042309EB0001C91CEC
:2097F00011F8010FFF2841D021283DD13889B7F84C200B30824202DA1A20BDE8FE8F7868AE
:20981000B8F8A020401E7860121202707868401E786098F8A02002707868401E7860019D70
:20983000057098F8A2007A68107098F89E2078681201401E786042F00F02027098F890C003
:2098500098F871207868401E786042EA0C1202707868401E7860212505707868F61DB6B2D9
:20987000401E7860052505705B1EB9D17868C6F30121401E786041F0880101707868401EA6
:209890007860067038893618B61C3E81BAF1010A09F108097FF474AF7868B86501E04FF056
:2098B000E80B5846BDE8FE8FA8110020EC1300202DE9F04F8A4609AF4FF08051ADF11C0D29
:2098D00090463D69059001F5D8700490D1F8B001D7F808B04169069327208847524C4FF05E
:2098F0000309143CC4F884970126C4F87C67C4F880970220C4F8FC06F868C4F8080430460E
:209910000DF0D8FED4F808040008F8D2D4F88C07800F28BFB14655D2681E41460C238DF806
:2099300000000DF1010011F8012B5B1E00F8012BF9D1022D19BF0020011C98F80C1000206C
:209950008DF80D108DF80E008DF80F000099C4F83C15019BC4F84035029AC4F84425039B5C
:20997000C4F848353968BAF1020F4FEAC542A1EB0A08A2F5002106D34FEA4A52A2F58002E4
:209990006FF315021143264A0A43C4F84C258246C4F85085BBF1000FC4F854A5214DC4F80D
:2099B00058B511D02E6078682060C4F808B030460DF080FED4F88C078008F8D3D4F88C0745
:2099D000000801D3CA4627E0C4F88497D4F88C0710F0030FFAD1D4F8800720F00200C4F850
:2099F00080073F7D47B1049F3868016A272088473868016927208847C4F87C670598C4F840
:209A1000806748B12E6006982060C4F80880C5F800642062C4F82880504607B0BDE8F08FEE
:209A3000C801042000004842184002402DE9F04F894609AF4FF08051ADF1240D92460590DD
:209A500038683D69079001F5D8700490D1F8B001D7F808B04169069327208847504C4FF012
:209A70000308143CC4F884870126C4F87C67C4F880870220C4F8FC06F868C4F808043046AD
:209A90000DF018FED4F808040008F8D2D4F88C07800F28BFB04653D2681E51460C238DF838
:209AB00000000DF1010011F8012B5B1E00F8012BF9D1022D19BF0020011C9AF80C100020E9
:209AD0008DF80D10019B8DF80E0000998DF80F00029AC4F83C15B9F1020FC4F84035039B45
:209AF000C4F844254FEAC542C4F84835A2F5002106D34FEA4952A2F580026FF3150211436D
:209B1000254A079D0A43C4F84C258146C4F85055BBF1000FC4F85495204DC4F858B511D009
:209B30002E6078682060C4F808B030460DF0C2FDD4F88C078008F8D3D4F88C07000801D394
:209B5000C14624E0C4F88487D4F88C0710F0030FFAD1D4F8800720F00200C4F880073F7D83
:209B700047B1049F3868016A2720884738680169272088470598C4F8806740B12E6006989C
:209B90002060C5F800642062079FA760A762484609B0BDE8F08FC046CC01042000004842F0
:209BB000184002402DE9FE4F524D286808B90DF081FB554C04F13800DFF83C91DFF840A105
:209BD000DFF8408107789FB94D46686880474B490F7847B95246A96817782FB98323424673
:209BF000137088476DE0A96802234246137075E0D4F8981009B104208847676D2A685FB189
:209C1000D06D20B102210023B8472A68676D106E10B108210023B8473C4E306A3C4F016CD5
:209C3000F86888474D46834668688047029033480578002D48D150460078002844D1D4F80B
:209C5000841000208847F42001A90AF0BFF89DF90400304D58451ADC6B79C3B9D9F808100F
:209C700002988847A878042801D00DF023FB042140466F790170D4F88410781C687109B1A8
:209C9000032088470320688100F006FD27E083214046346A0170636CF8686A4600219847A4
:209CB000B6F90400BDF90010884214BF0020012007F0FCF9D9F80810029888470835287822
:209CD00038700CF0F7FC0AE0022140460170D9F8081002988847D4F88410042088470E48DE
:209CF0000078012803D000200146FDF7FBFEBDE8FE8FC046640E00208C14002004320020AC
:209D10000632002008320020EC1300202816002088190020C8180020E81A00202DE9F843D0
:209D30004F4E84460120002430704E48504D04704D48DFF83881047005F14E00008804EACD
:209D50000307B146002F4FF0020606EA020608BF002E14D14FF0E04720461F401040002F00
:209D700008BF002803D11D2006F074FB54E0454695F90000401E28700DF092F84CE04246F0
:209D900092F900303C4E5B1E137043F20842824207D06F8E931C834203D0BA4218BFBB4244
:209DB00017D1304608300068826C60469047008843F6030181420BD0204601F0F7FF98F9E9
:209DD000000000283FD098F90000002838DD42E06F8EB5F86A1043F60400884205D0B84252
:209DF00003D0B5F84E20904203D12248007803281AD1B1F5505F05D0080B0BD31D2006F079
:209E100029FB07E01D480168304601F5C071016005F070F80DF020F898F9000098B198F97E
:209E3000000000280CDD16E0022811D0204601F0BDFF98F9000030B198F9000000280ADCDC
:209E50000DF038FA07E020460146FDF74BFE02E0204606F0FFFA89F80040BDE8F883C046D4
:209E7000E81A0020D01A0020CF1A0020D11A0020280D0020CA180020401600200C01002197
:209E90002DE9F041554C2079ADF1400D032818BF607140F09E8000256571A84601A824224D
:209EB0000823294684F804800DF012FD032001A98DF81C002A4601200DF0E2FC1D27A060CE
:209ED0002E46A5700AAB3846414604220CF063FE9DF82810E378A52907D19DF82900FE28FA
:209EF00003DC9DF82B20962A09D0242902D0B72918D11FE03E46EBB99DF8290019E0B5B1CE
:209F1000984203DAFE2B18BF01280BD1984203DD012B08BFFE2805D0284606F02BFE9DF8AB
:209F3000290004E0384606F025FEA57802E03D46A570E0707F1C1E2FC4DD8DB926B91D209B
:209F500009F084FD042015E0A67030464FF480510AF0E6F8E08041463046FDF715F80AE09E
:209F70001EB1304606F006FEA57828464FF480510AF0D6F8E0800AAF174D00970EA82968D0
:209F9000AE8801600EAB868093E8030042460C2306F02EFEE6880A2809D1384641460C2257
:209FB00006F0E3FE40F6EF70801BADF82E00BDF82C000EAF401CADF82C002968AE8839608C
:209FD0000EABBE8093E803000C220AAB06F032F9607910B0BDE8F0811E8B0100481A00201D
:209FF0002DE9F84F0F4605460CF0FBFB4FF6FF71814208BF682000F096804C4C410001EBD0
:20A01000C0002418D4F8026016B9D4F80630F3B1D4F80610B14208BF692000F084806078A0
:20A03000401E0FD0401E07D0801E10D13868864273D8814271D30AE0388886426DD88142EB
:20A050006BD304E03878864267D8814265D3384E7068804742F20208B346DFF8D8A00090E1
:20A07000A5EB0800012816D9113831D12078627856460021301806F078FE637838460DF09C
:20A090007FF8834298BF181C02D938460DF078F8024630461EE00BF097FF06463846314695
:20A0B00008F030FE361A5FFA86F9DBF80860B9F1000F30D0207862783946504405F0EAFAF0
:20A0D0001D484146A94218BF401C80F8009008E05046627821784018394605F0DBFADBF8F9
:20A0F000086008F11900A84204BF00208AF8870008F11A00A84213D19AF887009AF88610DE
:20A110004218322A01DC08430AD102208AF8860030278AF887700098B0476A20BDE8F88F37
:20A130000098B0470020BDE8F88FC046588001008C140020382F00204A2E00202DE9F0412F
:20A150000C4601467138022840F29680133824D04D4F4C387AD0401E61D0401E48D0401E2F
:20A1700036D0401E29D0401E1AD008460DF05FF806460B2E11D0424D6868804741498046AC
:20A19000B000425CBF1840184278394620460CF0ABFEA968404688470CE0F420BDE8F08172
:20A1B0002278022A68DA3949601C01EB820104220CF09AFE0020BDE8F081217832295BDA01
:20A1D000334FCA00201D02EB0112B9181822EFE72678022E50DA2C25601C05FB0671102297
:20A1F00039310CF081FE05FB0670C06C6061E1E72078022840DA2C2101FB0070667890F844
:20A210003800B04238DD23786278394602EB430201EB4201022201F5DE71A01CC8E720782E
:20A23000022829DA2C2101FB0070667890F83000B04221DD227860783223394603FB02005C
:20A2500000EB4000032209189031E6E72078022812DA2C2101FB0070667890F82800B04208
:20A270000ADD6278207839468018420002EBC00289180A227C31D0E7E820BDE8F081C04618
:20A290008C14002028790100A82100201C2800206C2300202DE9F0434D4CDFF8388194F852
:20A2B0003F600027ADF1140D002E57D198F86660002E53D0C768007A454600F00701C0F32D
:20A2D000021900E0BF1C0E46701EC1B24EB17A783878B5F88E6000EB0220B042F2D102271C
:20A2F00010E005F16406443600E008374846411E5FFA81F9A0B3304639460CF017FC002826
:20A31000F3D0032794F83F0040F0040084F83F0002A80BF0F5FD01200CF04CF904F1340163
:20A330008720FFF70BFF04F13C018520FFF706FF04F13D018620FFF701FF04F13E018820E9
:20A35000FFF7FCFE0120009004F134060196B5F88A30394602AA0520FDF7EAF9002F33D1C5
:20A3700098F871100F292FD0404690F890208A422AD090F88D0038BB1748007820BB1748E8
:20A390000078012803D001200021FDF7ABFB144C606880472146134C94F83B20022A11D1B3
:20A3B00094F83820FF2A0DD00F4A176857B9576A47B98968884704F1200009F085FA06F0B7
:20A3D000D7F901E08968884705B0BDE8F083C04640300020A811002022150020E81A002047
:20A3F0008C140020F0170020640E00202DE9F04F474C6068ADF1140D8047464A92461178AD
:20A41000DFF8148102919AF80020A168A146012A0CD001248AF80040884798F80000012815
:20A4300005D020460021FDF75DFB00E088473C4C3A4DDFF8F0B0E06805F1B001814206D1A6
:20A45000594691F90000002818BF00274AD1D9F80400804700270390374EA5F8B27006F1F1
:20A4700038000578002D07BF4FF48600391C2E482021226A95688DE8030031492B4A2C4BE8
:20A4900010683A46A847D9F808506080002827D45946767891F90000264B294A401C0870CA
:20A4B00093F90000E260401C187006B18027234EA08FB6F88E304FF67F7101400F4338432D
:20A4D000A087B6F88A00082204F13F0706F1A801A4F84A003846A4F848300CF005FD01276A
:20A4F0000398A847D9F804008047D9F8081017B9029A8AF80020884798F80000012803D0D4
:20A5100000200146FDF7EEFA384605B0BDE8F08F8C140020CE1A0020E81A0020280D002052
:20A5300028160020D21A002000004F8C94190020F1140000D11A0020EC130020A8110020F1
:20A55000D80D00202DE9F84F994692468B4606460DF0DEF94D4C0090B4F92610B4F9240004
:20A570000AAF401A40F6F871014008297ADAB4F92400401C6FF31F30A084B4F924800BF005
:20A59000DBFD054606F170000CF084F8C5F808B085F826A0C5F80490A5F824803C48EE608D
:20A5B00097E80C00202100271940104005F1100383E8030004F1140085F827700368002BC5
:20A5D00043D129460AF03EFE002844D0A6F8B88095F8270040F0800085F8270086F8BA70F0
:20A5F000E07920B1207810B1E7710120207200980DF08AF9A069002844D12078F0B9607945
:20A6100001283FD00DF084F90646A07988B9A86807F09EFE40B930460DF076F904F1D4008B
:20A6300004210CF0A9FC2DE004F1B0000DF034F902E0184901200870304621E001200CF0F8
:20A6500087F919200CF08EFE1CE004F1140029460AF0F8FD48B9B4F9240000F6FF706FF3AD
:20A670001F30A0846FF0010809E0A6F8B88095F8270040F0800085F8270086F8BA700098E8
:20A690000DF042F94046BDE8F88FC046700A0020F1EFFF9FFF3100202DE9FC414648474CDE
:20A6B000474F48490378A57862893878042D6DD101F13C063578884605F0F005357000265D
:20A6D0008E63414908335A43424391F838500092002D50D00D46AA6F002A4CD0EB6F002B6B
:20A6F00049D004F10801684690478446374BE178DFF8E8E020791A68BCF1650F31D0BCF180
:20A71000000F28D1107D052811D13148017871B9186890F82C00042809D119686D6D906DD7
:20A73000096B3346A847002808BF1A2016D0294D6868804728490E68002E08BFA96807D04D
:20A75000A96804F10C02964213D03668002EFAD1884738780FE0704606706046FEF760FEF0
:20A7700022E082F8690082F86A107046E96F06701C20884718E01A49009E04F10C0761619E
:20A79000B6FBF0F138460CF08BF90DE091F83C40083380005A43884604F0F004504388639B
:20A7B00044F0030481F83C4098F8740000F0F00088F87400BDE8FC8189190020C81800209D
:20A7D000CC190020280D0020EC130020640E0020351200208C140020281A0020083200207B
:20A7F000B59B00002DE9F04706464FF00108ADF1600D0922B07D8DF84C8006F117018DF8D0
:20A810004D000DF14E000CF06FFB464D68688047814616A98120FFF791FC707D002854D01C
:20A830009DF85800022817DA042000238DF80300347D8DF802809DF858708DF801306946B7
:20A850008DF80040781C8DF85800D220FDF75EF8812016A9FDF75AF800274FF0FF0A3C46DF
:20A87000307D8DF8217008A980F001008DF82000D120FFF763FCC0B99DF82200FF2814D0BD
:20A890008DF800006946D420FFF758FC20B1A96848468847192042E0307D69460DEB8000C8
:20A8B0000461D420FDF732F801E08DF822A08DF82440307D8DF8234008A98DF82000D12024
:20A8D000FDF724F87F1C322FCADB307D00279DF84D208DF840000DF14E018DF841700DF19B
:20A8F00042000CF001FB8DF84B80D02010A9FDF70DF8071C0FD1307D314610228DF8280016
:20A910000DF129000CF0F0FA30690AA90F90D320FCF7FCFF0746A96848468847F8B218B021
:20A93000BDE8F0878C1400202DE9FF410546080BC0F08680484E4449002401272246347046
:20A9500006F1580077720CF0DCFE40480CF09AFDF06841688868B04608B9C86828B13F4886
:20A970003F491C38C46150310160384608F022FA374E3460374846F81C0CA9684C80AA6865
:20A99000128840F60200904205D00B8B4FF60F421A400A8304E00B8A4FF60F421A400A8226
:20A9B00000F1080C6F74ACF10702531C00E039464F6837B13888844503D0824218BF8342D0
:20A9D000F5D127464F60487B00F0F00040F00100487308F114000CF0A9FE80680088824212
:20A9F0001BD0834219D0288CC8B195F82C006C8495F82D306F6200F0F00085F82C0003F0A1
:20AA1000F00040F0010085F82D0005F120024A60487B00F0F000487301E0C8F84840A86802
:20AA3000694602F051FD68460CF064FCA86802F009FC30680028FCD03460A86846F81C0C70
:20AA50000090BDE8FF81C046096A01006D3500001C10044001010E04700A00201C10044087
:20AA7000010007062DE9F84300204A4C8DF800000CF0D3FDE278484E414DDFF80C9101214C
:20AA900091404FF6FF725218024096F83800628120B3326F12B342F21A006946904737483E
:20AAB00027790378A3B19FB99DF8003083B1D6F8940068B180474946491C2A78097830B18C
:20AAD000678908314A43B0FBF2F0C019608127799DF80010608907FB01006081A078002817
:20AAF00047D1284F386AC06B80474E4680466489297870783B6A08304443D86B8F00804756
:20AB10006968224D2A787578214E3C23401AB0FBF7F103FA02F0B1FBF0F205F10803424398
:20AB3000891AB1FBF3F25A43891A05F10803691A641896F8581096F83C5098B2083401F00A
:20AB5000F00107FB048341F0020107FB0032736596F8744086F8581005F0F000B26340F0D9
:20AB7000020086F83C0004F0F00086F87400BDE8F883FFF791FDBDE8F883C0460032002017
:20AB9000CC190020281600208819002038120020280D0020C8180020EC1300202DE9F0435A
:20ABB0004A4D95F8E700ADF12C0D00287AD13F4F387B01240021242285F8E7407E6885F85C
:20ABD000E6000823C5F80C6101A80CF061FE002605F10C00069601ABADF814603449079683
:20ABF00032460CF051FE334905F1300001AB32460CF04AFE304905F1540001AB32460CF095
:20AC100043FEB96820468847DFF8BC802B4808F104037A7B00781868C0F3815922B1B9F110
:20AC3000030F04D185F8E140B9F1030F1ED0B9F1020F1BD0B9F1010F2DD14FF08059D9F88E
:20AC5000A4011F4F456831464FF040521C23032000903846A847D9F8A40131464FF40072DB
:20AC70000923456800943846A84714E002200AF025FDB9F1030F0CBF4FF47A7142F210714E
:20AC9000104800685435B1FBF0F128460CF0F4FD28460CF001FE40460068C00802D230460A
:20ACB0000AF00CFD0BB00020BDE8F0838C8A0100B3BC000089080100CD0201000132002053
:20ACD00000A00C40388B0100B03F0050940F00202DE9F84F05464448DFF8109183462E18F7
:20ACF000093699F8380034788846B0B1D9F8501099B10BEB8507786B00F0FF0088478246FB
:20AD1000D9F85010786B00F47F008847504480B218B131784018001DC4B238481230007870
:20AD300001280CD198F808704FB1314898F80930C1190E79C05C0019401DC4B200E0002644
:20AD50000D2D09D106EB0408B8F1F80FD8BF294F1CDD0CF0AFFA05E030198046801C0BF0EA
:20AD70007BFA074697B902200BF076FA011C0AD00BEB050090F825001A2708701E4E4F70A1
:20AD9000307807F065FD0020BDE8F88F08F10202384600210CF0DAFC07F10C00002174222D
:20ADB0000CF0D4FC07F13C00FF2110220CF0CEFC07F12C000F2110220CF0C8FCE019786054
:20ADD000022D3E810BDB0B2D09DA7868401E78606D1E05703889641EE4B2401C3881A7F8D1
:20ADF0004C403846BDE8F88FD8860100EC130020AC8A0100980E00201415002032120020E5
:20AE100046492DE9F0410A680646ADF1280D08A8026049684160424C94F8B30006F1280566
:20AE3000002877D07078002874D1706E002871D0012102AA05F0A0F800286BD19DF808009B
:20AE5000B073F06C38B1294605AA0DF11603F7F743FF00285ED10DF116000090706E2946CD
:20AE700005AB01F073FE002854D12E48007801284DD04FF4005006A908F09CFD06A808A9FD
:20AE900008220BF0FBF930B106A8294608220BF0F5F900283BD194F85900002837D0A66C1E
:20AEB000B4F8445042F2010004A908F083FD049A4FF000410020E2FB0610061C206D0CF00C
:20AED0009BF987190498B84202D86D1C3F1AADB2154E706880475FFA80F8206CB84204D14F
:20AEF000208FA84208BF002708D027642587002084F835000BF0CEFA0127E064B16840460D
:20AF100088470FB106F0FEF9012084F85800002084F859000AB0BDE8F081C046D88A010082
:20AF3000F02D0020ED1300208C1400202DE9F84F064630798028D4BF0020E820717900271E
:20AF5000092901DB0A2900DDE820B179002975D0042973DA002871D1DFF8F48098F87100F3
:20AF70000F286BD0B8F88A104FF6FF70884265D0B8F88410884261D0F079314C01280BD029
:20AF900040B1FF285AD194F83B00002856D101252F4602E0012500E00225DFF8A8A00AF184
:20AFB0002000834608F090FC0AF1100008F08CFC04F1200008F088FCDFF8989009F10400FB
:20AFD00000688047204B84F83B500246FF21002060631D6884F83810002D0CBF0121011CF5
:20AFF000012F84F83D10554684F83C7008BF032085F840004846816810468847B11DE8206C
:20B01000FEF748F9711DE720FEF744F9311DE120FEF740F994F83D00012802D120200CF0A5
:20B0300091F90A4898F871104FF47077A86207FA01F000F2636158460BF032FDBDE8F88F43
:20B05000F017002024310020640E002065210100A81100208C1400202DE9FE4F0BF00AFA30
:20B07000434C04F1080202901168E0604FF40050491C1160694608F09DFCDFF8FCA0DFF8F4
:20B09000FC9094F82F0000285FD0666B94F82D0000254FF0FF0BA0462F4654E0B07F8008C4
:20B0B00021D3F07F08F04AFE0146082268460BF0E5F8C0B1716802980CF02EFB2D498142A4
:20B0D00011D8F07FB7770AF009FA86F81FB0DAF80000804794F82E3013B15B1E84F82E30F6
:20B0F000D9F80810884798F82C006D1C2036ADB236E0F078800822D3307908F01FFE01468E
:20B11000082268460BF0BAF8C8B13088010402980CF002FB1749814211D83079F7700AF0BB
:20B13000DDF986F804B0DAF80000804794F82F3013B15B1E84F82F30D9F80810884798F813
:20B150002D006D1CADB2A842D3DC94F82E0048B1A046266B98F82C0000254FF0FF0B2F4668
:20B17000A8429BDC04F1100007F0AEFFBDE8FE8FAC2E002000A493D6901400208C140020F8
:20B190002DE9F04105466C78ADF1180D002C7CD14248B5F896100088884218BFE82405F1E5
:20B1B0008C0101A80F460BF003FD01A80AF094FE3B4B40B995F8990040B1A3F138000078EA
:20B1D00020B9E82461E0002085F89900002C5CD195F8990000280CBF0120052004262E757E
:20B1F0003946E8820DF10E000BF0E2FC686895F89840401E6860411E6960B5F896800470B7
:20B210002F7D69680024481C2862781E087028892C651A78AC65801C288142B305F16C0000
:20B2300005F18C010CF06AFA1E4F85F86B60386810F47F0F0CD085F82C60386805F12C018C
:20B25000012200F47F0028632846FEF76FFA386810F0FF0F0BD02A2085F83C00386805F1CF
:20B270003C0100F0FF002864284602F001FE0094284603210DF10E024346F8F7F3FC041CEC
:20B2900002D1284602F080FF2CB16C701A202870284607F0BBFD06B0BDE8F0813212002014
:20B2B000241400201C8701002DE9F04F0C4692468046994600213822ADF13C0D684605F059
:20B2D00054FD20686D4628606068686020892881207A032804D0022003268DF80C0002E011
:20B2F00003268DF80C60374C207818B104F12C000BF0C0FFA08DADF80A0060781F28B4BFF7
:20B31000411C00210027B8F1050F617040F080000BD0B8F1040F05D0B8F1020F08BF40F01D
:20B33000600004E040F0200001E040F040008DF80D00ADF828A04FF0010BCDF824902249EA
:20B350008DF80EB00A680BA802604968416005238DF83560B8F1050F8DF83660B4F85000AB
:20B370008DF8343012D0B4F85600B8F1040F08D0B8F1020F0ED1B4F85C00401CA4F85C0067
:20B3900008E0401C80B2A4F8560003E0401C80B2A4F850000D4918206A4604F00FFDC0B228
:20B3B00058B1B8F1050F09D1606A0AF0B7F9B4F85000401CA4F8500000E05F4638460FB063
:20B3D000BDE8F08F901200205D86010051650000F8B5071C00F08880B86840F60301202675
:20B3F0004A1C02E04068761EF6B260B15EB10388994218BF9A42F5D1F9681CC820311CC19F
:20B4100049C881E849007868BA690025BD6138B397F8270042F00202002300F00700401EC4
:20B4300009D0401E04D0801E08D14FF0805304E04FF0804301E04FF000532A4697F82700E9
:20B45000000908D397F8270010F0070F03D04FF080702A4303437C68F868B7F92410A04768
:20B470000CF056FA214C0646B4F92600401C6FF31F30E08404F12000016881F827500BF00A
:20B49000A9FD30460CF040FAB4F92400B4F92610884229D1F86890F8BA0000280CBF052018
:20B4B000072005F05DF8F86890F8BA60BEB90668AEB1E2680E4912680968B2F1FF3F13D075
:20B4D000B6FBF1F2012A8CBFB6FBF1F1012170300CF0D2F9F86870300CF0DEF9F8BD80F836
:20B4F000BA50012008F060FEF8BDC046700A0020388B01002DE9F041414C074620680028D1
:20B510007BD0DFF80081002F18BFE92F17D10AF081FF4546297801EB81016918C1F8020022
:20B5300095F8B560287800EB800029184E702878401C2870C0B20A28A4BF00202870324D7D
:20B5500068681C2F32D0314E4FB1F079032806D1E12F04D0002088F8B200072000E0052072
:20B5700008F010FC2468F07903280ED06CB1002084F86900E18A2648C90938BF293800781C
:20B5900084F86A003846FDF74BFF98F85700012833D168688047044606F03CFCA96820465F
:20B5B0008847002088F85700BDE8F08180470646A96894F82F0002281ADA216804F1240000
:20B5D0000BF028F894F82F00A968401C84F82F00304688472068007D252819BF012088F85D
:20B5F0005600012088F8550000202060BDE8F08130468847F120FDF713FFBDE8F081C046C1
:20B61000640E0020F02D00208C140020781600205A1200204549B0B5044601F13800007872
:20B6300000287FD094F88B00002871D13520207504F18D01112204F16C000BF055FC04F1C0
:20B650003C00FF2110220CF081F804F12C000F2110220CF07BF894F88C0004F13C0500286F
:20B670003ED0401E29D0401E14D0401E58D12A20287002272764042305F8103C4FF4102211
:20B690002263032184F86B10204606F0BFFF071C3BD137E02A200A272870042327644FF492
:20B6B0004C1205F8103C02212263204684F86B1006F0ACFF071C28D124E02A200227287002
:20B6D000042327644FF4102205F8103C01212263204684F86B1006F099FF071C15D111E05E
:20B6F0002A2002272870042327644FF4502205F8103C00212263204684F86B1006F086FF01
:20B71000071C02D1204602F03FFD381C0BD1B0BD01280AD1886C8047002808BF002002D052
:20B73000192000E018200BF017FDB0BDEC1300202DE9F04F09AF9A4616468846ADF1440D07
:20B750003C893D88D7F8049010900020AC428DF83C0001DACA4501D30BF0ACFD002E6AD0B3
:20B770003748875D042EA4EB07044FF00000A4B2B8BF01205FEA000B0EBF2D1BA1440024EB
:20B79000314807A90823ED1B2530ADB210F801295B1E01F8012BF9D14FEA186001F8010B39
:20B7B0004FEA184301F8013B4FEA182201F8012B01F8018B0E70234E109A30689DF83C1081
:20B7D0004369706898478046B8F1FF3F24D00BA9049101208DF801009DF83C308DF80230AD
:20B7F00007AA01928DF800B08DF80370CDF80890CDF80CA0ADF816403168ADF81850022334
:20B8100070680A6A8DF814306946904780463068826970680FA99047B8F1000F18BFE4203A
:20B830000AD147B14C4438460BA911F8012B401E04F8012BF9D1002011B0BDE8F08FC046D3
:20B85000B08A0100EC3100203212002070B5ADF1380DFFF7A3F93A4908682822082340F0CA
:20B870000200086001A800210CF022F8354E3D4C3549B078002301AA079004F1D4000CF092
:20B8900013F800213022082301A80CF019F8307800251921ADF81C502C4A099001AB0095D1
:20B8B00004F158000CF008F82822082301A829460BF0FEFFF078264901AA2B46079004F527
:20B8D00084700BF0F1FF01A82946302208230BF0F7FF01207278ADF81C001A2101AB0992A5
:20B8F00004F174001B4A00950BF0E6FF1A492A4604F1B00013460BF0C7FF18480BF0C2FD49
:20B910002E46052384F8503004F1400181E860004FF6FF70A4F8AC00334684F8AF3023711C
:20B930006371A371E371237263720D4A13704FF4FA76C4F84461C4F848610EB070BDC0460D
:20B95000002009402A8B0100596F01006D610100310101007D3201008D57010099E40000DB
:20B97000FE310020700A00202DE9FC410746BE6833687D68986B20F4FA609863AC6B44B110
:20B990003168886B40F4FA6088634FF0FF30BDE8FC81AA6329630024EC776C630CE09DF892
:20B9B0000000296B08706B6B286BAA6B401C2863581C6863501EA863A86B90B93168886B66
:20B9D00040F4FA6088636A6B6878296B0128A1EB0201296303D1EB68384698476A6B14469E
:20B9F00046E005F14000694608F010FF0028D6D50BF08EFF204F8046387820B9022009F0F1
:20BA10005DFE0120387040460BF07EFF1B49086840F4007008603168886B40F4FA6088630F
:20BA30006878D8B9696805F1EC000BF059FF90B9AC630BF06DFF0646387818B1022009F0E0
:20BA500025FE3C7030460BF05FFF1027696B286BEF77401A2863686BBDE8FC8195F82D00A0
:20BA700030B1686B20B1AC6305F19C000BF000FF2046BDE8FC81C046FC310020301000403B
:20BA9000F8B50BF041F9434E414F0446A00822D3B96901B33D460020A8618A69086906F1CF
:20BAB00008032040104340F0020088610A6918689043186001F1100090E80C0030681A1C0B
:20BAD0009043306005F1200009F0BCFB022105F1D4000BF051FAB869A10815D200F1100246
:20BAF0000CCA002122400B40002B08BF002A0BD0016985690C40F8612C434FF48041846146
:20BB100007F1D4000BF038FAB86900283ED107F1140420460BF00AFE051C37D0F868E96872
:20BB300088422DD1A86806F013FC60B1012008F03BFB58BBF86870300AF0ACFD07F1B0005A
:20BB50000BF0AAFEF8BD06F1080128690A6810430860326805F1100393E80300081C104327
:20BB7000306000233361A86846F80C0C06F1100000680028FAD020460BF02CFABD61F8BD4D
:20BB900007F1D4004FF480610BF0F6F9F8BDC046700A00200C1004402DE9F8438146D9F81D
:20BBB00008703868066CD9F8045046646A6CAB6CA86B16F4F06F0146A2EB03082AD1F009E0
:20BBD00011D270095DD301B395F83C40641EA14298BF0C1C4846214609F0DAF9A86B001B39
:20BBF000A8630DD04DE081B1484609F0D1F995F82D10A86311B9002843D101E00020A863B6
:20BC100005F19C000BF034FE3BE04846414609F015FE36E0F20A19D24FF00008444602E069
:20BC3000A86B401EA86340B34846012109F0B0F93868446814F00F04C0F80480F0D0286B41
:20BC5000401E2863686B401E686316E0386844680022202904F00F044260CCBF20270F1C9C
:20BC70004846394609F094F9C7F12007B845C8BFB8464846414609F0E1FDEC77484606F0ED
:20BC900099F9B0090BD3A96A49B10F46484609F0B7F9A86218B94846391D07F03DFEBDE83C
:20BCB000F88370472DE9F04105463E4804780F46002DADF1280D42D03B48466A002F3ED0D7
:20BCD0008046D6B17069C0B10123ADF8223006208DF8200029460C2200236846ADF8243070
:20BCF00003F0D8FC03A839460E2203F0D3FC766908A803C81A226B46B047787B012668B9D8
:20BD1000002C14BF0FA013A06988102207F0F2FF397B13A00A2207F0EDFF08E0002C14BF4A
:20BD300012A017A00BF05EFA19A00BF05BFA88F802600020314606F039F888F803600AB0F1
:20BD5000BDE8F0815265737461727465643A20307800C046537461727465643A203078002E
:20BD70004368616E6E656C3A2000C0464465766963652052657374617274656400C046C0B6
:20BD9000446576696365205374617274656400C04672657175656E637920486F7070696E4C
:20BDB0006700C04690120020A41000202DE9F8433E4C8146A07830F0010708D0042806D0B4
:20BDD000032804D0052802D00BF074FAA078384E257904210528324FDFF8C880317005F127
:20BDF0000101CDB225711CD1022D53DC3F68B9F1010F4FD07868398904F036FC7868008821
:20BE1000000905D34146087810B108F087FE257928460BF0A3FC8320307009F06FFDBDE8F9
:20BE3000F883DFF8849099F88810A94232DB032830D007F07DFEA078042809D141463839B8
:20BE500091F8380020B1D1F8841009B102208847E07899F89510421C9142C4BF401CC1B227
:20BE7000E1703D682989686804F0FEFB68680088000904D34146087808B108F04FFEFEF71B
:20BE9000F1FDA078042808D08320307008F076F8BDE8F883E12004F0DDFABDE8F883C046CD
:20BEB000640E002024140020A8110020C8180020083200202DE9F0430746ADF11C0D0BF0FD
:20BED000D3FC09F06BFB4FF000090646CDF80C900BF062FB30F0010002D00398B04202D184
:20BEF0006FF0040066E078684C4658B1B0F1FF3F05D004A909F03AFB30B1804659E04FF060
:20BF1000FF3000E0204604900BF0AAFC049D4FF001082D1802E00A463BE0049370680499E0
:20BF30000BF0DEFC00282DD0684607F0F7F8D8B99DF8040005A909F0B5F888B9BB68BDF8CC
:20BF500014009DF80610029A984748B1BDF814009DF80650B881029BBD73C8463B6111E049
:20BF7000029903A809F06AFD0498641CB0F1FF3FD4D00028D2D00BF073FC2B1A02D0049885
:20BF90009842CAD2039F0AF0DFFD06F1080547B13A4652F80C1C0029BDD1296842F80C1C0B
:20BFB0002F600BF001F824B170680BF095FC641EFAD1404607B0BDE8F08370472DE9F04F07
:20BFD000044609AF3D4D78681E46ADF1140DEB880290B7F80090A08988469246411D89B216
:20BFF0000391C918B1F5805F63DCE288217A971001F03F018DF80010A1888DF801701B1834
:20C0100002F00302C1F3051747EA821709078DF80270C0F3831200F03F0742EA11628DF8D6
:20C0300003204046B9008DF804106A4699B28B4608F00EF8029820B3EF885EB13A46404632
:20C050005146334607F000FBF01906EB0A0387B21FFA83FA029B40464A46394605F0AEFA29
:20C07000A689E98809EB070087B2F01B09188AB23AB109EB0A00134681B23A46404607F002
:20C09000E3FA9DF800204046594622F040028DF800200BF037F9EA880BF10401404689B281
:20C0B0000BF00BFBFF2806D00398801880B2E88001E00520687105B0BDE8F08F481A00206B
:20C0D00070B53F4C0646A07EADF1200DF0B994F85C0082281AD0394B40F2016046F25C0596
:20C0F000ADF8080034491868ADF80A50426A086802A99047012814BF6FF07F009DF90C006D
:20C1100009F09BFF94F85C10226B505494F85C00822814BF401C002004F1180584F85C0088
:20C1300094F85C0005EBE00292F82C00411082F82C10400807D294F85C00401C84F85C003B
:20C15000C0B28128ECDB94F85C0081282CDA05F14401E120FDF79EF802204FF6FF738DF832
:20C170001800A17EADF8103031F0020018D0012919BF0720832108208021002249350092C0
:20C1900004AA0195FBF7D4FADB2807D0E52805D0F32803D0DF2818BFE8280AD1607603E05F
:20C1B000304604F047FF04E02A203070304606F02DFE08B070BDC046941900204816002024
:20C1D000B83000202DE9F84F0E463A494FF000088346642744468A464D6B91F82D0086F832
:20C1F0001E80D1460AE099F800106D1C2034ADB231E099F82D00641C6D1DA4B2A04217DDAE
:20C21000E8780028F5D0287907F098FD594608220AF034F80028ECD1E878B0772888000485
:20C230007060287986F80B80F077A87847463073DAF83040002F39D086F81E8042F21900DA
:20C25000694607F0B7FB0AF015F982461A480178642745468146A94228DDA07F0028C2D025
:20C27000E07F07F06BFD594608220AF007F80028B9D1E07A022803D0E07A58B1612710E04A
:20C29000616850460BF048FABDF800200B495143814201D9474604E0A07F6C2740F008003D
:20C2B000A07730462146202203F0F4F93846BDE8F88FC046AC2E0020D82E0020808D5B0020
:20C2D0002DE9F04707467D68D7F8089090460E460BF01EFB8246A86A002864D105F5847005
:20C2F0000AF0D8F90024EC772E6250466C620BF00BFB0BF00DFB2F4E3378824623B90220F6
:20C3100009F0DCF90120307050460BF0FDFA2A49086840F4807008603846414608F070FE1C
:20C33000A862C0B93846414607F0F6FAA878D0B9A96805F1D0000BF0D3FAE8B9AC62102057
:20C35000E8774946284604F065FF0BF0E1FA8246307840B323E0D9F80010886B40F02000B9
:20C370008863A87810B12046BDE8F087A96805F1D0000BF0B5FA10B1686ABDE8F0873846B1
:20C39000414607F0C9FA1020AC624946E877284604F040FF0BF0BCFA8246307818B1022073
:20C3B00009F074F9347050460BF0AEFA4FF0FF30BDE8F087FD310020301000402DE9F04389
:20C3D000DFF8E0808946054617464FF0FF31ADF13C0D40460BF084FA334C04EBC504666845
:20C3F00025680BF095FA2168096800290BD42968002905DCB9F1000F09D04FF0FF3108E090
:20C41000B9F1000F03D00BF07FFA002442E02968491C29600BF078FA286802283ADA1FB934
:20C430000DA80BF004F90DAF38686860B76800213022082301A80BF043FA4FF0000906949B
:20C4500001AB307B194A09903946CDF8009005F12C000BF031FA01A82422082349460BF0B9
:20C4700037FA012705F1640001AA8DF81C7049460BF02AFA05F1480001AA39460BF024FA0E
:20C49000706801F01FFE0A4A05F118002346042109F0BEFC40460BF01FFA20460FB0BDE89F
:20C4B000F083C046B4310020008B0100716001006F7601002DE9F04106AF3D793E68984674
:20C4D00004460B1CADF1180D074611D0012B15D130797379641C3870B17904F8013B337A0C
:20C4F00004F8011BB17A04F8013B7389181201E03178707804F8011B04F8010B8AB9002D89
:20C510000CBF42F20C0042F20D00694607F052FA9DF80000BDF8003004F8010B181204F825
:20C53000010BB8F1010F34D0B8F1020F39D1002D0CBF42F2020042F203000DF1020107F001
:20C5500039FA7589CDB1681E01468B100DF1020201EB5371C910CBB2811000EB517121F05D
:20C570000701401AC0B20121401C01FA00F0D15CFF3080F0FF000843D054E81D0DF102012E
:20C59000C210204603F086F87089C01D04EBE00407E0002D14BF02210121204602F0ACFB0E
:20C5B0000419E41B06B0A0B2BDE8F0812DE9F04390460A68D8F800401678814600271D46B1
:20C5D0003846ADF1140D531C242E0B6053D112F8016F5B1C4C2E0B600ED1AA68E41C24F0E3
:20C5F0000304241D54F8040C494606F05DFB2968EF600127091A2960462E1AD1E41C24F083
:20C610000304241D54F8040CE41C029024F00304241D54F8040C002749460390AA68ADF81C
:20C63000047001A803F084F82968EF600127091A2960532E1FD1E41C24F00304241D54F891
:20C65000040CE861C8F80040288B0090A968EA69D9F800004346F7F757FED9F800400027F5
:20C6700014B10119C9F80010D8F800402968EF60091A01272960662E0AD12B8B23B9E41D34
:20C6900024F00704083403E0E41C24F00304241D1FB9E9690E700127EF60C8F8004005B01C
:20C6B000BDE8F0832C4870B50568B5F1FF3F08BF00250AF0CFF801284DD107F047FF1428FB
:20C6D00049DB26482649002601230660254A0B60254C136020680028FCD1264A131D234952
:20C6F000186820F00300014321480068C0080CD2106810F0030F0AD041F003001860106854
:20C7100000F003000328FAD101E041F001011A481960006820B1194800682846F5F726FEB1
:20C73000174818490660184D0A686FF35B4245EA0200086015490868C0F30130012806D1A2
:20C750000A681348104040F400320A60086020680028FCD170BDFEE71C130050840460423C
:20C770005C600C40082204430C00684204000020B03F005000400340800128430001204344
:20C790008C210840482003400000390104000940FFFFFCFC2DE9F041374D044668781F4612
:20C7B00016468846ADF1380D012803D0FFF74EF801206870B8F1000F0AD0C4F804803EB16A
:20C7D000A6600BF0A5F8A978022903DB0BF09CF800204DE005EB8102491CC2F83C41C9B21B
:20C7F000A9700BF091F801251FB909A80AF05AFC09AF386820607868E060387C2074B8682D
:20C8100065746061788A6082F86800B1A0610021A02204F1200004F0A8FA684600212422D5
:20C8300008230BF055F88DF8185004F1380000216A460BF049F868460021242208230BF013
:20C8500027F80E49069404F1700000226B460BF01BF868460021242208230BF019F80849D5
:20C87000069404F1940000226B460BF00DF820460EB0BDE8F081C046700A0020ED69010081
:20C89000E37601002DE9F04F09AF3C897D6816464FF0000A0246002EADF1440DA0461093E4
:20C8B0003C888DF83CA05CD0304810F80690042E03DAA8EB0900C8462D18F868A4EB080408
:20C8D00007AB0827A4B2C01D10F801C97F1E03F801CBF9D1080E264F03F8010B080C03F893
:20C8F000010B080A03F8010B386803F8011B9DF83C101E704369786898478346BBF1FF3FBF
:20C910002AD0042E04DA03208DF80000022002E002208DF800008DF8140002959DF83C6049
:20C930008DF8026001218DF8011038688DF8039007ABADF816800BADADF81840026A0193EE
:20C95000109E0495694678680396904783463868826978680FA99047BBF1000F18BFE42028
:20C9700000D1504611B0BDE8F08FC046B08A0100EC3100203A4834492DE9F0470125002447
:20C990000570DFF8C880DFF8CC900C70304901F16A06378882460220104004EA0306002E4B
:20C9B00008BF002810D14FF0E04720461F401040002F08BF002832D0424692F90000401E8B
:20C9D00010700AF06DFA2AE0424692F90000401E1070BFB94A8E43F20843204646469342D4
:20C9F00004D191F84010090938BF281CFFF7DEF94846047096F90000F0B196F90000002876
:20CA100017DD1DE0B7F5505F07D114481249006800F5C070086002F06DFA0AF01DFA48463E
:20CA30004246047092F9000030B192F90000002806DC0AF03FFC03E020460146FBF752F8E8
:20CA50008AF80040BDE8F087D01A0020D11A0020280D0020CF1A0020401600200C010021D1
:20CA7000E81A00202DE9F84F07463248DFF8C89000EB4706183699F83800348890468B467F
:20CA9000B8B1D9F85010A1B12C4D05EB8705686B00F0FF0088478246D9F85010686B00F454
:20CAB0007F008847504480B218B131884018001D84B225481230007801280CD198F8086000
:20CAD0004EB11F4898F8093081190D79C05C2418641DA4B200E00025281980B209F0BCFBA0
:20CAF0000646184890F80090D6B13046002122460AF02CFE4FF00008A41937700D4986F839
:20CB1000018006F180007460CA5D358159460AF0EBF94846314605F09BFE4046BDE8F88F9A
:20CB30008DF8007068461A2103F092F91A20BDE8F88FC04618830100EC130020D886010003
:20CB5000AC8A010014150020321200202DE9F04F364E0025ADF1340D07464FF0010AA8467F
:20CB7000A9460C93DDF858B00B914AE017F8020FAD1CADB2401E1BD0401E09D0401E04D07A
:20CB9000401E36D1022C34D138E0032C31D135E0072C2ED1B9787878FB1C40EA0120A6F83C
:20CBB0004400186806F14802106086F859A025E0052C1ED1CDF80890B91C0A8802A8028064
:20CBD000897881700B9803A9FFF7FCFA9DF82A00A0B1029B40F0020000F0F7008DF82A00A3
:20CBF00006F1500203931068049003A805F01AFB04E008EB0400801C1FFA80F8E719641900
:20CC1000A5B23846694608F0EDFB041CAED1022D03DC4D466720A84600E048460C990D804B
:20CC30000DB0ABF80080BDE8F08FC046F02D00207CB5354C054694F871000F285ED03348C3
:20CC5000697E0078890959D2297E002841F00201297639D069684A1C1078801010F0030F9C
:20CC700032D000F0030002280ED1B4F884304FF6FE70984208DD56791179002001EB062148
:20CC9000994208BF012004E004F17A00491D09F04DFFC8B9687E696840F0010068764A78BA
:20CCB000C2F38102022A2DD1491D4A7809784FF6FF7601EB02218E4224D1297E00F0EF0045
:20CCD00041F0200129761CE0687E114E40F0030068763078B0B994F8A7008DF80000FF2316
:20CCF0008DF8033094F8B6608DF8016094F8B7508DF8025068460AF0A2FC7CBD687E40F0E5
:20CD1000010068767CBDC046A8110020EC1300202B1800202DE9F04F9246ADF11C0D0493FF
:20CD3000071C039114BF5FEA0100EB205FD000200446CAF80000A146CDF8149078783D78B4
:20CD500045EA00255FEAE5380CBFC5F30626C5F3C3260498BF1C20B1B8F1000F39D00F2E73
:20CD700044D0082004232349ADF800000C22ADF8023001F124000168019268468847002873
:20CD90000CBF02980598834608B305990C2203F0ECFFDAF8003003B95446C4F800B05C46ED
:20CDB00084F8048066712679002E0CBF05F0FF05C5F30A05E580A760039EE08809EB0001CA
:20CDD000C719891C1FFA81F94E45B7DC0EE01A2000E018200590DAF8000038B1046809F010
:20CDF000E9FA201CFAD10020CAF80000059807B0BDE8F08F8C14002070B50546344C28788F
:20CE1000ADF1200D00284FD1208F04F148066B88ADF800003146ADF81030E2200AF022FAF1
:20CE30000DF1120031460AF0F3FB6988532009F0F3FE208F04F13E063146ADF80E004A20A9
:20CE50000AF010FA01A831460AF0E2FB00268DF80D60A08FADF8020094F83A308DF80C3022
:20CE7000304608F073FC5220314609F0C9FE94F850000F281CBF01206070E06828B10268B2
:20CE90001AB10DF10E0069469047032008F090FA94F85200032818BF042813D104F1080093
:20CEB000102109F08DFD0DE0002060700AF086F941F2883008F04AFC0649B1F84E00401C8D
:20CED000A1F84E00216E09B12846884708B070BD48130020901200202DE9F0470D460646C7
:20CEF0005FFA85FA280824BF2E4845402E494FEA8A03C85885EA00023240C2F300672B4A6B
:20CF100006EA0504B043224006F4E0240243B4F5E02F01D1500E14D306F4E020074310D07D
:20CF300002F4E027B7F5A02707D0B7F5803704BF22F4003242F4A02203E022F4803242F453
:20CF5000C022DFF86C80CA5008F1D00739680122002002FA0AF40C4218BF101C5FEA0009B1
:20CF700006D1F00D04D34146C5F3805001F80A00300E0BD30AF0CCFC290E34BF0021211C7E
:20CF90003A68A243114339600AF0BEFCB9F1000F06D0F00D04D34046C5F3805100F80A10D5
:20CFB000BDE8F087006000A000100840007F077F002002402DE9F04117460D460AF0A8FCF1
:20CFD000324C8046207800266DB16D1E04D06D1E55D0681E11D00EE0B4F8AC004FF6FF71B0
:20CFF000814202D005E0A06908B9802648E0A069808C388044E0842642E0386831465022C9
:20D01000054603F0B2FE022704F59E7C04F5A672A5F110015CF8040B41F8100F137A0B7358
:20D030005068486052F80C3B7F1E18448860F1D1A069002808BF02200ED0A069C068A76913
:20D05000286297F82600A36985F82C00D869A2696862106AA862032067698FB105280FDAE9
:20D07000FA6801016A5097F826204C192273FA6962603A6AA2603F68401C40B2EDE7387077
:20D0900040460AF041FC3046BDE8F081700A00202DE9BE410546DFF8CC802978B8F8600069
:20D0B000E1292FD0B8F86200E92926D0B8F86400D9B92D4C2869676A02903FB37F692FB36E
:20D0D000A16A1931814221D806208DF800000422ADF802200023ADF804309DE8030002AB66
:20D0F000B84708B90298A06210E0401C80B2A8F8640019A00AF0E4FA08E0401C80B2A8F89B
:20D11000620003E0401C80B2A8F86000687830F07F071ED000F06001402906D12F7827B9A0
:20D13000B8F85210491CA8F8521000F06001202906D1287820B9B8F85800401CA8F8580020
:20D15000602906D1287820B9B8F85E00401CA8F85E00BDE8BE81C04664617461436E663AA9
:20D170002000C04690120020A41000202DE9FC47314CA11C0888401C088009F07BF9002649
:20D19000B046354681462846694604F0F5F88246BAF1FF0F4CD09DF80030206B23B900EB95
:20D1B0004A104068010402E000EB4A10416848460AF0B2FA864203D29DF800700646D04650
:20D1D0006D1C0A2DDFDB1E4D281D0068804794F82F106FB9626B08EB88030026FF27491EF5
:20D1F000D218D67013791771C9B284F82F100CE0216B0022FF2701EB48118A77CB7FCF770F
:20D2100094F82E10491E84F82E100C4A643BD9B2136804EBC10138310B6052684A6094F8A3
:20D230008810491E84F88810A9688847BDE8FC870AF070FABDE8FC87AC2E0020E88A0100CA
:20D250008C140020E0B501880025A1F6020159B143F20402891A04D0491E57D190F82460CA
:20D2700000E00226C76901E0C67B4769002F4DD03F1F052044F2380357F8041F0A04120CB6
:20D29000934203D0401EF7D13F1D01E0C1F30345002D3BD01F4B3046401F18D01C4A401E54
:20D2B00010D0001F0CD0801E0DD0C01E06D00F3819BF1A1C6032184A443204E0121D02E0A0
:20D2D000121F00E0083A1068C0F3834003E01A461068C0F303200F2806D0A84216D921F471
:20D2F000702141EA004110E0761F0AD0761F08D0761F06D00F3E1CBF21F4702141F4802146
:20D3100003D121F4002141F4E0213960E0BDC0460011005020130050C4100050F0B5064688
:20D3300000210B22ADF1240D0DF119000AF00EFA2E4F2F4C3078C01E14D0801E04D0143887
:20D3500010D0801F01282DD801208DF8180006F18B0103A80AF0D2F9032538788DF814509E
:20D3700068B112E000208DF8180006F18B0103A80AF0C4F9032538788DF8145028B9B4F8A2
:20D390008E000225ADF8020005E00DF1020004F1A8010AF0B3F98DF80A50B4F88A00ADF83E
:20D3B000160017E002208DF8180006F1320103A809F0FAFE0DF1020006F1280109F0F4FEC0
:20D3D0008A34208806F11C01ADF816000DF119000AF091F90B208DF8000077788DF80170D8
:20D3F000684600F045F909B0F0BDC04624140020A81100202DE9F84F8A463149044601F1C1
:20D41000B400007828B920465146F8F743F8BDE8F88F0A25884642F2107B20465146F8F7F4
:20D4300039F898F8B410002848D19AF80060D4F80090002937D023480168C88AC20832D2A4
:20D4500080094FF0000702D3087D15282BD008F0F1FF98F800308446002B0EBF09235B1E4C
:20D47000DBB20A2003EB830208EB0201491C0A78964207D0002B0EBF09235B1EDBB2401E5E
:20D49000F0D110E0D1F8011060460AF045F9642101FB09018B4505D942F242706426401A10
:20D4B000B0FBF6F717B90020BDE8F88F20686D1E07442760B1D10AF02DF96120BDE8F88F74
:20D4D000F02D0020640E002080B50288A2F602073FB143F20502BF1A14BF002090F8240069
:20D4F00000E0C07B2C4AD2F88832401F0B6048D0401E3CD0001F30D0801E24D0C01E18D044
:20D510000F380CD0D2F890024860D2F894028860D2F8BC0220F0784040F080503AE0506969
:20D530004860D06A8860506C20F0784040F0704030E010694860906A8860106C20F0784056
:20D5500040F0F04026E0D0684860506A8860D06B20F0784040F0C0401CE090684860106A8A
:20D570008860906B20F0784040F0A04012E050684860D0698860506B20F0784040F040502A
:20D5900008E01068486090698860106B20F0784040F02050C86080BDC41000502DE9FC41D3
:20D5B000274A28491778002F41D02C48077837F07F073CD1244C488C94F87470234E284B65
:20D5D000401C0025488407F0F00084F87400012030701978256704F16807012902D029466A
:20D5F000FAF780FA0AF084F81E4E301D006880472A4680461C4DA4F86A20286A144B8468B0
:20D610001A4802218DE806000C3000683946A04710490028088005D40F4991F90000EF60DD
:20D63000401C0870B16840468847BDE8FC81888C401C88840020107009F008FABDE8FC813D
:20D6500006320020C8180020280D0020CF1A00200D09010098180020D11A002008320020B8
:20D67000E81A00208C140020281600208819002070B50646304930780D5C401F1CD0083813
:20D6900051D0401F4FD0284608F0E6FD041C0DD130780C2808D1706830B1301D07F056F894
:20D6B000284608F0D9FD0446002C43D02A462046314609F019FC37E0B07810BB327A307CD8
:20D6D00051005410401901F00E01091804F0380040182430C0B208F0BFFD041C2AD031467C
:20D6F000182209F001FC04F1180060607168242209F0FAFB6068243060617169327C0E4657
:20D71000D6E7012816D12435E8B208F0A5FD041C10D03146182209F0E7FB04F11800606046
:20D7300071682422EBE7344624B104480078214605F08EF870BDC046648A01003C1A00205B
:20D75000F8B509F0C9FE04F099FB09F0DDFE044604F00C000C284BD0E0081ED208F08CFA01
:20D77000264E376805460120014608F0F0FF31686943884211D2224C8220B0FBF7F0291A15
:20D7900020460AF079F820460AF086F80120F8F799FB204608F07EFF2CE0200928D21948BB
:20D7B00009F047FE0428FAD0174A610905D220B11168104621F0010103E01046016841F0FD
:20D7D00001010160983210684FF0805540F003001060D5F8B8018169202088470B4CD5F83A
:20D7F000B8712068B86B804701202060206801E009F08CFF09F076FEF8BDC046388B010004
:20D81000A00F0020004003408C2108402C2009402DE9FF412E482D4F00683E78C06B8047C4
:20D830007968401AB100B0FBF1F4B868FF680025A8464146BC4271EB080101DAB84206D825
:20D850002946424684428A413CDA074600E0294638463246F317001BA94109F069FB2727CE
:20D8700004464FF47A7200230D46ADF802700820ADF800002046F8F775FF019015480168A5
:20D8900068468847029843464FF0000100F6FC02A41A9D416042A94111DA0F480268294661
:20D8B0002046F8F75FFF0D4604464FF000016042A94104DA204606F029FE002000E00120BA
:20D8D000064908700090BDE8FF81C046CC19002048160020B014002084180020073200203A
:20D8F0002DE9F84F2E4C012683461D4690468946C4F87C670320C4F880670AAFC4F88407E4
:20D91000D4F88C0710F0030FFAD1387A58B14FF0805ADAF8B001016A27208847DAF8B00160
:20D930000169272088470220C4F8FC063868C4F80804304609F0BEFED4F808040008F8D23A
:20D95000D4F88C07800F28BF301C26D22868C4F83C056868C4F84005A868C4F84405E868DB
:20D970001049C4F848053879002814BF081D081CC4F84C05C4F850850020C4F85405C4F8B1
:20D99000580509490E60C4F800B0C4F80880C1F80064C4F82090C4F82880BDE8F88FC0468B
:20D9B0000440024028000020000048422DE9F843044609F0ADFF81462B48021992F8ED10E3
:20D9D000491ECFB2002F82F8ED7046D1294901EB84042578618835F07F07884618D1E90972
:20D9F0000FD24FF0805000F5DC76D0F8B8018169404688473068416B404688470228F9D193
:20DA10001EE000EB8800D0F800110020884717E04FF08056D6F8B801016A40468847D6F89C
:20DA3000B801816A40468847D6F8B801016B404688470E49012008600D4908688008FCD398
:20DA500005F03F003F2801D0FFF7B0FF607800F03F003F2801D0FFF7A9FF484609F054FFEE
:20DA70000020BDE8F883C046940F002028200860282008407C880100F8B5314D6868804786
:20DA900006462D4CA9682068002852D160698047676A40F01000002F4AD00022797E014089
:20DAB000884205D03A4657F80C7C002FF6D13FE004F12400394607F04FF8002F38D02760B7
:20DAD000787E30F07F0005D194F82F00401E84F82F0004E094F82E00401E84F82E00A96850
:20DAF0003046884723681889D98A08F032FCA0851248007808F068F8D98A090A0FD2407BBB
:20DB1000012803D0022816D1052005E0187E401080F0010000F00100FAF7CEF8F8BDD87ED4
:20DB300005F0AAFE206890F91C0009F001FBF8BDA96830468847F8BD640E00205F12002033
:20DB50008C140020F0B506460F4600251446ADF1240D8B200DF10E010095FCF7EFFA8A208E
:20DB700001A9FCF7EBFA707A00282ED1387AA0B9BDF80E104FF6FE70884205DCBDF80E10F3
:20DB9000884220D101A90DE020489DF80E700488BDF80E008DF812700CE0022807D003283A
:20DBB00011D1394604A809F0A9FD09240BE038888DF812008DF81040211200128DF811107A
:20DBD00005248DF81300284611E002280CBF05240924012818BF311C04D1892007A9FCF75C
:20DBF000ADFA07A9224604A809F07EF9B07A04EB0D01C8736A4604A8214603F047FB0028B8
:20DC100014BF281C009809B0F0BDC046321200202DE9F041294D012001462870F9F762FF67
:20DC300027496FF0010008702B480068C06B8047244C074621786068A2688B003E1AB6FB03
:20DC5000F3F05843361A88001F4902FB03F8B1FBF0F0904201D209F02DFBB91B1B486160B4
:20DC7000414400F03BF81A4CA06867682168404207F050FB002F08BFA16808D0A1687868A2
:20DC90008142DCBF401A78603F68002FF7D1E068884202D0A06005F071FF02F053FB0D4C64
:20DCB000606880470646FFF7B3FDA1683046884708F0E8FE00202870BDE8F081E81A0020B7
:20DCD000CC1A0020CC190020FFF6C2FF21DC0000281A00208C140020481600202DE9FE4F73
:20DCF000294D814668680091804729F00106274CDFF89CB0DFF89CA0274FDFF8A480274D01
:20DD1000019024F00104B44212D02BF00100B0421CD1514691F9000010F1020F18D02868CB
:20DD3000826B91F900103868904701280ED10FE0414691F9000010F1020F09D02868826B65
:20DD500091F9001038689047012801D009F0B2FA2868C56A1349009A38684B46A847051C0D
:20DD700001D509F0A7FAB44206D02BF00100B04204BF51460D7001E041460D7002490198A9
:20DD900089688847BDE8FE8F8C14002021DC000009F60000CD1A0020941900204816002073
:20DDB000CC1A0020280D00202DE9F04F0446B4F80AB0A08998460B46ADF1240DABEB000135
:20DDD0000690ABEB0000181885B228481FFA81FA81789146164642460027079101E0012720
:20DDF000521C3046411E8EB268B9002F08BF002039D0012F12D10798534499B24A464346A3
:20DE100003F0DCFB2DE02946481C85B2079809F054FC11784840E3D00842E0D01348069F6B
:20DE3000C188781D80B24018B0F5805F0DDD0294ADF80CA0ADF80E30ADF810900798CDF889
:20DE5000148002A9F9F7A0F80BE0CDF80090CDF80480079920465246FEF7B0F8584608F091
:20DE700047F90248407909B0BDE8F08F481A00202DE9F84F07460E1C14BF4FF000094FF0C2
:20DE9000E809002F4FD0B9F1000F4ED17868401E78603F210170BD6D002D0CBF8020002092
:20DEB0007968DFF890A00224083E491E7960DFF880B008703889A7F85440801C388116F8E8
:20DED000080FFF282CD02A2828D1706830B35546296D8847804678689BF80020A0EB080006
:20DEF0007860716829B96D6D3A460023A84748B10BE06D6D786871688DF800206B463A46C6
:20DF1000A84710B9EB20BDE8F88F3889B7F854504044388108EB0500A7F85400641ECED1A5
:20DF30007868386501E04FF0E8094846BDE8F88F90310020EC130020F0B52F4C0546A07E00
:20DF5000ADF13C0D022806D0012804D005281CBFE820607649D194F8600000284AD100217D
:20DF700009A81822617609F0F1FBCDF828D009A8294600F05BFC94F82E0094F85810814255
:20DF900020DD266B70B10746BDF80A007189884204D13046694607F059FE98B97F1E06F1C5
:20DFB0002406F1D194F82E00276B8100242201EB40117818694608F097FF94F82E00401C32
:20DFD00084F82E000D48007828B19DF8340010B994F8580028B909A8FFF74AFB94F85800BA
:20DFF00040B194F82E10884204D12A202870284604F00CFF0FB0F0BDB83000200E120020B4
:20E010002DE9B841804607F0DFFFC01DC51098F82300002849D198F87E4007F0D5FFA042A4
:20E0300043DD264A1368E010191891F86C1004F007042141CFB207E0401CC0B21918C40013
:20E0500091F86C7088F87E4047B9691E8142F3DC1068002188F87E10417029E098F97E1074
:20E07000C0000830884226DD401A79080BD298F87E10401E4FEA670701F1010188F87E10EE
:20E09000F3D1BDE8B88198F87E000D49087098F87E0088F8810098F87E00401C88F87E007B
:20E0B0000320F9F709FEBDE8B881002088F87E00072005F067FEBDE8B881C046640E002043
:20E0D00088190020F8B5064609F022FC2A4D0746A91991F8ED00421C002881F8ED2045D141
:20E0F000264C04EB8604267806F03F003F2801D0FFF7E8FF607800F03F003F2801D0FFF708
:20E11000E1FF648836F07F0018D1F0090FD24FF0805000F5DC75D0F8B80141692046884706
:20E130002868416B204688470128F9D11EE005EB8405D5F800110120884717E04FF080551B
:20E15000D5F8B801C16920468847D5F8B801416A20468847D5F8B801C16A2046884708492D
:20E1700001200860074908688008FCD3384609F0CBFB0020F8BDC046940F00207C8801000F
:20E1900028200860282008402DE9F041054608F0B1FF287E000904D2287D012808BF0227B2
:20E1B00000D00527DFF89C80464670688047264C04F124010B68002B08BF0D600CD07F1E5E
:20E1D0000026FFB202E07F1E1346FFB253F80C2C22B92FB143F80C5C012601E0002FF2D1F4
:20E1F000D8F8081088471EB3216928468847E88AA168C00818D2D8F80400804794F82F102D
:20E21000491C84F82F10D8F8081088470C4991F8380028B10846C06C10B18047BDE8F08110
:20E23000FFF72AFCBDE8F08128468847BDE8F081F1206870284603F04DFDBDE8F081C04699
:20E25000EC1300208C140020640E002070B5214E002086F85400032186F85500E82008F0C0
:20E27000E7FC5220012108F0CBFC1B4D482205F1700406F15C00214601F00CFA174868673D
:20E29000343CF4601648C5F880001648C5F888001548E8671548C5F8AC001548C5F8900050
:20E2B0001448174CC5F8A00013481649C5F89400124847F23052A86704F1980005F0F2FD92
:20E2D0004EF660221049A06104F1BC0005F0EAFDE06170BD481300209012002009CE0000FF
:20E2F000650E01000D0A0100894E0100ED5100007D0C0100BD1A010011E60000BD570100FE
:20E31000A4100020E96A0100456601001A481B4901641B4941641B4981641B49C1641B49AF
:20E330000165022280F8202019494165194981651949C16519490166194941661949816698
:20E350001949C16619490167194941671949016019494160194981601949C1601949016100
:20E37000002180F83C1080F83F101749C161C162012180F830107047403000208173000027
:20E39000D1320100453F010099370100C5230100C14E0100B5610100C9420100752E010053
:20E3B000DD460100096E0100FD0601000D430100796A010035730100A565010005FC0000C3
:20E3D000292401005177010065730100F0B52B4D05F12C0158C9ADF11C0D02AA58C20AC97C
:20E3F0004FF0805682E80A0047688468D6F8D001C16820688847216821488A6B10408863A8
:20E41000206840F2F271416497F83C0097F83D10C0100DEB80008068084321684863684626
:20E4300009F01AFAD6F8D001397F466805EB8101BA698B68797F206855F821101943BB7F9E
:20E4500005EB8305AB690B430199B0470D490A1F106840F010001060086840F00100086091
:20E47000A07D0027FF2802D0E07DFF2800D11FB1086840F44040086007B0F0BD10890100A0
:20E490000DF8FFFF30100040042998B54AD108F0F5FD254C04F1400282E8030004F114004C
:20E4B00009F044F900280EBFE068C068E06041681E4A09781160416812680978914207D020
:20E4D00087692FB16FF0FF0100224FF00073B847022007F0F3F81120FFF7F4FD012060711C
:20E4F000E168087C10B12079012803D00E20FFF7E9FDE16849680E488F680FB9CF681FB1C9
:20E510000021C1610B4F07600B4A40F2FF7111600027876109494161094808F0B3FF192048
:20E5300009F096F998BDC046700A0020D021084000100440510007060000046002000040BD
:20E550001591000029482DE9B0410025DFF8A080294C0570ADF1140D88F83B50012088F81C
:20E570003800201D006888F83D508047234924310F686FB1797E8A0806D341F001017976FE
:20E59000397E01F0FD01397657F80C7C002FF1D1A1688847102008F0DDFE082008F0DAFE7B
:20E5B00098F83C00E0B90920124C8DF80000B4F88A108DF80F50E027ADF8021094F8A7308F
:20E5D0008DF8017094F8B6208DF8043094F8B7108DF8052068468DF80610FFF749F801E0BC
:20E5F00088F83C5005B0BDE8B081C046EC130020F0170020A81100208C140020640E0020FD
:20E6100070B505462B4C2878ADF1200DEB2829D040B3E92806D0E12843D14FF4FA7007F0F1
:20E6300065F83EE004F156010878401C087094F85200032818BF042803D14FF4FA7007F02B
:20E6500055F894F85600032809D094F85200022827D104F10800102108F0B2F921E007F0AE
:20E6700013FC1EE094F85200022817D104AE6946304606F08BF85220002108F0C1FAE068AF
:20E6900020B1026812B1304669469047042006F08FFE04F10800102108F092F9002084F87C
:20E6B000560005482A30016809B12846884708B070BDC046481300209E13002010B5401E93
:20E6D000ADF1380D28D0401E09D0801E4FD0401E43D0401E3FD0401E3BD0002048E001A823
:20E6F00000F004FD04460CA942F2090005F062F99DF83000002808BF002203D0022007F0CB
:20E710005BF9024601209DF83010009001AB204605F07BFC0A3028E001A800F0E7FC044641
:20E730000CA942F2080005F045F99DF83000002808BF002203D0012007F03EF90246002045
:20E750009DF83010009001AB204605F05EFC001D0BE020200CE002200AE042F2130004A9AF
:20E7700005F028F904A808F00BFD80B200E004200EB010BD70B52A4D0C460646A00833D21F
:20E79000A00F48D306F034F9234808F07BFE2648401C0078012803D006F1380009F09CF8A6
:20E7B0001E4800240460022006F070FF1120FFF7FDF8307C10B90E20FFF7F8F81949AC71B0
:20E7D0000878EC7128B10C7005F1D400042108F0D3FBB5F92400B5F92610884214BF0220CD
:20E7F000072001F0BDFE70BD05F12006304608F09DFFFCF7EDFD304608F098FF30B924F004
:20E810000204A00F07D34FF0005100E0022105F1D40008F0B1FB70BD99E40000000004604A
:20E83000700A0020FF310020700A0020F8B505460E460520287096F849006968E870F06BE0
:20E850004861686806F1280108F0AEFCB6F842006968488196F8460069684874686800248E
:20E8700004761F4869680078C873686806F11C01193008F040FF307C69688873706810F867
:20E89000011B6A68918110F8013B6A68918941EA0321918107786A68F91117F007071174E2
:20E8B000214607EB470218BF012189184018401C10F8011B297201F00702E860491001F00D
:20E8D000380101EB420140187268318968618B18834239BF2C72211C801A091A2974F8BDC1
:20E8F0005E1200202DE9F84F274C834620888A460A254FF0FF09002604F138084746401CAD
:20E91000208038465946082207F0B8FC30B16D1E07F1080706F10106F3D100E0B146B9F19F
:20E93000FF0F05D12079401C2071FF20BDE8F88F4846694602F020FD0646FF2EF5D09DF8F3
:20E950000000012806D0606B06EB8601401880F804A004E0206B00EB461080F81FA00B49B6
:20E970000A6808EBC900026049684160084D6868804794F88810491E84F88810A96888473A
:20E990003046BDE8F88FC046AC2E0020E88A01008C1400202DE9FE4FDFF888804FF0010B05
:20E9B0000446DFF8849088F800B099F80000012803D058460021F9F795F8204606F090F835
:20E9D0001F4F7868804700241A4D02901749286A174A86684C8302238DE81800164B10685A
:20E9F00018318A462246B047B968A88000280AD4124A92F90000401C10700298C5F80CA07A
:20EA100088475C460BE0404604700298884748460078012803D020460146F9F763F82046C7
:20EA3000BDE8FE8FD01A0020E81A0020280D0020941900202816002039380100D11A00206B
:20EA50008C14002010F47C1F70B51CD110F00F0F1CD001460024012202EA0100914352008A
:20EA7000401E0BD0401E07D0801E03D0001F07D1093404E0241D02E0E41D00E0641DA4B2B4
:20EA90000029E9D133E010F00F0F01D0002070BD064602244FF4803505EA0600AE436D0077
:20EAB000B0F5803018D0B0F5803013D0B0F500300ED0B0F5802009D0B0F5002004D0B0F5C2
:20EAD00080100FD1072008E0062006E0052004E0042002E0022000E00120FFF7EFFD24184B
:20EAF000A41CA4B2002ED7D1022CD8BF0024204670BD704703B42DE9F04F92461E4609AFE7
:20EB1000BAF5806FADF1040DA8BF052041DA97F80090B9F1400FA8BF09203ADAB7F8028004
:20EB3000B8F5806FA8BF072033DABF88B7F5806FA8BF08202DDA194C2079032808BF032003
:20EB500027D04FF0000B09F03F01C8F30900C7F3090584F805B040EA013045EA0035E18846
:20EB7000A0782A4602F0F0FC014600290BDCA6F80CA0A6F80AB03560B780A6F8068086F8B8
:20EB900008900A2005E0A07889B2324602F0ACFE607901B0BDE8F04F02B07047481A0020FE
:20EBB0002DE9F0470020DFF89080224E234D88F83D0096F8719095F84000401CC0B20428FE
:20EBD00085F8400030D0202005F06CFF96F8B3100F2917D098F83E7096F87100B84211DD33
:20EBF000194C8946606886F87170804782461448144950F827008860C86004F0BFFFA16828
:20EC10005046884795F8401096F8713038F819404FF4707205F11000491C9A4001FB14214F
:20EC300007F096F9BDE8F08706F05AFBFFF78AFCBDE8F087A8110020F017002024310020CA
:20EC500050890100281A00208C14002090B5044600214022ADF1440D684602F086F8A07871
:20EC70008DF80000E0788DF801009DF8000000BB616811B101A805F0C8FB217A01F0070250
:20EC90008DF82820E0689DF82870C1F302118DF8301027B19DF828100B9000EB41009DF895
:20ECB000307007B10D90207C8DF8380067690F9719E0616811B101A805F0A7FB677A8DF856
:20ECD0002970A37A8DF82A30207A8DF82800E27A8DF82B20217B8DF82C10677B8DF82D70BB
:20ECF000E389ADF82E300348006801696846884711B090BD1C1A0020F0B501290446054633
:20ED1000ADF1140D04D0022941D142F2030001E042F20200694604F04DFE04B16D1C07F0A2
:20ED300053F9C01DC010C0B2002830D000230646ADF1010C1F4618461CF801EF00224EFAE5
:20ED500002F101F00101884211D028B97F1CBFB25CB102EBC30103E03CB102EBC301491E7F
:20ED700005F8011B091205F8011B80F00100521C082AE4DB761E03F10103DDD130B12CB16E
:20ED9000D800401E05F8010B001228700FB9002005E004B12770012000EB870080B205B0E7
:20EDB000F0BDF0B50446ADF12C0D08F0CBF9002818BFFC2048D168462146112200F06AFC42
:20EDD000E67CA07C8DF81360257D8DF81200677C8DF81450637D8DF81170A67D8DF81530D5
:20EDF000002006B1012094F82450E28C8DF81600267E8DF8245094F82530ADF826208DF814
:20EE10001860E07D8DF825301A258DF8170057B9812007F0B1F804460A94A4B1FF21812207
:20EE300008F094FC09E09DF81510880000EB411080B207F0A1F804460A9424B1072069467E
:20EE500003F054F9002528460BB0F0BD2DE9F843254C80466068804781466946722006F052
:20EE700087FF3225FF27002600994046091D07F05DFE012808D000986D1E06F1010600F1AF
:20EE900018000090F0D100E03746A16848468847FF2F18BF381C22D1144DD4F804900A27F8
:20EEB0000026383512492846082207F0E7F930B17F1E05F1080506F10106F3D10DE040462F
:20EED0000168296040686860C847064A92F88810491C82F88810A16888476436F0B2BDE80F
:20EEF000F883C046AC2E00208C140020AC2E0020E88A0100F8B5214C236813B908F0DAF91E
:20EF10002368234808380068044608F0FDF8D860204607F08DFD1F4D188268688047064604
:20EF30001748A9680278832A24D1164CE21D17783FB98522027030468847002001F08AFA5A
:20EF5000F8BD86210170082007F034FB26340E4F0E49114B208840F64852B962401C19789C
:20EF7000208007F12000B2FBF1F101F2A32107F097FDA96830468847F8BDC046640E002055
:20EF900008320020C818002098180020D93B0100481600208C140020CC190020F0B52348CF
:20EFB000214D4FF08056A861D6F8D801204C036801210A46ADF13C0D20469847D6F8D801F2
:20EFD00042680121204690471A48012606601A48F9F7D6FA05F01AFB05F11C07384607F06F
:20EFF000B7FE05F134044FF4E13039462060002005F02CFB11493C22082308600021684675
:20F0100008F022FCA4344FF46170002307940C4908906A46069605F1880008F011FC08F06C
:20F030000BFC0FB0F0BDC04608020020FB7601000040034004011CE21888010068060020F6
:20F050007D28000038B504F073FD02F079FE204D05F13800007820B11F480838016801202C
:20F0700088471E48007810B91D48007808B108F021F91C4C606880471B4AA1681378022B45
:20F090001CD1144CA31C1B78042B1CBF832313708847A17831F0010008D0042906D005297B
:20F0B00007D10020207108F059FB01E0FBF7DAFCA178042903D007F0FDFA00E0884795F87F
:20F0D000380020B1E86C10B1102008F043F938BDEC130020C81800204016002004320020BE
:20F0F000063200208C1400200832002070B50446E820ADF1280D09A904F068FE9DF824007F
:20F11000694607F006FB00280CBF00981E480DF125016060E82004F059FE9DF8250004A9A9
:20F1300007F0F7FA58B90599C8200322B1FBF0F0401EB0FBF2F15143401AC0B200E0002043
:20F15000207206F041FF00216081656821700F4B61700A4608925968A9420CD1197A267AA6
:20F17000B14208D15989814205D1187820705E786670104606E008990C33491C0629089123
:20F19000E9D901200AB070BD38C40D00D41500202DE9F047254C01258246984691460E46CE
:20F1B000C4F87C570320C4F8805708AFC4F88407D4F88C0710F0030FFAD1387858B14FF0C8
:20F1D0008057D7F8B001016A27208847D7F8B0010169272088470220C4F8FC06C4F808940F
:20F1F000284608F067FAD4F808040008F8D2D4F88C07800F28BF281C15D2B8F1010F14BF02
:20F2100008200C20C4F84C051021C4F850150020C4F85405064A1560C4F800A0A160C2F81A
:20F2300000542662A162BDE8F087C04604400240000048422DE9F041DFF8948006460C46DD
:20F2500036F07F0015D1002E3ED1224D243D686880471E49096831F81620144321F8164072
:20F27000A968884741461431086807F033F9BDE8F081042006F0F0FF071C25D04FF6FF7054
:20F2900038807C8008F082F941468C78A7F10C05FF2802D0C96A40184478FF2C06D1384643
:20F2B00007F0CEFF07F0ACFABDE8F081304607F005FC01463A46FF20A872204605F026FFD9
:20F2D00010B1384607F0BCFFBDE8F0812C2D002068180020B014002025483EB5007800281A
:20F2F00043D042F20100694604F064FB42F2050002A904F05FFB1D4D95F8540010B39DF8DF
:20F31000080000249DF80810009B2864642285F85440581A02FB00F1E96705F1780003F035
:20F33000D3FE01A805F0B0FA124801992E300078B1FBF0F2451E4243891A01918D4214D973
:20F35000204610E09DF8081064204843E86705F1780003F0B9FE288F401C288700242C64AE
:20F37000012085F8540004F00DFD3EBDF02D002035120020382F00202DE9F041224C064666
:20F3900004F1580005780F46002D04BF0020011C1CD0204D1D49281D0B780068D3B91C4832
:20F3B0000568E06C07F028FF228FB0FBF5F1B0FBF5F3891889B203FB05F2236C3980801ADE
:20F3D000C018306085421CD8401B491C30603980BDE8F08180475FFA80F804F1780007F0DF
:20F3F000F7FF226C4FF47A73410001EBC001B1FBF3F0238F3060A9683B8080183060404610
:20F410008847BDE8F081C046F02D002035120020402F00208C1400202DE9F043254C0746F7
:20F43000243C606AADF1240D00283ED0002F3CD0387A002839D004F01DFF5FEA000834D00A
:20F45000062000250323A1468DF808002E46ADF80A30B5F5FA7F28DAD9F82400ADF80C5049
:20F4700004AB02AA0469009392E803000A230022A047B0B9387A9DF81810814210D10228C8
:20F4900004D1BDF810103A88914207D0032807D104A93846082206F0F1FE08B9284606E0F4
:20F4B000761CB04505F10105D3DC4FF0FF3009B0BDE8F083C8100020F0B520480127F84264
:20F4D00001D004F0A7FB204D204F214EBD4206D203CD0478A4003459401CA047F6E71D4891
:20F4F000002800D08047164D164FBD4202D210CDA047FAE7F0BD03251BE0416808300A1C26
:20F510002A400BD11A1C2A40AB4305D0046804300C600431043BF9D1131C05D00478013037
:20F530000C700131013BF9D1021C2A4001D0A84304300368002BE0D17047C046FFFFFFFF8F
:20F550000000000000000000400E0000A00E0000000E000055C5011070B504466068254EBC
:20F570004078ADF1480DC00921D3B4F842003546B63DB5F88A10884219D11D480078A0B986
:20F5900095F8940098B104F1280006F0A5FC70B9012000901C340194B5F88A3005F17A02A5
:20F5B00003210620F8F7C4F81FE007F033FA0BA80021182201F0D9FB02A821460C900BA8F0
:20F5D000FFF734F92C208DF82C000BA803F01EFC3546503D287810B19DF83C0028B1052003
:20F5F0008DF82C000BA8FEF743F812B070BDC046ED1300205E120020F8B5234D012001463D
:20F610002870F8F76FFA6FF00100204C1D4927690870381C28D0A1684268914203DA07F00A
:20F6300049FE27693846C8B105F07AFC7968884224BF2769381C11D200F084FE14E0266937
:20F650007068002802D507F035FE2669304604F03BF9B168307B88472769384620B105F005
:20F670005FFC79688842EAD2094C606880470646FEF7CEF8A1683046884707F003FA00206B
:20F690002870F8BDCD1A0020E81A0020281A00208C140020002A4AD05FEA000C8B071CD1AA
:20F6B000830722D1102A08D370B4103A78C978C0103AFBD270BC103238D0042A2CD3082AD5
:20F6D00005D30C2A24BF08C908C008C908C008C908C092072AD0920F22E00B780370491CCD
:20F6F000401C521E22D08B07F7D1C30714D18307D8D0121F12D308C903801B0C4380001D90
:20F71000121FF8D20AE008C903701B0A43701B0A83701B0AC370001D121FF4D2121D05D050
:20F730000B780370491C401C521EF9D1604670472DE9F843002A894607464CBF47F6FF7518
:20F75000151C002F08BF002032D03888002808BF002403D02A4600F0E5FA0446281B26DDDB
:20F77000388828B1291B484612A204F00BFE0419B868E0B1D7F804802E1BB8F1000F0DD05E
:20F79000404607F0FDFC401DB04207DC291B484609A2434604F0F6FD04192E1B122E06DB3D
:20F7B000BB68291B484606A204F0ECFD04192046BDE8F8833A2000C0222573222C2000C01A
:20F7D0006C696E652025643A200070471CB51F4C04F1780006F0A4FA04F15C0006F0A0FA99
:20F7F00004F1940006F09CFA0021882204F1340007F0ACFF07F024FC06F0E6FB84F85A008A
:20F81000134984F85B001348086001200DF1010184F8B30042F2040004F0CCF842F2050069
:20F83000694604F0C7F80C489DF80110A0666420414321660949C4F884109DF800104843F5
:20F85000E0670748C4F8A0001CBDC046F02D002038160020BD54010079390100E9F200007C
:20F87000A1760100D0B5244C04F124010F68002F3FD0002215280AD13B7D0126022B08D07E
:20F89000032B06D0052B04D0042B02D000E03B7D0026984200D016B17B7E5B0905D23A466C
:20F8B00057F80C7C002FE5D123E00846394605F053F9F88A2760000A03D397F91C0007F0DF
:20F8D00037FC387D022818BF052802D1012006F071FE2068407E30F07F0005D194F82F0033
:20F8F000401E84F82F0004E094F82E00401E84F82E003846D0BDC046640E0020F0B50546B6
:20F91000224CAF686068ADF12C0D5FBB0C2000F0E5FD071C1DD0684600212422082307F054
:20F93000B7FF002306976A466968ADF810301848059307F07DFF386070B908200C26ADF8B0
:20F950002400616AADF8266009A88847384606F05FF86FF0030017E0E86878602869B86008
:20F97000AF6009E080470646386806F093FE2869B860A168304688473868696807F07CFF6B
:20F99000386807F089FF00200BB0F0BD8C140020A17401002DE9F0418046204800680E46A9
:20F9B0004169272088471E4D0124C5F87C470327C5F880771B480460C5F88477D5F8040435
:20F9D00020F00300C5F80404D5F8040440F00100C5F8040404FA06F6C5F8FC6312480460A0
:20F9F000C5F800801020A860204607F063FED5F88C074008F8D3D5F88C0710F0404F0AD187
:20FA1000C5F884770020C5F8FC06D5F80004864218BF201C00D10020BDE8F081B0010010CB
:20FA30000440024000E04842000048422DE9F843234D884606464FF0FF3105F12400814611
:20FA500007F04EFF00200CE0FF2909D02A688A4204D905EB8101D1F894700FB1002627E0DE
:20FA7000401CB8F1000F03D018F82010FE29EBD10024346074600127B46011E0FF280ED0AE
:20FA900005EB80000B787268C0F8946007FA03F0104370600A680949304605F0B9FB641C63
:20FAB000B8F1000F04D008EB84010878FE28E5D1484607F011FF3046BDE8F883007FC767FE
:20FAD000542B0020B0B5456884682349607DA27DADF1180D40F000400090207D0027FF2A61
:20FAF00041EA000001904FF0020002D0E27DFF2A00D13FB1E37DA07D1943039140F0004001
:20FB100002900420FE214DF8201005F158006946FFF78CFF6866002808BF381C1AD0617D34
:20FB30000F2205F0F9FF686E217D102205F0F4FFA17D3846FF2902D0E27DFF2A00D140B129
:20FB5000686E112205F0E8FF686EE17D122205F0E3FF012006B0B0BD0000C0A098B5244C10
:20FB70000746A8B1401E0BD0401E2CD1204690F8402042F0080202F0EF0280F8402022E0F4
:20FB900094F84020204602F0E70242F01002F4E7214601F17402107891F83C3000F0F000DD
:20FBB000107003F0F000002281F83C0091F840308A6343F0080000F0EF0081F84000F4202E
:20FBD000413104F003F9002F08BF44F620600CD007F028FD4FF4FA670A2244F6206390FBF3
:20FBF000F2F15143401A07FB0030A06498BDC046280D002038B5054695F83000032839D114
:20FC100095F83A00032835D105F128044A202146F9F740FB8A202146F7F778FE6C6861789C
:20FC3000207800EB0120ADF8000069465020F9F731FBA41C6178207800EB0120ADF800004E
:20FC500069464B20F9F726FB8B206946F7F75EFEA41CE1202146F9F71DFB641C61782078A4
:20FC700000EB0120ADF8000069465320F9F712FB002000E0E82004492A24087028462C707F
:20FC900003F0C4F838BDC046D13000202DE9F8432020EFF3118780F31188214CA0680121DB
:20FCB00007F0C2FD4FF001094FF0000865692168A4F81C906A1A2168A4F81E80461B401A4D
:20FCD000904227D387F3118840464519361A4846294607F0A5FDB042F7D92021EFF31187EE
:20FCF00081F31188E18B012903D14046294607F097FDB0F1FF3F06D0A169801B814238BFE9
:20FD1000081C411901E0A069291807F085FDA4F820902560A4F81C8087F31188BDE8F88375
:20FD3000780100207FB503461F480D4601881F480088144614A6984205DB32462146284650
:20FD500004F020FB1DE0994206DB184606F0C2FC0028F2D04268F1E715480088002808BF79
:20FD70000CA2EBD00095002C48BF47F6FF74114E0020114901946A46346802901846A04701
:20FD9000029800907FBDC0467B6D6F64756C652325647D007B6D6F64756C652D726F7065D9
:20FDB0003A25787D00C046C08A8A01002E8B01008E1400004C8B01003D5901000FB42DE960
:20FDD000F04106AF8046ADF1300D07F0E5FB3E1D002526F00306361D0A961420ADF8240026
:20FDF000FF24079508268DF826407868ADF80060164F0B901A203968ADF802006846884737
:20FE100008B99DF80440ADF80860ADF80A600320ADF80E800AAB8DF81000243F8DF80C4048
:20FE3000796A059302A8884706A8069504F0B4FF012804D018B9069808B106F0CBFA0A984C
:20FE500000680CB0BDE8F04104B07047B014002090B50C46214A0178575CADF11C0D0B2F1A
:20FE70008DF8007035D0002F36D00C2F04D0112F29D107F0E5F926E01A2C22D090F89910B6
:20FE90000190C7688DF80210038A0297C28AADF80C30510905D21249827E98310978891A2F
:20FEB00000E000218DF80E10877F8DF8107090F91F308DF81130826A0592417F8DF80F10FE
:20FED00001E0002001908DF801406846FDF7D0FB02E04470FDF722FA07B090BD24830100FB
:20FEF000A81100202DE9F04107467868BE68044600F5847006F0CEFB30681C498069096836
:20FF1000C0F3C00008BB07F003FD194D8046287820B1022005F0BAFB00202870404607F006
:20FF3000F3FC3168134D886B20F020008863286820F480702860606A216A091A2162236918
:20FF5000626A38469847BDE8F0814FF4FA70B0FBF1F1012998BF012104F58474204607F027
:20FF70008BFC204607F098FCBDE8F081388B0100FD310020301000407CB515460E46044627
:20FF900000E004192046694605F02CFA00282ED014F8021F8E42F4D1491E04F1010420D0EB
:20FFB000491E12D0491E08D0491E18BF622029D102281CD12078287023E0032817D114F886
:20FFD000010B2870207868701BE007280FD161782078A41C40EA0120288020682E1D30606C
:10FFF0000FE0052803D120780628287001DD67204E
:020000040001F9
:200000007CBD2D1D0020641C2860A678AE702088288000207CBD70472DE9F0410646756829
:20002000B46807F07DFCA96A39B921688969090903D207F071FCBDE8F0810027AF6207F024
:200040006BFCA17D3846FF2902D0E17DFF2900D118B12846214601F0E5F82168886B20F054
:20006000200088630D49086820F48070086007F057FC0B4C8046207818B1022005F00EFB5B
:200080002770404607F048FC686A296A091A29622B696A6A30469847BDE8F08130100040A2
:2000A000FD31002038B50C4644220546002100F064FE04F12801284606F076FE04F1320171
:2000C00005F10A0006F070FEE06B6861B4F840002883B4F842006883B4F84400A88394F891
:2000E0004600A87794F84700E87794F9480085F8200094F8490085F82100B4F8500068849C
:20010000E06C6862A07B85F8280094F8520085F82900606D0B2204F11C01E86205F1300009
:20012000FFF7C0FA2089A5F840006068E86338BDF8B507F0F5FB204C0746D4F8A80010F4BC
:20014000602F2CD0D4F8A800400CC6B2700807D2B00803D2F00828BF022602E0012600E00E
:200160000026751D68B202F035FFD4F8A83006F111010120884023EA00013846C4F8A810F1
:2001800007F0CAFBB00004F190010A18D7684FB1085800224FF000632946B84702E038461A
:2001A00007F0BAFBD4F8A80020B104F58470002106F0EAFEF8BDC046700A002070B51E4D7D
:2001C000AC68064606F084FD4FF47A71001B4843030C05F0E9FD2969401A48BF404240F6DF
:2001E000B8319B19994210D306280EDAE9688C420BD8286848B1114A091B51438A0C02EB6D
:200200001141884288BF011C08E00D49486840080ED208687D2100F0FF004143C82905D3FE
:20022000B1F57A6F88BF4FF47A6103E0C82101E04FF4FA61084670BDD031002040420F0052
:20024000AC3F005003B42DE9F0411F4DA8684FF0FF3106AF98461446ADF1180D07F048FB90
:20026000396804A80160B988818004A803C822466B46FEF747FC0026071C0FD1BDF80C00DC
:2002800084421CBFADF80C40BDF80A6008D12246684631464346FDF78FFD07460A2F09D1DE
:2002A0006846414603F0BEFD07461EB1304605F027FF6F79A86807F017FB384606B0BDE8D4
:2002C000F04102B07047C046481A00207CB5042005F0FEFB022818D0032816D019480068CD
:2002E000C0F38150032814BF41F288324FF47A721649174C096854342046B2FBF1F107F0B9
:20030000C3FA204607F0D0FA7CBD4FF08056D6F8A4010D4D446800214FF040521C230320DE
:2003200000902846A047D6F8A40100214FF4007209230126446800962846A047022005F08E
:20034000ADF97CBDB43F005000A00C40388B0100940F0020F8B51E4C002528462268A168CB
:20036000256190420CD05268914209DD04F0E0FD0146206842689142C8BF41602061A16807
:20038000676837B118B142687B689A4201DD38462061C8B14068814216DD0E4E044606F123
:2003A00008000068A04201D806F08CFF0A4D686880470746F460204601F0F0F9FDF730FAA4
:2003C000A96838468847F8BD05F03CFF2561F8BD281A0020CC1900208C1400202DE9F84327
:2003E0001C481F4D07786868804781461A4883680026344680469C4212D013F8020C8742FB
:2004000008D134B163B138464FF40041FEF71AFF13E01C4604B91E4653F80C3C002BECD109
:200420005FB9686880470D49096831F817206FF3DF3221F81720A96888472CB108F1080065
:200440002146324604F090FBA968484688472046BDE8F88314150020681800202C2D0020E8
:200460008C1400202DE9F041804600271A481D4D07701A481A4E077096F83800D8B1F36F53
:200480002C68C3B1207D352809D16068218900F0F3F860680088000901D304F047FBF16F70
:2004A000404688471048007801280BD038460146F7F720FB06E003F043FB01F049FC404672
:2004C000F8F7B6FF286810B1007D352801D006F0CBFCBDE8F081C0460032002008320020F7
:2004E000EC130020640E0020E81A0020F8B5001D84B214F0030002D0241A241DA4B206F085
:200500002BFB1A4A102C01461769D160C8BF5769388800221646C30BDD0319D126B984425B
:200520000ADD3A46012617E01388C3189BB29C42138011DC174618469FB1001B80B2042891
:20054000B4BF3C88385344F400443C803F1D08E080F40040002680B2C71938880028DAD1DE
:200560000027084606F028FD3846F8BD8C140020F8B5054607F0D4F91D4C064604F5B87165
:200580000878A84304F59E7508702868002808BF002706D02868943007F0E6F8002700B1EF
:2005A0000127686838B1943007F0DEF80025384318BF01252F4694F87001A8B9012F13D046
:2005C000D4F8640198B1406988B10746304607F0A3F9D4F8640100214FF400030A46B84782
:2005E0000020C4F86401F8BD304607F095F9F8BD700A00202DE9F8431E4C00264FF0010892
:200600004FF002093746A41EA51C15F8020F03280ED0022822D16878236802281ED007F0D2
:2006200093F80146384606F08FFF85F8019010E007F08AF8014623686878012805D0384641
:2006400006F082FF85F8018003E0404606F07CFF6F700246C9B2184604F0DEFB761C042EBA
:20066000D3DB05F005FC18B104F1240007F068F8BDE8F8835E1700200829C8B50BDA00292C
:200680003BD00278491E92FAA2F24FEA226200F8012BF6D1C8BD464206F00306891B3718A7
:2006A0008AB2361802F00301864209D9361A0378761E93FAA3F34FEA236300F8013BF6D1D4
:2006C00022F00302D71987420AD93A1AD21C96100268761E92FAA2F212BA40F8042BF7D166
:2006E000CF19874209D93F1A01787F1E91FAA1F14FEA216100F8011BF6D1C8BDF8B50546C8
:20070000012004F0D7F91D4C04F1140003F0E4F804F1240003F0E0F869684A78087800EBD1
:200720000220ADF800008F7804F114066FB953206946F8F7B7FD05F128014A20F8F7B2FDC8
:2007400005F128018A20F7F7E9F806F1200005F11C010B2206F0D0FBBDF80010384604F0B2
:20076000ADFD94F83F00800803D36878002106F03FFB002084F83F00F8BDC046403000204F
:200780001C491B4898B5FF220F7890F83B301A4980F83820012B15D091F8710091F8901042
:2007A000884224D015480024047006F0A9FF01F09FFE13480078012819D020460146F7F7DA
:2007C00099F998BD002380F83B3087B18DF8032091F8A7008DF8000091F8B6708DF80170F2
:2007E00091F8B7408DF80240684606F030FF98BDF0170020930E0020A81100200532002072
:20080000E81A002070B50025ADF1200D07A8ADF81C5006F037FD1B4CBDF81C10208F8842F6
:2008200027D194F85300032811D004280DD0022810D104AE6946304603F0B0FFE06820B12F
:20084000026812B1304669469047042000E0032004F0B6FDA06D04F051FF5220294606F079
:20086000D7F94FF47A7004F061FF284604F076FF05E0032006F0AAFC052004F0A1FD08B03D
:2008800070BDC046481300202DE9B84107F048F81C4C1B4D804604F1E000007848B92C460E
:2008A000A168022088470746102003F051FD0FB31DE001F023FD70B9134800683221B1FBC5
:2008C000F0F101B901213034204606F0DDFF204606F0EAFF0EE0002084F8E0002C46A16895
:2008E000022088470746102003F032FD17B1A16803208847404607F00FF8BDE8B881C0463D
:200900008C8A0100940F0020388B0100F8B51B4E0024012004EA0307194D3070002F4FF072
:20092000020000EA020008BF00280DD14FF0E04004EA02011840002808BF002904D112490C
:20094000888D401C888503E095F90000401E287006F084F806F088FA0A48047095F9000074
:2009600030B195F90000002806DC06F0ABFC03E020460146F7F7BEF83470F8BDE81A0020B2
:20098000D11A0020CF1A0020C81800201D491E482DE9F041352751F8048B51F804EB51F87B
:2009A00004CB51F8046B51F8045B40F8048B51F8044B40F804EB51F8043B40F804CB51F8AA
:2009C000042B40F8046B40F8045B40F8044B40F8043B7F1E40F8042BDDD151F8045B51F809
:2009E000044B40F8045B51F8043B40F8044B51F8042B40F8043B40F8042B09680160BDE835
:200A0000F081C046C802000000C0002138B505461B491D4C2878E0B96878012815D002285E
:200A200009D0032826D10846002181704021083005F0CEFF1EE004F13A000078FF280CBF69
:200A40000120022006F0C2FB14E004F108002021EEE76A78032A08BFEA2804D0012A09D1D8
:200A600041F2883000E0074891F8542081F8552004F074FE7434216809B12846884738BDEE
:200A800048130020E09304004813002070B51B4C05461022ADF1200D04F171016846FEF70B
:200AA00001FE0026049509208DF8146004F10D018DF8160001258DF815500A680DF1170021
:200AC00002604A684260097A01720D496A461820FFF77CF90B4918208922631DFFF776F9A5
:200AE0007120314606F0E6FBD520214606F0E2FB5D20294606F08CF808B070BD50860100C6
:200B0000F5A700001D7900002DE9F0431C4E044600271D468846A2EB0409ADF1140DC6F837
:200B2000B071012006F0CEFD3068C00FF9D3306A0090706A0190B06A0290F06A039044B15C
:200B400028462346694611F8012B5B1E00F8012BF9D10320C6F838026CB108EB09016D1EB3
:200B6000491E11F8010F15F8012F904218BF042002D1641EF5D1384605B0BDE8F083C0467F
:200B8000504502402DE9FC410021054606F09DFDB72806D140F6FF712846CA1E05F0D2FCBA
:200BA00040BB154C626805F0B1FEDFF8508001281CD190470646684604F018FB280305F0B6
:200BC0006DFE0746009805F077FEA1683046884737B928460021B72206F09CFBBDE8FC8106
:200BE0000221404641710171BDE8FC8140460B21401D0170BDE8FC818C140020481A002022
:200C000003B42DE9F0431C4DA8684FF0FF3107AF1C469146ADF11C0D06F06AFE396804A88B
:200C20000160B988818004A803C822466B46FDF769FFA846061C14D1BDF80C30BDF80A2060
:200C4000D01A484481B298F802006518AA4204DAA342B4BF0526062603E0BB68224605F000
:200C6000A2FFD8F8080006F03FFE304607B0BDE8F04302B07047C046481A00202DE9184163
:200C80000446DFF870802078E02828D1404642788178012A0AD049B990F85220012A05D16F
:200CA00090F8540001281AD001200CE0104BB3F86620521CA3F8662041B9491CC9B2817052
:200CC00000234370022006F081FA08E0002004F015FD032006F07AFA052004F071FB404605
:200CE0007C30016809B120468847BDE81881C0469012002048130020F8B500680E461746A9
:200D00004FF0FF310446483006F0F2FD4FF0FF35092E08D0217A0120B040084211D1084318
:200D20003546207210E0227A0721012303FA01F0104202D0491EF9D503E0227A0D46104362
:200D40002072B5F1FF3F0ED06FB129463846FEF729FE40B1217A0120A8404FF0FF3580F09E
:200D6000FF000840207204F1480006F0BDFD2846F8BD002213460A46194671B510F0030F28
:200D80000BD0002A82BF00F8011BB2F1010210F0030FF6D1002A08BF71BD11F0FF0141EA2F
:200DA0000121042A18D341EA0141082A0FD30E46102A08D30C460D46B2F10F0312F00F02A1
:200DC00072C0103BFCD812F0080F18BF42C012F0040F18BF40F8041B12F0020F18BF20F88B
:200DE000021B12F0010F18BF017071BD03B42DE9F041DFF86C80D8F808004FF0FF3106AF91
:200E00001C461546ADF1180D06F072FD396804A80160B988818004A803C822466B46FDF779
:200E200071FE061C12D1BDF80A00BDF80C10411A691889B261188842B8BF062606DBBB68AD
:200E4000294622466846FCF7B7FF0646D8F8080006F04AFD304606B0BDE8F04102B0704798
:200E6000481A002038B505461B4C287868BB607801282AD0281DFEF7D7FAB0F1FF3F24D1B4
:200E8000298AC81321D001F00F010F291DD12046018F4FF6FF728A4204BFE9890187A97C52
:200EA00080F83A10AB888387298A01F00F020F2A05D080F85020C1F3031180F8511090F85F
:200EC00050100F2904BF012141706C34216809B12846884738BDC0464813002070B51C4CC1
:200EE00006460E220D4604F12C00FEF7DBFB687B20B9022020776B88A38208E003202B1D57
:200F000020771A6804F114010A6058684860606A04F00CFC30462946FAF7CCFE20780128B5
:200F20000CD0687B50B9288869882A1D002301F053FD011C02D002A006F0CAFB70BDC0461E
:200F400041757468204572726F723A20307800C09012002038B51B4D95F871000F2824D0D3
:200F6000194C3B3C94F83810FF291ED094F83A0068B102290BD103F0DBFF216B0F4C95F884
:200F80006820401A2178083101FB12010BE003F0CFFF616B0A4B95F89020081A1988401A67
:200FA00034F81210411A002901D5002038BD4FF6FF708842C8BF88B238BDC0468919002078
:200FC000900E0020A81100202B1800201649B0B505461B4C0F7820780FBB144A8100B2FB2C
:200FE000F1F1A94202D206F06DF920786168104F800005FB00143868C06B8047211AA1F53D
:201000004871090806D30B4A011B891A090828BF00F5487408482146FCF768FEB0BD0749A3
:2010200001200870B0BDC046E91A0020FFF6C2FF4816002000093D0021DC000007320020B1
:20104000CC1900201C4938B591F85C3001EBE304657F012203F0070302FA03F383F0FF03E6
:201060002B4063778B7E01F11800032B18D091F86030012B10D0022B08D0B1F856108A40FF
:201080009102A1EB821101F570710EE0B1F856209101A1EB820108E0B1F856108A4001E077
:2010A00004490A789102A1EB82111C3005F000FD38BDC04641120020B83000202DE9FC41A8
:2010C0001B4E074670688047184D804605F120000068154C436C04F10C00006802216A46C6
:2010E00098479DF8000028B90D48007890B906F0E9F80FE00B492A6A91F83D00936900F025
:20110000F00040F0010081F83D00E0683A464FF0FF319847B16840468847BDE8FC81C0464C
:20112000E91A0020280D002088190020281600208C1400202DE9F84380461948077817B991
:20114000184D287810B90120BDE8F883164E243E70688047814668880124B8F1000F0ED1A8
:20116000214603464FF6FF72B9404A40104068807BB170B9002004F0B1FF044609E018B931
:20118000204604F0ABFF68882146B940084380B26880B168484688472046BDE8F883C04694
:2011A000141500206C0A0020B014002000B500212022ADF1240D6846FFF7DFFD1848018F15
:2011C000ADF8181090F83A108DF80B10808FADF80E0002218DF8161009208DF80C00012164
:2011E0008DF81F1003208DF80D0000208DF808008DF81B006A468DF81A0007498DF81D00F8
:201200001820FEF7E3FD0549B1F84C00401CA1F84C0009B000BDC046037601009012002085
:201220004813002038B50C4621680546886B20F020008863686E217D012202F017FE686E9E
:20124000217D012203F0E8FD686E217D002204F06BFC686EA17D002204F066FCA87801284F
:2012600006D005F1D0004FF0FF3106F041FB03E0216888690009FCD2686E217D102204F063
:2012800053FCA17D0020FF2902D0E27DFF2A00D118B1686E112204F047FC38BD2DE9F84F13
:2012A000834689467120114604F06AFD174681206946F8F74BFF4FF0F308002507E0B8F17E
:2012C000000F23D038686D1CEDB22C3038609DF80000A8421ADD3868066890F804A000247C
:2012E00002E0641C0A36E4B2A245E8DD737A002B0CBF052009208145F3D14A4630465946AA
:2013000005F080F90128ECD14FF000084046BDE8F88F70471A487CB5007880B342F2050052
:2013200001A902F04FFB42F20100694602F04AFB144C9DF80400216C88420BD80098884217
:2013400003D806F0EFF901250DE00022012584F8542004E001259DF8040084F85450401A6C
:2013600064214143E16704F1340606F1440004F0DFFC06F1440001F0AFFE84F858507CBDAD
:2013800035120020F02D0020F8B50B461A4991F82D704D6B4C796430C2B25FB100206D1FE1
:2013A0006D1DEE7816B12E79B24207D07F1E00F10100F5D1641CE0B2487104E0FF281CBFFE
:2013C0000021197016D10120187091F82C700C6B4B795FB10020203C2034A67F16B1E57F43
:2013E000AA4207D07F1E00F10100F5D15B1CD8B24871FF20F8BDC046AC2E002038B505460F
:2014000001201A4C68712879B0B905F0A5FB2178002904BF6FF00704051C15D0491EC9B2F6
:20142000217039B905F0C8FD606804F09FFA0020687118E0054613E005F08EFB054620788A
:20144000FF2805D16FF00604284605F0B5FD0BE0401CC0B20128207002D1606804F09DFA79
:20146000284605F0A9FD0024204638BD5C1A002070B50646B079F4680628A4F10C042CDA7F
:201480003079062829DA05F067FB154DB27991000C3501EBC20169184968E1B105F08CFDCB
:2014A00030792071B0796071307AA071B179880000EBC1002818F1684068083004F0C6FAB2
:2014C000B179880000EBC1002D186868406806F00BFA002070BD05F06FFD6FF0020070BDBA
:2014E000C014002003B4B0B504AF3878ADF1180D002808BF092027D0164D2C46A0684FF08B
:20150000FF3106F0F5F904A83968BD88016004AB858093E8030000226B46FDF7F3FA254673
:20152000071C0DD1BDF80A0004F0EAFDA878E988009A00F011F86C790028D4BF271C0227E0
:20154000A86806F0D1F9384606B0BDE8B04002B07047C046481A0020F0B516460C46074661
:201560000025ADF1140D0AE0241AA4B205E0641E3846A1B202F0DCFD04466D1CADB2092C9F
:201580001DD3641F38466A46A4B2214600F0B4F90098B04207D19DF8091031F07F0004D0CC
:2015A000C80902D20CE09DF809108808DFD2BDF80C008442D8DC04490520487108716C421E
:2015C00020B205B0F0BDC046481A00202DE9FC47194C6779984691460D46034657BB174EE9
:2015E000301D026805F092F901281CBF0B20607120D105EB033590478246684603F0F6FD68
:201600004A464046294605F03BF9009805F054F9B168504688476F1E4846411E1FFA81F9B7
:2016200040B117F8010F18F8011B8842F4D0022060712071BDE8FC87481A00208C140020F2
:20164000F8B50C461A4991F8AF00C2080AD391F8AE20A24206D100F0FB0081F8AF000027FD
:2016600081F8AE7006F05CF90746204601F0B2FC0D48210201F47F41084304F0A9FB0B49D2
:2016800005460868012604F10C0306FA03F290430860384606F040F905F0FF05012D0CBF95
:2016A000301C8320F8BDC0460100080408100440700A0020F8B51B4D0129044611D005F11D
:2016C0007400064605F02EFE012802D1304606F039F82CB305F0B2FC074605F0AFFC6A694E
:2016E00010E005F15000064605F01CFE012802D1304606F027F89CB105F0A0FC074605F0B2
:201700009DFC2A6900EB0720611090FBF1F34B43C01A0918104605F0A2FF304606F010F8C2
:20172000F8BDC046A410002038B544688568606E05F006F8296817488A6B10408863164855
:201740000068C168286888476868FCF737F904F1800006F065F804F19C0006F05DF8A078EA
:2017600018B904F1D00006F053F8607818B904F1EC0006F04DF804F5847006F045F806F0B7
:20178000CFF80021217006F0C7F804F16C0004F0E9FE38BD0DF8FFFFD0010010154998B55B
:2017A0000F7817BB144A1178144F52688B00890000FB0324B7FBF1F1814201D205F082FDF8
:2017C00011480068C06B8047211AA1F54871090806D30B4A011B891A090828BF00F5487425
:2017E0000A482146FCF782FA98BD06490120087098BDC046E91A0020CC190020FFF6C2FF4B
:2018000000093D00073200204816002009F6000038B517481749007818B90846007828B910
:2018200006E00846007830F07F0001D005F04AFD114D68688047114C0C3C2178A278914230
:2018400007D10F4AA9681278D20803D28847012038BDA968884705F053FFA078FDF7A2F85B
:20186000012804BFA078207005F0FEFA38BDC04624140020083200208C14002094190020AD
:20188000053200202DE9F8438146EFF31188202080F31188174D154C134F012605F11C00B2
:2018A0000660A4F114000660F86A016A14208847D9F81000810C14BF000C04202060386852
:2018C00002682321002090470948066054F8180C20F4C02040F4803044F8180C2E6088F3FB
:2018E0001188BDE8F883C046840100101820094080022443000024433EB514460D460522FC
:201900006B4605F050F99DF803109DF804009DF80430658101F00F01801040EA81109DF807
:201920000150A0819DF803109DF8020003F003030A11800642EA90529DF802006372811150
:20194000A28041EA85019DF800009DF80050E18000F03F0041EA003105F0C005207242EAD6
:20196000013222602B4363723EBD30B504460D4642F20900ADF12C0D09A902F023F89DF88A
:20198000240008B342F20B000DF10E0102F01AF800230094BDF80E000293000401906846C6
:2019A00002F05CFD044604A942F2030002F00AF804F012FB024604A9B4FBF5F06843241A47
:2019C000E0B202F055F906E042F20D0003A901F0F9FF9DF80C000BB030BDFEE72DE9F843FA
:2019E000194D064628780C469846012805D0687A012818BF6FF0010023D162600A202080A5
:201A000001F0BCFA071C1BD4A77005F089FF8146204604F0DDF90446484605F07DFF04F045
:201A2000FF04012C05D0384601F0D4FA6FF0010706E005EB8705903545F8088C45F8146C48
:201A40003846BDE8F883C046700A0020F8B5064605F066FF184C0125074606F19400E5703E
:201A600004F020FE2078012811D094F8700170B1B4F92400B4F92610884208D1384605F0CA
:201A80004BFF0720FEF774FD05F04AFF0746B4F92600B4F92410884218BF86F8BA5007D12F
:201AA00006F1700004F0FEFD284602F085FBE571384605F031FFF8BD700A0020F0B50546B8
:201AC000194C2878ADF11C0DE9281CD028BB002694F8520084F8566002281ED104AF6946A9
:201AE000384602F05BFE5220314605F091F82046C06820B1026812B1384669469047042002
:201B000003F05EFC09E094F85600401C84F85600C0B2032801D104F0BFF98C34216809B161
:201B20002846884707B0F0BD481300202DE9F04107461748174CC01F067860688047804681
:201B40001549A268087886281CD1104D05F12A021088401C10808720087005F00DFDA168D8
:201B600040468847082004F05BFBA879B04207D127B90020FEF776FCBDE8F0811B20F9E71B
:201B8000E920F7E740469047BDE8F081C81800209C3100208C140020083200202DE9F84393
:201BA0000024002B16460F468046254606D5002FC3F1000302D57F42761E2D259946384658
:201BC000494602F00BFE0CA0405CB7FBF9F7002F04F1010408F8010DF1D1A64205DD30217D
:201BE000301B401E08F8011DFBD10DB108F8015D4046BDE8F883C0463031323334353637EE
:201C0000383961626364656600007047B0B5ADF1400D05F07DFE044600213C2208236846E5
:201C200005F01AFE1148416806918168006804900F480068002205900E480891694605F010
:201C4000DFFD071C01D105F04FFD04F085FF0546384602F04BFA08B905F046FD284605F09E
:201C6000ABF9204605F050FE10B0B0BD848501008C140020F572010030B5401E4FF0000432
:201C8000ADF12C0D0AD0401E04D0401E20D1F6F7DFFF1DE000F02EF9044619E001A82146E0
:201CA0002422082305F0FCFD06940D4DADF8144009490794012201AB05F1780005F0ECFDD0
:201CC000064A23462C2105F19C00009305F0FCFD20460BB030BDC046ED2A01005546000024
:201CE000940F002080B501460A7D012A05D0152A03D0252A18BF352A02D1087E00091DD335
:201D0000087EC30916D2012A18BF152A01D1000909D24F781B2F04D00B4807B10E30805C88
:201D200002E0232000E0312008700848007800F097FD80BD48780021884780BD4A7808464F
:201D40001146FEF78DF880BDEF860100141500209EB51849A1F12404606880472146124CF4
:201D6000E288A38893421CD0104B1F78CFB9104B89681F7837F07F0714D1A28088471027F6
:201D8000A088ADF8007001A9ADF8040009880DF10203198008480068426AE0686946904754
:201DA0009EBD896888479EBD881900200632002008320020B01400204816002038B50429BE
:201DC00005462CDA05F0C0FC0346084605F0BCFB134C0246022904EB450000F10400017052
:201DE00012BF0329002141702068D9B203F014F804F03EF850B904F12400044605F092FAEB
:201E000001280CD1204605F09DFC38BD04F12400044605F087FA10B9204605F091FC38BD54
:201E20005C1700202DE9F843174C04F1240108688846074628B300261D25387D35281BD175
:201E400040463946324602F08FFE787E30F07F0005D194F82F00401E84F82F0004E094F8E7
:201E60002E00401E84F82E007D7057F80C9C3846FFF738FF4F4602E03E4657F80C7C002F9C
:201E8000DBD1BDE8F883C046640E0020164880B507683FB315498B6803EA5300C00E21D298
:201EA000134A106880081DD2486880081AD21068096810F0050F4FEA114101F0F00101F552
:201EC000E0710AD1B9420DD2190F38BF40F00100D90E38BF40F0040003E0B94202D920F0D1
:201EE0000500106080BDC04628500940AC3F00500000094098B5154C94F8E100002710B9DA
:201F00001348007860B105F00BFD94F8E310002906BF012184F8E310012705F0FDFC0FB10C
:201F2000002098BD022003F0D1FB0E20FCF7D2F80849086840B9084A402010600127CF612C
:201F4000002084F8E20098BD012098BD940F00209A8A010004800C402C500C402DE9F04171
:201F600080461748243007680E46ADF1300DBFB13869A8B1B8F1000F12D08EB106208DF85C
:201F800028000125ADF82A500022ADF82C2002AC00943C690AAB93E803001A23A04708B1CA
:201FA00000200AE002A940460C22FDF77BFB05A930460E22FDF776FB28460CB0BDE8F08155
:201FC000A4100020F8B50646B06801687568886B20F4FA6088631349086820F400700860D2
:201FE00005F09EFC104C0746207820B1022003F055FB00202070384605F08EFC05F090FCAD
:20200000A96B11B905F088FCF8BD0021A96305F083FC686B296BEB68091A29636A6B30465F
:202020009847F8BD30100040FC310020F8B5844640F6FF741CF8013B002210E0481B401EFC
:2020400010F8015B7F1E01F8015BF9D103E01CF8010B01F8010B521C5B08082AEADA580831
:20206000F5D21CF8010B1CF8015B05F00F07FF1CC5F30315122F45EA001508D11CF8016B35
:20208000300A24BF1CF8010B60F3DF16F719AC42D4D1F8BDB0B5184C05460F46101C28D0D6
:2020A0000DE03868606197F82700394640F0040087F8270004F1200003F0CCF86769D7B19F
:2020C000F8688542EDD014E0386888B13868C06885420DD139680868386091F8270040F059
:2020E000040081F8270004F1200003F0B3F800E03F68002FE8D1B0BD700A00202DE9F843C2
:20210000DFF85880044608EB440000F11805008B894604F0A9F8074611480678AFB12A885C
:202120003846002105F01AFB00253C7041467D700A5D381D494604F0DFFE3046394600F0B0
:202140008FFB40B92846BDE8F8838DF8004068461A21FDF785FE1A20BDE8F8831883010053
:202160001415002010B5164A144C92F83D0094F8401048B91348006860B9012082F83D0039
:20218000202005F0E7F805E0481CC0B2042884F840000DD00C4971310A784FF4707304F117
:2021A000200003FA02F101F2636104F081FC10BD202002F07FFCFCF7CDF910BD2431002072
:2021C000F0170020640E0020A811002010B5044600212822ADF1280D6846FEF7CEFD134956
:2021E00011226846FDF75EFA05208DF812008DF8114000218DF8151001208DF816100B225C
:202200008DF81700FF208DF8180009208DF8130003208DF814000DF11900FEF7AEFD0449E5
:2022200018206A46FDF7D2FD0AB010BD67860100B3ED0000C8B50146164AC87AB8B992F87D
:202240002D70506B2FB3401F401DC6781EB1CA7F03799A4202D07F1EF6D1C8BD8A7FC270E4
:20226000CA880280CA7F0271097B8170C8BD92F82C70106B6FB120382030867F3EB1CA7F2E
:20228000C37F9A4203D12022FDF70CFAC8BD7F1EF2D1C8BDAC2E0020F8B5044605F0ECFADA
:2022A00001F024FF071C17D004F056FC0546A18811480022183030F80C6F46B901804760B9
:2022C000A168816022737868206100240EE08E4205D1284604F070FE6FF0020409E0521CDA
:2022E000062AE8D305F000FA6FF00304284604F063FE2046F8BDC046A814002038B50120D0
:2023000003F0E6FB012820D0114DD5F82401C4681048342101220023A047002808BF00206B
:2023200014D0286803F090FD04F0D2FC0B4A0A4D93681168D060C01AA1EB910105FB00F3AC
:20234000180C884228BF011C1160012038BDC0468000001000A00C4040420F00D0310020D0
:2023600098B50446207B00F00F00022824D100F007FFA168081A8108114800F10C0217688C
:20238000002F14BFFB6840F6C41303F57A728A4212D20A4A12686FF050448C420CD3C91AE6
:2023A000B1FBF2F3012B8CBFB1FBF2F10121B03005F06AFA012098BD002098BD388B01007C
:2023C000700A002010B50446012002F073FB208900280CBFEB2000201249607091F83F0019
:2023E000C20824BF20F0040081F83F00820809D2400813D32B202070EB236370204600F0BF
:202400000DFD0BE091F83F0000F0FD0081F83F00217C6078C1F3001104F0EAFC204604F0EC
:2024200091FF10BD4030002030B5174C054605F12801ADF1140D04F17A0003F00FFC08B316
:20244000EF2309208DF801306B688DF800005A781978181D01EB0221ADF802102A890178A9
:20246000082A8DF8041014BF94F8B600C07805F11C018DF805000DF1070005F044F96846C2
:20248000FBF7FEF805B030BDA811002010B504460320ADF1180D04F128018DF8020000201F
:2024A0008DF8030001A805F031F96068007804F11C018DF80C000DF10D0005F024F904F1D7
:2024C000280003F011FD58B14FF6FF7453206946ADF80040F6F7E6FE044920460A310880C4
:2024E0000DF10200FBF7CCF806B010BD2212002070B5164D286808B105F032F8144C606837
:2025000080470C3DE9690A68002616710968E961A16888470A4A0B49107810B908460078E8
:2025200060B1167008460670FCF794FD06480078012803D030460146F5F7DCFA70BDC04648
:202540000432002006320020E81A00209C3100208C140020F8B50025114C1348A5604FF42C
:20256000700665600068E660C06B80470D49C0F1FF3008600D48C76865700FB90C49C1604B
:202580000C480570012001F0C9FF08B104F09AFE304601F0FBFAE068FFF700F9F8BDC04605
:2025A000CC190020083004404816002068180020012C01000732002070B5164604460D1C01
:2025C00008BF052426D034F07F0001D004F020F9002C18BF032407D155F80C0C18B915F84F
:2025E000020CFF2804D00524284604F031FE11E0012E094805F8024C03D0294602F0ACFE7E
:2026000002E0294604F00EF820464FF40041FCF719FE0024204670BD7018002030B50446ED
:20262000606800252062ADF1140DA5657820A4F84C0094F82C0025650F2807D004F12C0170
:2026400020460122F7F77AF808B116E0284694F83C10FF2901D1A16D21B104F13C0120462A
:20266000FBF70EFC48B92B4601208DF80C30032101AA00902046F1F7FDFA05B030BD70470D
:20268000F8B5044605F0F8F801F030FD071C04D105F02AF86FF003041DE004F05DFA054638
:2026A0000E480022183030F80C6F56B94FF6F871018047600026866022717868A0603446D9
:2026C00006E0521C062AEED305F00EF86FF00304284604F071FC2046F8BDC046A814002088
:2026E0002DE9FC41144C154F06468846700809D320684568002101220B461FFA88F000906A
:202700003846A847B00809D3206845680021022201231FFA88F000903846A847F00809D3B8
:2027200020681FFA88F600210C220223446800963846A047BDE8FC81A401001000A00C409C
:202740000246F8B5084611464C68203821D0401E1CD0401E18BF6FF001001ED18D6805F02A
:20276000DFF80E4E07463068016928688847B0F1FF3FF8D10025A564606C401EE0642565AA
:202780003846A56305F0C8F82846F8BD0021084601E00121002084F82D10F8BDD0010010FA
:2027A00038B5154C04F1180005461C3001F094F803F012FD042003F033FDA07E032801D146
:2027C000607EA0B105F14501E120F6F76BFD05F14601E720F6F766FD084894F85F100078E1
:2027E000884204D005F14701E820F6F75BFD2846FAF746FF38BDC046B83000205F12002078
:2028000038B50120124C114D94F8711085F83D000F2917D00F490870202004F09BFD94F8E0
:2028200071200E490C4835F81220886201F1200091F84010491C5143490001F2A32103F03C
:202840008FFB38BD02F054FD38BDC046F0170020A8110020EC130020B1EB0000243100208B
:2028600070B502460D4632F07F0004D110460022FFF7A2FE70BD04F091FE104908398C78C6
:20288000A5F10C06FF2802D0C96A40184478FF2C02D103F0BDFF0DE0104604F017F9014615
:2028A0002A46FF20B072204602F038FC20B1284604F0CEFC012070BD002070BD701800209B
:2028C0001CB5002922D04C08002948BF494242105440002848BF404200230A1C904201D971
:2028E0005200FBE790425B41904200D3801A914201D25208F6E7191C002C48BF40426400CC
:2029000048BF4942021C081C111C1CBD0123DB0710B1A8BFDB431846FDF77DFB1CBDFEE709
:2029200038B5144DFF2822D0B63D95F8B410012915D1032844F6206416D00F48006890F8C6
:20294000690088B104F076FE0A224FF4FA6390FBF2F15143401A58432418A4B204E0032809
:2029600014BF4FF4FA540024A5F8B64038BD0020288038BDA62E0020640E0020B0B5044655
:2029800004F012FE30F0010008BF6FF004041ED004F072FF054604F0DFF801460D480622B7
:2029A000343030F80C7F6FB1A388BB4208D1406800680022854208BF0122A260002403E0F3
:2029C000521EEED14FF0FF34084604F0F5FA2046B0BDC0468C14002000B5ADF1240DADF863
:2029E0000000ADF80210116801A801605168002241600E490693887D8DF80C200D318DF8B8
:202A00000D000B680DF10E0003604B684360097A017218208DF81C2005498DF81D206A46C2
:202A2000FDF7D4F9C0B209B000BDC04650860100FD59000098B5154B1B1D18680004070C3E
:202A400021D003F0B1F9104991F90720824205DD10F1800FB8BF6FF07F00C8718C88BC4208
:202A600010D80A68D3F8D40F801A801C1F2888BF1F203F1B4008C7404FF6FF70E719B842F4
:202A800038BF071C8F8098BDF43100203010094003B4F0B5144CA0684FF0FF3105AF1D46A0
:202AA0001646ADF11C0D04F023FF396804A80160B988818004A803C8B2B26B46FCF722F854
:202AC00007460A2F02D007B9012704E06846294601F0A8F90746A06804F006FF384607B0A0
:202AE000BDE8F04002B07047481A002008B51348134A14490078801E0A2807D8DFE800F066
:202B00001814100614100614100609C004F0D0FE11E010688008FCD250688008FCD20AE0DD
:202B200008688008FCD306E008688008FCD202E010688008FCD3F6F78BF808BD7810002094
:202B400034600C4038600C40084610B500F0005100F0040008431CD0012002F0B9FF104C0B
:202B6000012811D00B4801683220B0FBF1F2012A8CBFB0FBF1F101218834204604F084FEF2
:202B8000204604F091FE10BD034804F083FC0348046010BD388B01006D350000001004408B
:202BA000980A0020F8B5134C134940F27C622046FCF778FD002102220B46181932278D3030
:202BC00000F8031F41707F1E8170F9D1521E03F19603F2D1094E04F5E2753227284631462D
:202BE000182204F089F918357F1EF7D10220A070F8BDC046A821002054790100187B01003B
:202C000070B5134C6068804712490025064648784D70A168820808D2C00816D330468847F5
:202C200028460146F4F766FF70BD304688470A480078012803D001202946F4F75BFF6068BA
:202C400080470646FAF7ECFDA1683046884770BD8C140020CC190020E81A00201549096856
:202C600021280ADC212819D00C380FD00D380FD0001F0FD0C01E0FD01AE0253810D0001F9B
:202C800010D0401E10D0401E10D011E0086870474868704788687047C868704708697047A3
:202CA0004869704788697047C8697047086A704700207047F0010020F8B50646B08815467F
:202CC0000F46FDF737F80446002D02D4281B0A2806DB3368291B38460BA201F05BFB04196B
:202CE000B08978B1002D06D4B06804F051FA291B401D884206DCB368291B384603A201F054
:202D000049FB04192046F8BD257000C02827257327290000F8B50746C81D01F00705C610F9
:202D2000002F4FF0010000FA05F0A0F1010C14BF0029002019D00020BEB17F1E33460246A5
:202D4000941B17F8011FB4F1FF3F08D10DB10CEA010104E001F1FF04401C2140C0B20029F2
:202D6000F8D15B1E02F10102EAD1F8BD38B50C4620B141680122A240114201D1022038BDB1
:202D8000914341600E480025231800EB8401C1F8945003F140010978FF291ABF406850F854
:202DA000211044F020410548FAF79EF820464FF0FF3103F08FFD284638BDC046007FC7670F
:202DC000542B002010B5144CE2685168496839B110B102F093FEE268506840688047E26892
:202DE0005268916809B9D06880B1094B18680028FCD00020186019B108468047E0684268C4
:202E0000D06800B18047034802F0E2FF10BDC0461C10044001000706700A0020144BB0B535
:202E2000997B03EB81010A69017801F07F014D000170AC185219527803EB82052F6907B135
:202E40009A732278141103EB84031F6C2FB90C290CDA1821FDF704F8B0BD02F00F0257F8BB
:202E6000221011B904F02EFAB0BD8847B0BDC0461415002038B50546012001F01BFE124C81
:202E80002046143000F028FD288900280CBFEB200020687094F83F00C10824BF00F0FB006A
:202EA00084F83F0080080BD394F83F0000F0FD0084F83F00297C6878C1F3001103F098FFAA
:202EC000284604F03FFA38BD403000202DE9F0410120114E114D307028781F469046022808
:202EE00001D004F0EFF90024022104EA070001EA0801002808BF002902D104F0E3F907E053
:202F0000074991F90000401E08702C7003F0C4FF3470BDE8F081C046E81A0020E91A0020AA
:202F2000D11A00202DE9F041054612480E46002100782960012802D00120F4F7DBFD0E4CEB
:202F4000606880473768804630463FB16A687968914203DC38463F68002FF8D10560306898
:202F60002F60854201D1FDF7F5F9A16840468847BDE8F081E81A00208C140020134A38B5A7
:202F8000B2F8AC504FF6FF71A9421BD00024012000FA04F32B4212D05940B2F8AC300C4D03
:202FA0001940A2F8AC10291D0A6804F10C03984010430860022003F0D3FC204638BD641C54
:202FC0000F2CE5DB6FF0010038BDC046700A00200810044038B5044604F0A2FC0546114838
:202FE000D43890F8AF10C90803D390F8AE10A14214D0B0F8AC30012101FA04F21A430A4B81
:20300000A0F8AC20181D026804F10C0399408A430260006810B9022001F0CEF8284604F035
:203020007BFC38BD440B00200810044038B5044642F209000DF1020100F0C4FC9DF802009D
:2030400050B19DF8020002281AD1A08894F82710FEF78BFC054606E042F20D00694600F04B
:20306000B1FC9DF80050284600F00EFC0020A4F87C5094F82130607013B1102004F072F9CE
:2030800038BD38B5046845682068002808BF4FF0FF301FD004F044FC2168002954BF491E01
:2030A0000021216004F038FC206890B904F12C0004F0B6FB04F1480004F0AAFB04F1640080
:2030C00004F0A6FB6868FAF779FC04F1180003F049FA002038BDFEE72DE9B841124C054630
:2030E000201D00688047804603F0BCF96F7E002F08BF6B6807D069682A69AF68091A521861
:20310000B9180B466960E968286105F11402184602F01EF8012768686F76A168A860404604
:203120008847BDE8B881C0468C140020D0B5044604F0A2FB02F03AFA061C08BF6FF004004A
:203140001DD003F009FDB168002908BF002709D051F80C2C0023B2600F4641F80C3CFF26CF
:2031600001F8026C03F028FFA7603FB117F8080C207117F8070CA0710020D0BD0220D0BD94
:2031800010B504F0CDFB104C217829B10F490C6804F0C2FB204610BD04F0BEFB03F076FF1A
:2031A0000B4A002303F0CCFEA26B002314001B184FF07A024FF0905044EB0104C11842EB4F
:2031C00004021046001C10BD700A00200430044000093D00B0B5134C6068628800B325887C
:2031E0000021AA42C8BF01210B46AA42C6BFA91A01F58061A91A8FB28FB1012B03D0A118C1
:203200003A46083109E0A118C2F58062083104F002FA606804F108012A4604F0FCF965808D
:20322000B0BDC04664060020012838B51ED1012002F04EFC01281BD003F062FD0E4D0D4C15
:20324000012105F1E000017020683222B2FBF0F404B90C463035284603F024FA28462146D0
:2032600004F012FB284604F01FFB01E001F0A4FF002038BD388B0100940F002038B5124879
:20328000104C0168114D0C40E1430160A10907D34068800904D328464FF4005103F074FE47
:2032A00014F4602F0DD02846D43800F1A8010A6804F4602400F5847014430C60002103F0D8
:2032C00063FE38BD20000E0008100440440B0020134910B5044691F83F00ADF1180D40F079
:2032E000020081F83F00012003F06CF9607890B9211D02A803F064FC03F06EFD0146012079
:20330000009004F110030193E38902AA0520F4F717FA607010B1002103F06AFD06B010BDB9
:20332000403000201FB5014604208DF8000048788DF80100B1F896000DF10203ADF80C0000
:203340008C31184603F03CFC02F0CEFD60B14FF6FF7453200DF10E01ADF80E40F5F7A2FFA1
:20336000044920460A3108806846FAF789F900901FBDC04622120020C8B5071C01D103F08B
:20338000A1FF79684878C6111FD03B89F96400204A78C2F3C3020F2A09D00A781018801C51
:2033A00080B25218834202F10201F1DC01E0801C80B2834206DB79683E8941187960311A6F
:2033C000398100E00020A7F85000C8BD10B5044600211C22ADF1200D6846FDF7CEFC607842
:2033E0008DF80000A0788DF80100E0788DF8020020791122611D8DF8030001A8FCF752F912
:20340000A07D8DF8150008B1A06906900348006881696846884708B010BDC0461C1A0020A2
:20342000F8B504460D46084611220021FDF7A5FC94F800C0BCF1000F1AD0641C00214FF039
:20344000010EE078A37843EA0023207809E0C610AF5D00F00702401C0EFA02F2C0B23A43F7
:20346000AA558342F3DA491C241DC9B28C45E8DCF8BD80B502465378107840EA0320C71359
:203480000F7007BFC0F3062300F0FF00C0F3C323C0F30A004B70802848800DDA02280BDBA4
:2034A000012B0CD0022B0AD0042B08D0052B06D0062B04D0072B02D00022104600E0921CE1
:2034C0004A6080BDDCB5044604F0D6F902F06EF8064604F069F830F0010014BF002E6FF0ED
:2034E000040017D0606858B1B0F1FF3F05D0694602F044F830B107460BE04FF0FF3000E018
:20350000002000907068009904F0F2F9002700B901273846DCBD704770B5114C2068E8B132
:20352000104D686880470646216894F82F00022806DBA96830468847F120F5F779FF70BD04
:2035400004F1240003F06EF8002394F82F00A9682360401C84F82F003046884770BDC04608
:20356000640E00208C14002038B5044642F208000DF1020100F026FA9DF8020040B19DF858
:203580000200022817D1204601F048FB054606E042F20C00694600F015FA9DF8005094F8ED
:2035A000200030B9284600F06FF9A4F87C50002000E00120207038BDF8B5114C60680D4609
:2035C0008047104A8446A16892F82C70106B9FB1002420382030867F56B1C27F954207D13E
:2035E00000228277FF22C277604688472046F8BD7F1E04F10104EDD160468847FF20F8BD28
:203600008C140020AC2E0020F0B5124D00260C460746ADF1140DC5F8B061012004F052F83B
:203620002868C00FF9D3286A0090686A0190A86A0290E86A03903FB13846694611F8012BFF
:20364000401E04F8012BF9D1032005B0C5F838023046F0BD504502402DE9FE431F1C144665
:203660000D4680461BD0DFF83C90082FACBF08263E1C09F10200007829466B46324603F07A
:2036800092FA404621466B463246FDF79FFFBF1BBFB230197319002F84B29DB2E5D1BDE8C7
:2036A000FE83C046481A002003B4B0B5114C04F1080000684FF0FF3104AFADF1180D04F04A
:2036C00017F9396804A80160B988818004A803C800226B46FBF716FA00280CBFBDF80C509A
:2036E0000025A06804F000F9284606B0BDE8B04002B07047481A00201249D0B524310F6860
:20370000ADF1180DCFB17E69BEB1B0B106218DF810100226ADF812600024ADF814404388BC
:20372000ADF8003042680192816802917C6904AE96E803000C226B46A047032003F08CFA81
:2037400006B0D0BDA41000201048114908B54FF42372FBF7A7FF4FF00451002081F89003B3
:20376000012081F87903022081F87503032081F87703042081F8AE03052081F8AB0306204A
:2037800081F881030348C1F8C00308BD1C0400213C000000BD05002110B50446012001F01F
:2037A00089F92078212804BFEB2060700D4991F83F00C20824BF20F0040081F83F008008E9
:2037C00005D22B2020702046FFF728FB10BD91F83F0000F0FD0081F83F006078002103F092
:2037E00007FB10BD4030002070B5114D95F87100B5F896400F2810D00E483430066801F036
:2038000097FB2018864208D895F871104FF4707088402418A41B04F57074044D284600F0B6
:203820005BF82146284603F043F970BD54300020A8110020F0170020114898B50121017027
:20384000022111400F4A4FF0E0471F40002F08BF002903D092F90010491E1170044692F98C
:20386000000030B192F90000002806DC03F02AFD03E000200146F4F73DF90020207098BD48
:20388000E81A0020D11A0020B0B50546802D01DD03F018FD0D4C606880470D4B0D490A4ACE
:2038A0001F780A390D701FB91778A1682FB907E01778A16837F07F0702D088470120B0BDFE
:2038C0008847FDF7A5FFB0BD083200208C140020241400209419002070B505460F48007896
:2038E000012803D001200021F4F704F90C4C201D006880470B49064628460B4602F05CFF32
:2039000018B9191D284602F057FF1869A84201D1FCF720FDA1683046884770BDE81A002000
:203920008C140020281A002070B540680C46054600F5847002F0B6FE0D482A7F0168687F1E
:203940008018AA69C01D80B244430A4805F584766043B0FBF2F008186330B0FBF1F1491C0B
:20396000304603F091FF304603F09EFF70BDC046388B010040420F000F4838B50078C8B18B
:203980000E4D0F4C95F82E106420503C4843206604F15C00FFF7A0FBE08EE26B95F82E101D
:2039A000401C80B28918E08600B900210020E16300F0F0F938BDC04635120020382F002072
:2039C000402E0020F8B50E4602F013FF05464FF6FF70A84208BF682013D00B4C6068804753
:2039E00008490A4B0746680000EBC50008180278991842783046FBF755FEA16838468847A6
:203A00000020F8BD588001008C140020382F0020B0B5054603F030FF044603F0C5FD30F0C0
:203A2000010008BF6FF0040414D003F095F80A4A002132F80C7F4FB153681B689C4204BFEA
:203A40002971002404D0491C0629F2D36FF0040403F0B2FA2046B0BDC014002070B5114C2C
:203A60000546E01C0078FE28AEBF0126401CC6B203219622284603F04DFC022101222846BF
:203A800003F048FC01212846324603F043FC0021A522284603F03EFC607908B9A570E6702D
:203AA00070BDC046481A0020104938B54A39C9690C692579002101E0491CC9B28D42D8BFFB
:203AC0004FF6FF7010DD23680A4602EB82029B1893F900209042EFD105490839C87803EB4B
:203AE0004003B3F80100C88038BDC046721600209019002038B5EB2003F06FF80D48002557
:203B000005700B480078862802D1284600F064F8094C6068804709490C39CA6913681D7173
:203B20001268CA61A168884702F0FAFF38BDC04608320020063200208C1400209C310020C3
:203B400038B50D4C6068804705460C48007870B90B48007830F07F0009D10A48007830B959
:203B60000948007830F07F0001D103F0C9FDA1682846884738BDC0468C14002005320020FA
:203B8000043200200632002008320020F8B506460F4800680D4CC06B80476168401A21785E
:203BA0008900B0FBF1F0B04201D303F08BFB094D243D686880470746A6603046FDF706FAA6
:203BC000F9F72EFEA96838468847F8BDCC19002048160020B014002038B50F49104C088D19
:203BE000401C08856068804705460C480178862903D0A1682846884738BD8721017003F06C
:203C0000BBFCA16828468847082002F009FBE920FCF728FC38BDC046C81800200832002014
:203C20008C140020F8B506460F4D104F7388002417E0A00000EBC400321851689068D26876
:203C400052B9AF420BD00A7855F822200346491C08461946904701E0FBF724FD7388641CDB
:203C6000A4B2A342E5DCF8BD000E00000C0E0000F8B5034600208C460446074613E01CF8E5
:203C8000015B082685F0010101F001014018C0B2411E994206D0641C761E4FEA6505E4B209
:203CA000F0D100E00127A24203DC27B903F03AFD01E0002FE3D02046F8BD3EB5054615F845
:203CC000060C03281DD12B681869009058690190986902906C6859689A681868DB68A047EF
:203CE0002968086015F8080C01F098FD0446012002F0BAFA011C04D0422008702046FEF7ED
:203D0000AFFD3EBD2DE9F04117468846064603F03FFA0D4C0546002128222046FDF72DF884
:203D200031462A462046FBF7BDFC40463A46291900F0E4F8204602F05DFF02A002F05AFFD6
:203D4000BDE8F0810D0A00C06831002038B50446642C13DA0D4D686880470246694672208F
:203D600002F00EF80099E00000EB04104018A9680090104688470098001D38BD0448643C1F
:203D8000E1B2383000EBC10038BDC0468C140020AC2E002070B50F4C05462179E079814246
:203DA00017DD6179A94214DDA3680B4E23B1294632469847E0796179A07101FB0050216842
:203DC00000EB800009180878E071D1F801103046884770BD78160020242E0020F8B502F07B
:203DE000CDFC0D4607463A2F08BFF42012D00B4C606880470646BA0007480949835C801830
:203E000042784E39C918284603F076F8A168304688470020F8BDC046308201008C14002015
:203E20005A120020FEB505460F4CA889E2880F46411D8EB2A178B218B2F5805F0BDD084670
:203E40000021F3F7A9F8864203DD607900B90520FEBDA889A1780090002228460197134641
:203E6000F8F7B4F86079FEBD481A002038B50D460E49144660390A68AA4205D901EB850159
:203E8000D1F89410884201D0022038BD03F048FD074B103B1A68AC400121A9408A43144391
:203EA0001C6003F039FD002038BDC046B42B0020E020024070B50E46144605460823002197
:203EC0002422ADF1280D684603F0EAFC002006900590ADF81000084800684FF47A716B46AB
:203EE000B1FBF0F080B2314604FB00F2284603F0D3FC28460AB070BD388B0100FEB5074653
:203F0000052400266B4697FBF2F05043381AC0B20A28ACBF372530254019187097FBF2F52E
:203F2000AFB22FB1641E03F1010306F10106EAD1761C13F80109761E01F8010BF9D10020E3
:203F40000870FEBD10B50F4C94F83F00ADF1180DB0B940F0010084F83F00012002F032FBEB
:203F600002A801F0D5FF343401200090064B019403F18A000388032102AA0520F3F7E0FB10
:203F800006B010BD40300020A81100200E4808B50178081C05D0401E12D0801E01280FD9C1
:203FA00008BD03F0A5F838B10948084900680968884238BF002004D31C20FCF753FA08BD4F
:203FC0000846F0F7CDFC08BDCA180020600D0020D01900201FB5144600900A79487940EA5A
:203FE00002208A7942EA0022C87940EA022001900A78487840EA02208A7842EA0022C87812
:2040000040EA02200290684600F028FAB0FBF4F16143401AC0B200901FBDF8B5051C0E4674
:2040200006AF04D0012D0CBF0624002400E002240EB9A41CA4B2012A06D0022A0ED15889E0
:20404000C01D04EBE00008E03878002814BF022101210020FAF758FE001984B22046F8BD0B
:204060002DE9F04115468046287840F0C000287028790C4604262F1D40F00200287117F86D
:2040800001293119404689B203F044F9761EF6D52A79241D4046A1B202F0FD022A7103F020
:2040A00039F9BDE8F08100000F4800B50068ADF1240D69466C30F8F78DF810B99DF80B004D
:2040C00008B900200DE0684601F099FF9DF808104FF47A73B0FBF1F24A43801A091A03FB28
:2040E00001F009B000BDC046640E002070B5054602F032FD0D4C0221064654F80C0F58B9F0
:20410000002025600146A0600A4603F0C1FB606038B903F0E9FA04E0A84202D0491EECD169
:204120000024304602F048FF204670BDA814002038B505460C4600200090042C0BD3241FB2
:20414000284604226B46A4B2214602F02CFD0098B0F1FF3FF1D001210A4600F0FF03FF2B7C
:2041600018BF111C000A521C0090042AF5DD091988B238BD2DE9F04103F022FA0D4D603D95
:204180002B688046A3B105F194060024012707FA04F018EA000F07D056F8240020B102680C
:2041A00012B1214690472B68641CE4B29C42EED3BDE8F081B42B002010B5044603F0B0FBF4
:2041C0000C4A117819B903F0A7FB822010BD11460B7884F0FF0213400B70097811B103F0D7
:2041E0009BFB05E003F098FB0348082102F0CCFE002010BDFE310020440B002038B50D46A3
:20420000044603F093FA6368A1688B4204D103F083FB4FF0FF3038BDE168491CB1FBF3F24B
:204220005A432368891ACD54E1606269A168491C8A42A16038BF616103F06EFBA06838BD39
:204240000C4885460C4885446F4607208743BD460A486F4607600A48002803D07946491D99
:204260008E460047FBF730F902F05EFE03F0C4FAFEE7C046004B002000050000D81A00209C
:20428000CD7501000F48B0B507680025ADF1180DADF8105097B106208DF808000223ADF8FE
:2042A0000A30ADF80C5004AC00943C6902AA92E803002A46A04708B1ADF81050BDF81000D7
:2042C00006B0B0BDC810002010B50446012000F0F1FB2078212804BFEB2060700A4991F85C
:2042E0003F00C20824BF20F0040081F83F00800809D391F83F0000F0FD0081F83F0060785D
:20430000002102F075FD10BD4030002030B50E4D95F87100ADF1AC0D0F280CD10B4C343C4B
:2043200004F11400FFF7D8FAB5F8961004F1140002F0BEFB05E02F208DF800006846FEF749
:204340006DFD2BB030BDC046A81100207430002038B50F4C0546204603F0C0F8A8B920461D
:2043600003F0E6F90446A068054209D0E3682269284600219847002818BF4FF0FF3005D172
:20438000204603F0D7F9041CEDD1002038BDC046940F00200CB4F0B505AF061C0C4627F094
:2043A0000303ADF1040D03F1040304D03068002818BF051C00D100253A68284602F0FAFFD0
:2043C000844238BF601E15B131684118316001B0BDE8F04002B07047D0B504463C20FCF74C
:2043E00085F8071C14D000213C22082303F034FA207AB86160893862E06838616068394610
:20440000002203F0FDF90646384601F009FB16B96FF00300D0BD0020D0BD08B50B4602F067
:20442000C3FC5989418199898181997B8173D97BC173197C002201B10122597C417459698D
:204440004161197E0274002201B10122027603F119010B221930FBF725F908BD4168826852
:204460000D4B0068C91AD21AC01A4A40A2EBB1425040A0EB72504140A1EBF0114A40A2EBC7
:2044800031425040A0EB32704140A1EBB04181EA0200A0EB31207047054152210B4A08B523
:2044A00002F10C000068C00A01D200F0F1FB10684008FCD3064800684168022088470549EF
:2044C0000A6882420CBF0448086008BD08800240CC01001024280020EFBEADDE10B5082129
:2044E000ADF1180DADF800100A4C04901B21ADF80210606A02900121019105490648039127
:204500000168684688470299616206B010BDC046315C010068180020B014002010B5ADF159
:20452000180D0C4C01900A4808210390002004902069ADF800101B2102900748ADF8021099
:204540000168684688470299216106B010BDC046ED570100CC190020B01400200D4808B58F
:204560000068020F0C48036803F0FF03802B28BF002302F077F901464FF0FF30012907D140
:20458000111C04D0891E04BF143358B208BD0A2008BDC04618130050A0100050D0B50E4C4B
:2045A0000646A0684FF0FF3103F0A2F9277977B9E088C0F5805000B2864203DC002E18BF8F
:2045C000042704D1A0780021F2F7E6FC6779A06803F08AF93846D0BD481A00200E4938B5A8
:2045E000CA68824210D1087801280DD103F098F90546084801F0ECFB0446284603F08CF936
:2046000004F0FF00012802D06FF07F0038BD4FFAA4F038BD01000304700A0020B0B503F00D
:2046200085F805460A48017801290DD00121094F0170387840B1084C0746206881682046DC
:2046400088470C347F1EF8D1284603F065F9B0BDD31A00201C8B0100B88A01000B4B80B536
:204660001F7800227FB10A4B1B7883420BDD8A4208BF0849084F820002EBC002B818026816
:20468000D26890470246104680BDC046D31A00201C8B0100B8890100B88A010030B50E4DAE
:2046A0002868ADF1240DA0B10024FFF7F7FE04EB0D020021CB00491C20FA03F3042902F8B5
:2046C000013BF7DB241DE4B2202CEEDB29686846884709B030BDC046D41A002010B5044609
:2046E000012000F0E7F9EB200B49607091F83F00C20824BF20F0040081F83F00800809D3F5
:2047000091F83F0000F0FD0081F83F006078002102F06EFB10BDC0464030002008B5642034
:204720006946FFF75BFB0A490A48C1F8D8000A48C1F8DC009DF8000000280CBF49F24E0050
:2047400047F60E20C1F88000C1F8C00008BDC046280D0020AC31002058160020F8B5071CC1
:2047600001D102F0AFFD0C4C201D006880473E6805465EB107498A68A6F10C00964204BF85
:2047800000228A600021396001F00CFEA16828468847F8BD141500208C14002038B50E4B0E
:2047A00005460C46281D03F1480102F039FF188F2880B3F8460003F13E016880201D02F026
:2047C0002FFF93F83A00207300206073188F2080988F608038BDC046481300201CB50A1CA5
:2047E00017D000230124E407A04238BF041C944201D95200FBE790425B41904228BF801A01
:20480000914201D25208F6E7191C021C081C111C1CBD00B1C843FBF7FEFB1CBDB0B50D4606
:20482000044602F083FFA76897B121692268515C297063682169A768491CB1FBF3F25A4312
:20484000891A2161791EA16003F066F8A068B0BD03F062F84FF0FF30B0BD00000D4910B592
:2048600009780446A1B1617871B9217839B194F8201021B9FEF778FE0020207010BD94F88B
